:100000000C9434280C9465280C9465280C9465286D
:100010000C9465280C9465280C9465280C9465282C
:100020000C9465280C9465280C9465280C9465281C
:100030000C9465280C944AD90C9465280C94652876
:100040000C9465280C94DA7A0C9465280C94652835
:100050000C9465280C9465280C9441600C94ADD4E4
:100060000C9465280C942C880C9465280C946528B5
:100070000C9465280C9465280C9465280C946528CC
:100080000C9465280C9465280C9465280C946528BC
:100090000C9465280C9465280C9465280C946528AC
:1000A0000C9465280C9465280C9465280C9465289C
:1000B0000C9465280C9465280C9465280C9465288C
:1000C0000C9465280C9465280C9465280C9465287C
:1000D0000C9465280C9465280C9465280C9465286C
:1000E0000C946528CD59D059BF59C359C959075ADD
:1000F000D459D859DE59E259E659EC59F059F45916
:10010000075AFA59FE59025ABF5AC45AC95AD35A01
:10011000DD5A565BE75AEF5AF75A015B0B5B155BEA
:10012000245B2E5B565B385B425B4C5B084AD73BDB
:100130003BCE016E84BCBFFDC12F3D6C74319ABDB6
:1001400056833DDA3D00C77F11BED9E4BB4C3E91DA
:100150006BAAAABE000000803F05A84CCDB2D44EC9
:10016000B93836A9020C50B9918688083CA6AAAACB
:100170002ABE000000803F004E414E494E4954596E
:10018000494E46CDCCCC3D0AD7233C17B7D1387762
:10019000CC2B329595E6241FB14F0A000020410078
:1001A00000C84200401C4620BCBE4CCA1B0E5AAEC2
:1001B000C59D74434F4D4D554E49434154494F4E93
:1001C0000044525952554E004552524F5253004925
:1001D0004E464F004543484F0020746F6F206C6FB0
:1001E0006E6720657874727573696F6E20707265C2
:1001F00076656E7465640A0020636F6C64206578B0
:1002000074727573696F6E2070726576656E746551
:10021000640A0047322F47332062616420706172A4
:10022000616D65746572730A00536C6565702E2E7E
:100230002E00205A3A200020593A200042656420BE
:10024000583A20004368656170334420563330309B
:100250002072656164792E00526573756D696E67F1
:10026000207072696E7400436C69636B20746F2038
:10027000726573756D652E2E2E004E6F206D6F7634
:10028000652E00456E642066696C65206C69737428
:100290000A00426567696E2066696C65206C697347
:1002A000740A005344207072696E74696E6720622C
:1002B00079746520004E6F74205344207072696E0B
:1002C00074696E670A0046696C652064656C6574C4
:1002D00065643A0044656C6574696F6E2066616997
:1002E0006C65642C2046696C653A20006F70656E01
:1002F000206661696C65642C2046696C653A200053
:100300002569730025696D202569730025696820BA
:1003100025696D2025697300256964202569682099
:1003200025696D2025697300256979202569642078
:100330002569682025696D20256973005072696EF2
:10034000742074696D653A200050726F746563742F
:1003500065642050696E0A004525692025730043B5
:1003600068656170334420563330302072656164B3
:10037000792E00D401CF01C801C101B3016F6666B7
:100380000044454255473A004B494C4C45442E20C9
:10039000004D3131332053006F6B00486561746943
:1003A0006E6720646F6E652E003F0A0020573A008A
:1003B00045256920257300436865617033442056E4
:1003C0003330302072656164792E004265642064A8
:1003D0006F6E652E003F0A0020573A004265642088
:1003E00048656174696E672E0043686561703344C7
:1003F0002056333030204F66662E00563330302082
:100400004C312050494420423A312054303A312076
:1004100054313A30204649524D574152455F4E4182
:100420004D453A4D61726C696E20312E312E30206F
:10043000284769746875622920534F555243455FB8
:10044000434F44455F55524C3A68747470733A2F69
:100450002F6769746875622E636F6D2F4D61726CC2
:10046000696E4669726D776172652F4D61726C6954
:100470006E2050524F544F434F4C5F564552534994
:100480004F4E3A312E30204D414348494E455F543E
:100490005950453A436865617033442056333030D3
:1004A0002045585452554445525F434F554E543A97
:1004B0003120555549443A63656465326132662D91
:1004C000343161322D343734382D396231322D6375
:1004D00035356336326633363766660A007A5F6DC5
:1004E000696E3A2000795F6D696E3A2000785F6D21
:1004F000696E3A20005265706F7274696E6720658C
:100500006E6473746F70207374617475730A004D38
:1005100031343520533C696E6465783E206F7574C4
:10052000206F662072616E67652028302D31290AA0
:100530000053657474696E672054726176656C202F
:10054000416363656C65726174696F6E3A20005334
:10055000657474696E6720526574726163742041BA
:100560006363656C65726174696F6E3A20005365F0
:100570007474696E67205072696E7420416363659C
:100580006C65726174696F6E3A20005365747469AA
:100590006E67205072696E7420616E6420547261BF
:1005A00076656C20416363656C65726174696F6E1A
:1005B0003A2000205A00205900580020204D617830
:1005C0003A2000205A00205900580020204D696E22
:1005D0003A20004F6E20004F666600536F6674200D
:1005E000656E6473746F70733A200020643A002063
:1005F000693A0020703A004F666673657473206133
:1006000070706C696564004572723A20546F6F2097
:100610006661722100546F6F206661722066726F8E
:100620006D207265666572656E636520706F696EB8
:10063000740A00454550524F4D2064697361626CE5
:1006400065640A003A20007A5F6D696E3A20202DB9
:100650003230207A5F6D61783A20203230005A20A3
:100660004F666673657420004E6F2063617365206A
:100670006C696768740A004163746976652045781F
:100680007472756465723A2000556E6B6E6F776E8A
:1006900020636F6D6D616E643A2022004861726460
:1006A000636F6465642044656661756C742053658E
:1006B0007474696E6773204C6F616465640A00200E
:1006C000204D383531205A005A2D50726F62652006
:1006D0004F666673657420286D6D293A0A002044C0
:1006E0000020490020204D333034205000204400A9
:1006F00020490020204D3330312050005049442003
:1007000073657474696E67733A0A0020460020426C
:100710000020480020204D3134352053004D6174B5
:10072000657269616C2068656174757020706172B2
:10073000616D65746572733A0A00205A0020590091
:1007400020204D323036205800486F6D65206F668E
:10075000667365743A0A00204500205A002059004B
:1007600020580020420020540020204D32303520F7
:100770005300416476616E6365643A20533C6D6951
:100780006E5F66656564726174653E20543C6D6998
:100790006E5F74726176656C5F66656564726174C4
:1007A000653E20423C6D696E5F7365676D656E7472
:1007B0005F74696D655F6D733E20583C6D61785F55
:1007C00078795F6A65726B3E205A3C6D61785F7A1A
:1007D0005F6A65726B3E20453C6D61785F655F6A5C
:1007E00065726B3E0A0020540020520020204D32DA
:1007F0003034205000416363656C65726174696FC9
:100800006E2028756E6974732F7332293A20503C1C
:100810007072696E745F616363656C3E20523C72F6
:100820006574726163745F616363656C3E20543C00
:1008300074726176656C5F616363656C3E0A00206B
:100840004500205A0020590020204D3230312058D8
:10085000004D6178696D756D20416363656C6572EB
:100860006174696F6E2028756E6974732F733229F5
:100870003A0A00204500205A0020590020204D321D
:1008800030332058004D6178696D756D206665655F
:100890006472617465732028756E6974732F73298F
:1008A0003A0A00204500205A0020590020204D39E6
:1008B0003220580053746570732070657220756E15
:1008C00069743A0A0020204D3230302044300A004A
:1008D00020204D3230302044002044697361626C26
:1008E00065640A0046696C616D656E742073657499
:1008F00074696E67733A002020473231203B2055DF
:100900006E69747320696E206D6D0A0A0025753A50
:100910002530327500253032753A25303275002584
:10092000756420253032753A25303275005A0059E9
:100930000058000920000000000000000000000036
:1009400000007FFFE0000000000000000000000049
:10095000007000E000000000000000000000000047
:1009600061F860000000000000000000000000418D
:10097000F82000000000000000000000000040F02F
:100980002000000000000000000000000040602087
:100990000000000000000000000000005801A07FDF
:1009A00080000000000000004104005C63A0FFC064
:1009B000000000000000002082005EF7A0FFC000E1
:1009C0000000000000002082005EF7A0FFC00000D1
:1009D00000000000004104005C63A07F8000000074
:1009E000000000008208005801A07F800000000085
:1009F000000001041000406020FFC0000000000063
:100A0000000104100040F020FFC0000000000000C2
:100A10000082080041F820FFC00000000000000034
:100A200041040061F8603F00000000000000000089
:100A300000007000E01E0000000000000001FFFF49
:100A4000807FFFE00C0000000000000001FFFF803D
:100A50000000000000000000000000000000007F17
:100A6000FFE0000000000000000000000000700037
:100A7000E0000000000000000000000000630C60C7
:100A8000000000000000000000000000470E2000F1
:100A900000000000000000000000004F0F200000D8
:100AA000000000000000000000005F0FA000000038
:100AB0000000000000000000005E07A07F80000032
:100AC0000000000000410400406020FFC000000062
:100AD0000000000020820040F020FFC00000000065
:100AE00000000020820040F020FFC0000000000055
:100AF00000004104004060207F80000000000000F2
:100B0000008208005E07A07F800000000000000156
:100B10000410005F0FA0FFC00000000000000104EF
:100B200010004F0F20FFC0000000000000008208EE
:100B300000470E20FFC0000000000000004104003C
:100B4000630C603F00000000000000000000007027
:100B500000E01E0000000000000001FFFF807FFF9A
:100B6000E00C0000000000000001FFFF800000001A
:100B70005072696E742061626F72746564004E6FAA
:100B80002053442063617264005072696E74206661
:100B9000726F6D2053440053746F70207072696ED1
:100BA0007400526573756D65207072696E740050C3
:100BB00061757365207072696E7400436F6E747234
:100BC0006F6C00507265706172650054756E6500DF
:100BD000496E666F2073637265656E0000060900DA
:100BE000FE000000000001090008FE0000050808E2
:100BF00006000040F0C888889878100508080600AC
:100C000000C0F88888888888F80505050600012056
:100C100030F830200508080600002070F820202059
:100C200020E00509090600FF2070A8A8B888887090
:100C3000200509090600FFE080C0B0A82830282858
:100C40000509090600FFF8A88888888888A8F8059B
:100C50000A0A0600FE205050505088A8A888700349
:100C6000030306000340A0400000210024002700E9
:100C70002A002D00300033000101000004010701AB
:100C80000A0100002200250028002B002E00310060
:100C9000340002010000050108010B0100002000E2
:100CA0002300260029002C002F0032000001000044
:100CB00003010601090105050505070508080808DF
:100CC000020202020A0A08080404040401010101E4
:100CD00001010101030303030303030304070707DF
:100CE0000C0C0C0C0C0C0C0C020202020606060684
:100CF000060606060B0B0B0B0B0B0B0B0102102051
:100D00002008081020401020408002010201080441
:100D100002010102040810204080804020100804D5
:100D2000020180040201804020100804020108042E
:100D30000201010204081020408001020408102072
:100D4000408000000A0B02090C0D0E080703040185
:100D50000000000000000000000000000000000093
:100D60000000000000000000000000000000121160
:100D70001000000000000000000000000000000063
:100D800000000000000000004B494C4C45442E2060
:100D900000202D20496E76616C696420657874723C
:100DA00075646572206E756D62657220210A00207F
:100DB00020506C616E6E657242756666657242792E
:100DC0007465733A20002046726565204D656D6F2D
:100DD00072793A2000436F6D70696C65643A204DFA
:100DE000617920313920323031370A00207C2041AE
:100DF0007574686F723A20286E6F6E652C2064657A
:100E00006661756C7420636F6E666967290A0032CB
:100E10003031372D30352D30342031323A303000FA
:100E2000204C61737420557064617465643A2000CD
:100E3000312E312E300A004D61726C696E002053E4
:100E40006F6674776172652052657365740A00205D
:100E50005761746368646F672052657365740A0034
:100E60002042726F776E206F7574205265736574BF
:100E70000A002045787465726E616C205265736556
:100E8000740A00506F77657255700A00737461724E
:100E9000740A006572726F722077726974696E6786
:100EA00020746F2066696C650A00456E6473746F08
:100EB000707320256320256320256320256300208F
:100EC0005A3A0020593A0020583A00656E6473740B
:100ED0006F7073206869743A2000446F6E652073E8
:100EE0006176696E672066696C652E0A004D32393D
:100EF0000070012C0190012701B0012201C0011DE9
:100F000001F00118011002130130020E0160020904
:100F10000190020401C002FF000003FA004003F543
:100F2000008003F000D003EB002004E6007004E131
:100F300000E004DC004005D700C005D2004006CD2B
:100F400000D006C8008007C3003008BE00F008B912
:100F500000C009B400B00AAF00B00BAA00D00CA5C5
:100F600000000EA000500F9B00C010960050129180
:100F70000000148C00C0158700B0178200B0197DE6
:100F800000D01B7800001E730040206E0090226984
:100F900000F024640040275F0090295A00E02B55A0
:100FA00000102E500020304B0010324600E033413C
:100FB0000090353C001037370070383200A0392DD2
:100FC00000B03A2800A03B2300603C1E00103D19F1
:100FD00000903D1400103E0F00703E0A00C03E0518
:100FE00000003F0000403FFBFF803FF6FFC03FF1A5
:100FF000FF4572723A204D494E54454D50204245AE
:1010000044004572723A204D494E54454D50004DB2
:10101000494E54454D502074726967676572656426
:10102000004572723A204D415854454D502042457A
:1010300044004572723A204D415854454D50004D80
:10104000415854454D5020747269676765726564F4
:10105000001FFFFFFFFFFFFF600000000001FF40D7
:101060000000000000FF8000000000007F83CF0030
:10107000000C303F87FF80000C301F867980000C09
:10108000000F8C30C7838C30E78C30CFC7CC31F366
:101090008C30DCECEC33B98C30D86C6C33198C3080
:1010A000D06C0C33198C30D86C0C33198C30DC6C50
:1010B0000E3B198C30CF7C079F198C30C77C038F77
:1010C0001940000000000002600000000000061F40
:1010D000FFFFFFFFFFF8006000000000006000005D
:1010E000E00000E0000001F80000000001F800034B
:1010F000F80003F8000007FE0000000007FE000FE4
:10110000FE000F1E00001F0F81C000381F0F803F20
:101110000F803E0F80007C03E1C000387C03E0FCC0
:1011200003E0F803E000F000F1C00038F000F1F057
:1011300000F1E000F000C00071C00038C00071C0D4
:101140000071C0007000C00001C00038C003E1C0E1
:101150000031C0003000C00001C00038C00F81C0A5
:101160000031C0003000C00001FFFFF8C07E01FF69
:10117000FC31C0003000C00001FFFFF8C1F001FFEA
:10118000FC31C0003000C00001FFFFF8C7C001FF04
:10119000FC31C0003000C00001C00038FF0001C0B9
:1011A0000031C0003000C00001C00038FC0001C0A8
:1011B0000031C0003000C00031C00038E00031C054
:1011C0000031C0003000E000F1C00038E000F1C0A4
:1011D0000031C00070007C03E1C000387C03E1C036
:1011E0000031F001E0001F0F81C000381F0F81C0E7
:1011F0000031FC07C00007FE0000000007FE0000F1
:101200000001CF0F000001F80000000001F800000D
:101210000001C3FC0000006000000000006000004E
:101220000001C0F00000000000000000000000000D
:10123000000000600000000000000000000000004E
:10124000000000000000000000000000000000009E
:10125000000000000000000000000000000000008E
:10126000000E00001F03000000000000000000004E
:10127000003F80007FC3000000000000000000006D
:1012800000FFE001FBF30000000000000000000090
:1012900003E0F807E0FF000000000000000000008D
:1012A0000F803E1F8E3F0000000000000000000085
:1012B0000E001F9E3F8F0000000000000000000095
:1012C00000001F98FFE30000000000000000000085
:1012D00000007E19FFF30000000000000000000085
:1012E0000001F819FFF300000000000000000000FA
:1012F000000FE019FFF300000000000000000000F4
:10130000001F8019FFF30000000000000000000033
:101310000007E019FFF300000000000000000000DB
:101320000001FC19FFF300000000000000000000B5
:1013300000003F19FFF30000000000000000000063
:101340000C000F9C7FC700000000000000000000A0
:101350000F001F9F1F1F0000000000000000000082
:101360000FC07E0FC07E00000000000000000000E3
:1013700003F1F803F1F80000000000000000000095
:1013800000FFE000FFE0000000000000000000009F
:10139000003F80003F8000000000000000000000CF
:1013A000000E00000E000000000000000000000021
:1013B000000000000000000000000000000000002D
:1013C000000000000000000000000000000000001D
:1013D000000000000000000000000000000000000D
:1013E00000000000000000000000000000000000FD
:1030D00000000000000043616E6E6F7420656E7426
:1030E0006572207375626469723A2000022E2E00A8
:1030F0004D61696E00436172642072656D6F766523
:1031000064004361726420696E7365727465640063
:10311000466C6F7700466C6F770046616E20737067
:103120006565640046616E20737065656400426584
:103130006400426564004E6F7A7A6C65004E6F7A67
:103140007A6C650053706565640053706565640052
:103150004D61696E005072656865617420504C4124
:1031600020426564005072656865617420504C416E
:1031700020456E64005072656865617420504C4152
:1031800000507265706172650050726568656174A7
:103190002041425320426564005072656865617445
:1031A0002041425320456E64005072656865617429
:1031B000204142530050726570617265004D343297
:1031C0003800507265686561742041425300507246
:1031D000656865617420504C4100436F6F6C646F8B
:1031E000776E004D38340044697361626C652073FA
:1031F000746570706572730053657420686F6D65D7
:10320000206F6666736574730047323800417574C9
:103210006F20686F6D65004D6F766520617869730A
:10322000004D61696E004D6F76652058004D6F76D8
:10323000652059004D6F7665205A00457874727587
:10324000646572004D6F766520302E316D6D004DD6
:103250006F766520316D6D004D6F76652031306D74
:103260006D004D6F766520617869730045787472E2
:1032700075646572004D6F7665205A004D6F7665F6
:103280002059004D6F7665205800534420636172C9
:1032900064206F6B0A006F70656E526F6F742066EA
:1032A00061696C65640A00766F6C756D652E696E78
:1032B0006974206661696C65640A00534420696E14
:1032C0006974206661696C0A006175746F25692EE6
:1032D00067004D3234004D32332025730057726938
:1032E00074696E6720746F2066696C653A20006FA0
:1032F00070656E206661696C65642C2046696C653A
:103300003A20006F70656E206661696C65642C20E0
:1033100046696C653A200046696C652073656C658A
:10332000637465640A002053697A653A200046692F
:103330006C65206F70656E65643A20006F70656E15
:10334000206661696C65642C2046696C653A2000D2
:103350002066696C653A20004E6F7720002220704D
:103360006F73002220706172656E743A22005355AB
:1033700042524F5554494E452043414C4C207461B4
:10338000726765743A22004B494C4C45442E20002C
:10339000747279696E6720746F2063616C6C20733E
:1033A00075622D67636F64652066696C657320774D
:1033B00069746820746F6F206D616E79206C65761A
:1033C000656C732E204D4158206C6576656C2069C4
:1033D000733A004572726F723A0024F4D43050C3CD
:1033E0008E20C2A24017828B7011127A910D816CCF
:1033F000D90AA861E108C7586607615143061E4B08
:103400005D05C145A7041A411104093D98037139AE
:1034100031034036DB0265339102D4305402802EF2
:103420001D02632CEE01752AC501B028A0011027EA
:1034300081018F2564012B244B01E0223401AC2152
:103440001F018D200D01801FFC00841EED00971DC3
:10345000DF00B81CD200E61BC600201BBC00641AAB
:10346000B200B219A8000A19A0006A189900D11771
:10347000910040178B00B516840031167E00B315FD
:1034800079003A157300C7146F0058146A00EE13E0
:1034900066008813630025135E00C7125B006C1280
:1034A000570015125400C111510070114F00211125
:1034B0004B00D61049008D10470046104400021002
:1034C0004200C00F4000800F3E00420F3C00060F3C
:1034D0003B00CB0E3800930E37005C0E3500270EF4
:1034E0003400F30D3200C10D3100900D3000600D3D
:1034F0002E00320D2D00050D2C00D90C2B00AE0C2A
:103500002900850C29005C0C2700350C27000E0CC7
:103510002600E80B2400C40B2400A00B23007D0B25
:1035200023005A0B2100390B2100180B2000F80A48
:103530001F00D90A1E00BB0A1E009D0A1D00800A3A
:103540001D00630A1C00470A1B002C0A1B00110AFD
:103550001A00F7091A00DD091900C4091900AB099E
:103560001900920917007B091800630917004C091C
:10357000160036091600200916000A091500F5087C
:103580001500E0081400CC081400B8081400A408C2
:103590001400900813007D0812006B0813005808EF
:1035A0001200460812003408110023081100120806
:1035B000110001081100F0071000E0071000D0070B
:1035C0001000C0071000B0070F00A10710009107FE
:1035D0000E0083070F0074070F0065070E005707E2
:1035E0000E0049070E003B070D002E070E002007B6
:1035F0000D0013070D0006070D00F9060C00ED067F
:103600000D00E0060C00D4060C00C8060C00BC0639
:103610000C00B0060C00A4060B0099060C008D06E9
:103620000B0082060B0077060B006C060B00610690
:103630000A0057060B004C060A0042060A0038062C
:103640000A002E060A0024060A001A060A001006BE
:10365000090007060A00FD050900F4050900EB054D
:103660000900E2050900D9050900D0050900C705D0
:103670000900BE050900B5050800AD050800A5054F
:1036800009009C050800940508008C0508008405C5
:1036900008007C050800740508006C050700650536
:1036A00008005D050700560508004E0507004705A0
:1036B00007004005080038050700310507002A0506
:1036C0000700230507001C050600160507000F0567
:1036D00007000805060002050700FB040600F504C4
:1036E0000700EE040600E8040600E2040700DB041D
:1036F0000600D5040600CF040600C9040600C30472
:103700000600BD040600B7040600B1040500AC04C1
:103710000600A6040600A00405009B04060095040C
:103720000500900406008A04050085040500800455
:1037300006007A04050075040500700405006B049A
:10374000050066040500610405005C0405005704DB
:103750000500520405004D0405004804050043041B
:1037600005003E0404003A04050035040500300459
:1037700004002C04050027040400230405001E0493
:1037800004001A04040016040500110404000D04CA
:103790000400090405000404040000040400FC0300
:1037A0000400F8030400F4030400F0030400EC0335
:1037B0000400E8030400E4030400E0030400DC0365
:1037C0000400D8030400D4030400D0030400CC0395
:1037D0000400C8030300C503030024F404D9201B1C
:1037E000C40C5C0E9804C4095F0265077101F405FE
:1037F000F900FB04B30048048700C10369005803C3
:10380000550003034500BE023A0084023100530212
:103810002A002902250004022000E4011C00C8013E
:103820001900AF0117009801140084011300710101
:1038300010006101100051010E0043010D0036011E
:103840000B002B010B0020010B00150109000C01DE
:10385000090003010800FB000800F3000800EB006A
:103860000700E4000600DE000600D8000600D200D3
:103870000600CC000500C7000500C2000500BD0021
:103880000400B9000400B5000400B1000400AD005C
:103890000400A9000400A5000300A20003009F008B
:1038A00004009B00030098000300950002009300B1
:1038B0000300900003008D0002008B0003008800CD
:1038C00002008600020084000300810002007F00E5
:1038D00002007D0002007B000200790002007700F8
:1038E0000100760002007400020072000100710005
:1038F00002006F0002006D0001006C0002006A000F
:103900000100690002006700010066000100650017
:10391000010064000200620001006100010060001B
:1039200001005F0002005D0001005C0001005B001F
:1039300001005A0001005900010058000100570021
:103940000100560001005500010054000100530021
:10395000000053000100520001005100010050001E
:1039600001004F0001004E0000004E0001004D001C
:1039700001004C0001004B0000004B0001004A0018
:103980000100490001004800000048000100470014
:10399000010046000000460001004500000045000F
:1039A0000100440001004300000043000100420008
:1039B0000000420001004100000041000100400001
:1039C00001003F0000003F0001003E0000003E00FB
:1039D00001003D0000003D0001003C0000003C00F3
:1039E00000003C0001003B0000003B0001003A00E9
:1039F00000003A00010039000000390001003800E1
:103A000000003800000038000100370000003700D7
:103A100001003600000036000000360001003500CD
:103A200000003500000035000100340000003400C3
:103A300000003400010033000000330000003300B8
:103A400001003200000032000000320001003100AD
:103A500000003100000031000100300000003000A3
:103A60000000300001002F0000002F0000002F0098
:103A700000002F0001002E0000002E0000002E008C
:103A800001002D0000002D0000002D0000002D0081
:103A900001002C0000002C0000002C0000002C0075
:103AA00001002B0000002B0000002B0000002B0069
:103AB00001002A0000002A0000002A0000002A005D
:103AC0000100290000002900000029000000290051
:103AD0000000290001002800000028000000280044
:103AE0000000280000002800010027000000270037
:103AF000000027000000270000002700010026002A
:103B0000000026000000260000002600000026001D
:103B10000100250000002500000025000000250010
:103B20000000250000002500010024000000240002
:103B300000002400000024000000240001002300F5
:103B400000002300000023000000230000002300E9
:103B500000002300000023000100220000002200DA
:103B600000002200000022000000220000002200CD
:103B700001002100000021000000210000002100C0
:103B800000002100000021000000210001002000B1
:103B900000002000000020000000200000002000A5
:103BA00000002000000020000000200001001F0095
:103BB00000001F0000001F0000001F0000001F0089
:103BC00000001F0000001F0001001E0000001E007A
:103BD00000001E0000001E0000004D383420582058
:103BE00059205A204500526573656E643A20006F73
:103BF0006B00627573793A20706175736564206635
:103C00006F7220696E7075740A00627573793A205C
:103C100070617573656420666F7220757365720AD2
:103C200000627573793A2070726F63657373696EA1
:103C3000670A004B494C4C45442E20004B494C4CE4
:103C400020636175736564206279204B494C4C2078
:103C5000627574746F6E2F70696E0A004B494C4C1C
:103C600045442E20004B494C4C20636175736564BC
:103C700020627920746F6F206D75636820696E61B2
:103C800063746976652074696D65202D2063757293
:103C900072656E7420636F6D6D616E643A200050C2
:103CA0006C65617365207265736574005052494E8E
:103CB0005445522048414C544544005072696E743A
:103CC00065722068616C7465642E206B696C6C2869
:103CD000292063616C6C6564210A00656E717565ED
:103CE0007565696E6720220000000000000000007A
:103CF000000000005761726E696E673A20486F6D70
:103D0000696E672042756D702044697669736F72C1
:103D1000203C20310A000000A0400000A04000002C
:103D20000040000096430000964300009643FFFFCA
:103D3000FF7C3C3E5E2B3D3F2F5B5D3B2C2A225C93
:103D40000020746F6F206C6F6E67206578747275D9
:103D500073696F6E2070726576656E7465640A00B3
:103D600020636F6C6420657874727573696F6E2060
:103D700070726576656E7465640A0020706F736991
:103D800074696F6E206F7574206F662072616E6744
:103D9000652E0A003F50726F62652000486F6D65A6
:103DA000202573257325732066697273740020665D
:103DB000697273740A005A0059005800486F6D65A3
:103DC00020005374616E6461726420446576696199
:103DD00074696F6E3A20002052616E67653A200068
:103DE000204D61783A2000204D696E3A20004D65E3
:103DF000616E3A200046696E69736865642100202F
:103E000072616E67653A2000206D61783A2000206B
:103E10006D696E3A2000207369676D613A20002059
:103E20006D65616E3A20003A207A3A2000206F6674
:103E30002000205A00205900205800476F696E6703
:103E400020746F3A00436C6F636B776973650A0087
:103E5000436F756E7465722D0020446972656374DA
:103E6000696F6E3A2000202020616E676C653A20F1
:103E7000005374617274696E67207261646975734E
:103E80003A2000506F736974696F6E696E672074B1
:103E900068652070726F62652E2E2E0A003F4E7587
:103EA0006D626572206F66206C65677320696E2095
:103EB0006D6F76656D656E74206E6F7420706C61C9
:103EC000757369626C652028302D3135292E0A0002
:103ED000590058003F53616D706C652073697A65B5
:103EE000206E6F7420706C61757369626C65202838
:103EF000342D3530292E0A004D3438205A2D507279
:103F00006F6265205265706561746162696C697485
:103F10007920546573740A003F566572626F736549
:103F2000204C6576656C206E6F7420706C617573C3
:103F300069626C652028302D34292E0A0020424009
:103F40003A0020403A00202F0020423A00202F0063
:103F500020543A004578747275646572004D6F762E
:103F600065205A004D6F76652059004D6F766520AB
:103F700058005072657061726500526573746F729B
:103F800065206661696C736166650046696C616D88
:103F9000656E74004D6F74696F6E0054656D706569
:103FA000726174757265004D61696E00507265686A
:103FB0006561742041425320636F6E6600507265E4
:103FC0006865617420504C4120636F6E66005049F3
:103FD000442D44005049442D44005049442D49008B
:103FE0005049442D49005049442D50005049442D1A
:103FF0005000200820466163740020082046616359
:1040000074002008204D6178002008204D61780060
:104010002008204D6178002008204D696E0020089E
:10402000204D696E002008204D696E004F666600C5
:104030004F6E20004175746F74656D700046616E3F
:104040002073706565640046616E207370656564F9
:104050000042656400426564004E6F7A7A6C6500C8
:104060004E6F7A7A6C6500436F6E74726F6C0042AB
:10407000656400426564004E6F7A7A6C65004E6F2D
:104080007A7A6C650046616E2073706565640046DF
:10409000616E2073706565640054656D7065726152
:1040A00074757265004573746570732F6D6D00458E
:1040B00073746570732F6D6D005A73746570732F10
:1040C0006D6D005A73746570732F6D6D0059737444
:1040D0006570732F6D6D005973746570732F6D6DFE
:1040E000005873746570732F6D6D0058737465702C
:1040F000732F6D6D00412D74726176656C00412DDA
:1041000074726176656C00412D72657472616374BE
:1041100000412D7265747261637400416D61782095
:104120004500416D6178204500416D6178205A005D
:10413000416D6178205A00416D6178205900416DD0
:104140006178205900416D6178205800416D617897
:104150002058005654726176206D696E0056547274
:104160006176206D696E005654726176206D696EBD
:1041700000566D696E00566D696E00566D696E0071
:10418000566D6178204500566D6178204500566D6A
:104190006178204500566D6178205A00566D61782F
:1041A000205A00566D6178205A00566D617820596A
:1041B00000566D6178205900566D6178205900567F
:1041C0006D6178205800566D6178205800566D61F9
:1041D0007820580056652D6A65726B0056652D6A09
:1041E00065726B0056652D6A65726B00567A2D6A92
:1041F00065726B00567A2D6A65726B0056792D6A6E
:1042000065726B0056792D6A65726B0056792D6A5E
:1042100065726B0056782D6A65726B0056782D6A50
:1042200065726B0056782D6A65726B004163636539
:104230006C00416363656C005A204F666673657459
:10424000005A204F666673657400436F6E74726F18
:104250006C0046696C2E204469612E0046696C2E04
:10426000204469612E004F6666004F6E2000452095
:10427000696E206D6D3300436F6E74726F6C004E0B
:104280006F204C696E65204E756D6265722077698E
:10429000746820636865636B73756D2C204C617363
:1042A00074204C696E653A20004B494C4C45442EB5
:1042B000200053544F505045442E20005072696ED8
:1042C0007465722073746F70706564206475652006
:1042D000746F206572726F72732E20466978207435
:1042E0006865206572726F7220616E6420757365F7
:1042F000204D39393920746F20726573746172747E
:104300002E202854656D7065726174757265206920
:10431000732072657365742E205365742069742050
:1043200061667465722072657374617274696E6718
:10433000290A004E6F20436865636B73756D2077A3
:10434000697468206C696E65206E756D6265722C8B
:10435000204C617374204C696E653A200063686577
:10436000636B73756D206D69736D617463682C2068
:104370004C617374204C696E653A20004C696E651F
:10438000204E756D626572206973206E6F74204CCB
:10439000617374204C696E65204E756D6265722B79
:1043A000312C204C617374204C696E653A20004DAD
:1043B000313130004D3331004D38342058205920F0
:1043C0005A20450053442072656164206572726F03
:1043D000720A00446F6E65207072696E74696E6750
:1043E0002066696C650A0020496E76616C696420FC
:1043F0006578747275646572200000009643000051
:1044000096430000964300000000000000000000FA
:104410000000205A3A200020593A200042656420CA
:10442000583A200043616E6E6F74206F70656E2085
:1044300073756264697220006563686F3A00205A80
:104440003A0020593A0020436F756E7420583A00A4
:1044500020453A00205A3A0020593A00583A0020A4
:10446000643A0020693A0020703A0043290A00614A
:10447000626C656420286D696E2074656D70200023
:10448000436F6C6420657874727564657320617223
:104490006520004B64200023646566696E652020FA
:1044A00044454641554C545F004B692000236465E8
:1044B00066696E65202044454641554C545F004B6B
:1044C00070200023646566696E652020444546417E
:1044D000554C545F00504944204175746F74756E9B
:1044E000652066696E697368656421205075742063
:1044F000746865206C617374204B702C204B6920AC
:10450000616E64204B6420636F6E7374616E7473AC
:104510002066726F6D2062656C6F7720696E746FB4
:1045200020436F6E66696775726174696F6E2E687D
:104530000A00504944204175746F74756E65206699
:1045400061696C6564212074696D656F75740A001A
:10455000504944204175746F74756E6520666169B9
:104560006C6564212054656D706572617475726547
:1045700020746F6F20686967680A00204B643A20D6
:1045800000204B693A2000204B703A20000A20435B
:104590006C617373696320504944200A002054758C
:1045A0003A2000204B753A2000206D61783A2000B7
:1045B000206D696E3A200020643A20002062696113
:1045C000733A20006265640A002C20737973746565
:1045D0006D2073746F707065642120486561746527
:1045E000725F49443A200048656174696E672066CD
:1045F00061696C65640048656174696E6720666115
:10460000696C65640048656174696E6720666169FC
:104610006C65640048656174696E67206661696CE9
:10462000656400544845524D414C2052554E415707
:10463000415900546865726D616C2052756E6177E6
:1046400061790000060900FE070192032120FFFFA7
:1046500008FF07FF00000006000001070706020030
:1046600080808080800080030202060105A0A005F2
:1046700007070600005050F850F85050050707068D
:1046800000002078A07028F020050707060000C071
:10469000C810204098180507070600006090A04049
:1046A000A89068020303060104C0408003070706C0
:1046B0000100204080808040200307070601008021
:1046C00040202020408005050506000120A870A894
:1046D000200505050600012020F82020020303061E
:1046E00002FFC04080050101060003F80202020635
:1046F0000200C0C005050506000108102040800525
:1047000007070600007088888888887003070706F6
:10471000010040C040404040E0050707060000702F
:104720008808708080F8050707060000F810201040
:104730000808F005070706000010305090F8101028
:10474000050707060000F880F008088870050707CD
:10475000060000708080F08888700507070600005A
:10476000F808102020202005070706000070888820
:104770007088887005070706000070888878080828
:1047800070020505060200C0C000C0C00206060691
:1047900002FFC0C000C040800407070600001020D0
:1047A0004080402010050303060002F800F80407CB
:1047B0000706010080402010204080050707060002
:1047C0000070880810200020050707060000708888
:1047D0000868A8A870050707060000708888F88890
:1047E0008888050707060000F08888F08888F005AB
:1047F000070706000070888080808870050707061C
:104800000000F08888888888F0050707060000F80F
:104810008080F08080F8050707060000F88080F0AF
:10482000808080050707060000708880B88888703F
:10483000050707060000888888F888888801070728
:1048400006020080808080808080050707060000C7
:10485000381010101090600507070600008890A01F
:10486000C0A09088050707060000808080808080B7
:10487000F805070706000088D8A8888888880507F3
:10488000070600008888C8A89888880507070600DA
:104890000070888888888870050707060000F088FF
:1048A00088F080808005070706000070888888A847
:1048B0009068050707060000F08888F0A09088053A
:1048C0000707060000788080700808F005070706D3
:1048D0000000F8202020202020050707060000887F
:1048E0008888888888700507070600008888888877
:1048F0008850200507070600008888888888A85007
:10490000050707060000888850205088880507079B
:104910000600008888885020202005070706000030
:10492000F80810204080F8030707060100E08080A7
:10493000808080E005050506000180402010080306
:104940000707060100E02020202020E005030306E1
:104950000004205088050101060000F8020202064A
:104960000205804005050506000070087888780576
:1049700007070600008080B0C88888F00505050696
:10498000000070808088700507070600000808682E
:10499000988888780505050600007088F8807005FD
:1049A00007070600003048E0404040400506060684
:1049B00000FF70888878087005070706000080806F
:1049C000B0C88888880107070602008000808080C0
:1049D00080800308080601FF200020202020A0403E
:1049E000040707060000808090A0C0A0900307077E
:1049F000060100C04040404040E0050505060000BB
:104A0000D0A8A8A8A8050505060000B0C888888811
:104A100005050506000070888888700506060600F2
:104A2000FFF08888F080800506060600FF788888F9
:104A3000780808050505060000B0C88080800505D7
:104A40000506000070807008F004070706000040AB
:104A500040E0404040300505050600008888889801
:104A600068050505060000888888502005050506AC
:104A700000008888A8A85005050506000088502079
:104A800050880506060600FF8888887808700505A6
:104A900005060000F8102040F80307070601002073
:104AA000404080404020010707060200808080804F
:104AB000808080030707060100804040204040803E
:104AC00005020206000268900000000600000000D7
:104AD00000060000000000060000000000060000C4
:104AE00000000006000000000006000000000006B4
:104AF00000000000000600000000000600000000AA
:104B00000006000000000006000000000006000093
:104B10000000000600000000000600000000000683
:104B20000000000000060000000000060000000079
:104B30000006000000000006000000000006000063
:104B40000000000600000000000600000000000653
:104B50000000000000060000000000060000000049
:104B60000006000000000006000000000006000033
:104B70000000000600000000000600000000000623
:104B80000000000000060000000000060000000019
:104B90000006000001070706020080008080808078
:104BA000800507070600002070A8A0A87020050750
:104BB00007060000304040E04050A805050506000B
:104BC000008870507088050707060000885020F89C
:104BD00020F8200107070602008080800080808086
:104BE000050808060000304820505020906003015E
:104BF00001060107A0050707060000F888B8B8B845
:104C000088F8050707060001700878887800F8051D
:104C100005050600012850A05028050303060001E1
:104C2000F80808020202060206408005070706008F
:104C300000F888A88898A8F8050101060006F8047D
:104C4000040406000360909060050707060000203A
:104C500020F8202000F8040505060003609020409D
:104C6000F0030505060003E020E020E00202020652
:104C7000020640800508080600FF8888888898E8B2
:104C800080800507070600007898987818181802A1
:104C90000202060202C0C00202020602FF408003B6
:104CA000050506000340C04040E005070706000177
:104CB000708888887000F8050505060001A0502856
:104CC00050A00507070600008890A858B8080805F6
:104CD00007070600008890B848982038050808069D
:104CE0000000C040C048D838080805070706000083
:104CF0002000204080887005080806000040200041
:104D00007088F88888050808060000102000708860
:104D1000F888880508080600002050007088F88888
:104D2000880508080600006890007088F8888805E3
:104D300008080600005000708888F8888805080870
:104D40000600002050207088F888880507070600B4
:104D5000003860A0B8E0A0B80508080600FF708819
:104D6000808088702060050808060000402000F858
:104D700080F080F8050808060000081000F880F0B0
:104D800080F8050808060000205000F880F080F840
:104D90000507070600005000F880F080F8030808B7
:104DA000060100804000E0404040E00308080601A2
:104DB00000204000E0404040E003080806010040B9
:104DC000A000E0404040E0030707060100A000E02B
:104DD000404040E0050707060000704848E84848A2
:104DE0007005080806000068900088C8A898880523
:104DF0000808060000402070888888887005080828
:104E00000600001020708888888870050808060051
:104E10000020500070888888700508080600006827
:104E2000900070888888700508080600005000709F
:104E300088888888700505050600018850205088FC
:104E40000508080600FF1070A8A8A8A8704005086B
:104E500008060000402088888888887005080806B1
:104E600000001020888888888870050808060000DF
:104E700020500088888888700508080600005000C7
:104E800088888888887005080806000010208850E7
:104E9000202020200509090600FFC0407048487006
:104EA0004040E00408080601FF609090A09090E068
:104EB0008005080806000040200070087888780502
:104EC0000808060000102000700878887805080897
:104ED0000600002050007008788878050808060051
:104EE0000068900070087888780507070600005071
:104EF00000700878887805080806000020502070A7
:104F000008788878050606060000D02878A0A85002
:104F10000506060600FF70808870206005080806F8
:104F200000004020007088F8807005080806000026
:104F30001020007088F880700508080600002050D6
:104F4000007088F880700507070600005000708820
:104F5000F8807003080806010080400040C040400F
:104F6000E003080806010020400040C04040E00384
:104F7000080806010040A00040C04040E0030707C9
:104F8000060100A00040C04040E005070706000001
:104F9000A040A010788870050808060000689000FE
:104FA000B0C888888805080806000040200070887E
:104FB000888870050808060000102000708888881E
:104FC0007005080806000020500070888888700569
:104FD0000808060000689000708888887005070738
:104FE00006000050007088888870050505060001DD
:104FF0002000F800200507070600FF1070A8A8A8E9
:1050000070400508080600004020008888889868DD
:1050100005080806000010200088888898680508A0
:105020000806000020500088888898680507070651
:105030000000500088888898680509090600FF105C
:105040002000888888F808700407070601FFC04020
:1050500060506040E00508080600FF50008888881E
:105060007808700237E2C1E111241FBECFEFD1E210
:10507000DEBFCDBF00E00CBF14E0A0E0B2E0E2EA8A
:10508000FFED01E00BBF02C007900D92A636B107FD
:10509000D9F724E1A6E6B4E001C01D92A339B20716
:1050A000E1F718E2C3E3D8E200E006C02197010966
:1050B000802FFE010E943AEFC233D10780E008073B
:1050C000A9F70E9412DA0C94C0EF0C9400002F9202
:1050D0003F924F925F926F927F928F929F92AF9288
:1050E000BF92CF92DF92EF92FF920F931F93CF93D5
:1050F000DF93CDB7DEB7C657D1090FB6F894DEBF40
:105100000FBECDBF8091AE0620E6829FC001112464
:10511000825D9A4F90932C0D80932B0D8091EE0D14
:1051200080FF1BC0E8E3F4E484918F010F5F1F4F01
:10513000882321F00E941C87F801F6CF00912B0DE7
:1051400010912C0DD8018D918D01882319F00E94AA
:105150001C87F8CF8AE00E941C87E0912B0DF0910C
:105160002C0D8081803231F43196F0932C0DE09338
:105170002B0DF3CF8E3469F010912B0D00912C0D77
:105180006AE270E0812F902F0E9488EF009721F54E
:105190002AC0818190ED980F9A3010F08D3261F71E
:1051A0003296F0932C0DE0932B0DE0912B0DF091A6
:1051B0002C0D808180538A3010F43196F2CFE0912B
:1051C0002B0DF0912C0D80818032B1F63196F09349
:1051D0002C0DE0932B0DF3CFFC01319682918032A0
:1051E00031F08A3221F0A12FB02F9D9102C01082A0
:1051F000F5CFFD01808111968032D9F380538A303A
:1052000020F0E8E3F4E40C947140E12CF12C2AE066
:105210002E9DB0012F9D700D11247B01B0E3EB1A80
:10522000F1088191E80EF11C87FDFA94808180538A
:105230008A3070F38F013196D8018C918032D1F38E
:10524000109371040093700421E030E030932A0D34
:105250002093290D9D3411F40C94FA31943511F4F6
:105260000C940740973411F00C941F40B4E0EB16F7
:10527000F10409F486C640F48091AA02F2E0EF1628
:10528000F10408F020C11FC02AE5E216F10411F470
:105290000C94493160F44CE1E416F10409F4AFC612
:1052A0005EE1E516F10409F42FC70C9468408BE524
:1052B000E816F10409F4F1C79CE5E916F10409F4D4
:1052C000F1C70C946840882311F40C9468400E9444
:1052D000EAAB80913102882321F08DE49DE00E94A9
:1052E0005A880E940D498091EE0D83FD9BC0C090AD
:1052F000590DD0905A0DE0905B0DF0905C0D20910F
:10530000090530910A0540910B0550910C05C70124
:10531000B6010E942CE8882309F484C08091E90D2D
:1053200081113CC0609198047091990480919A0415
:1053300090919B040E9493ED072E000C880B990B13
:105340000E9432E820913F02309140024091410298
:10535000509142020E942CE887FF20C0C0920905AC
:10536000D0920A05E0920B05F0920C05E8E3F4E414
:1053700084918F010F5F1F4F882321F00E941C87AB
:10538000F801F6CFE8EFF1E084918F010F5F1F4F36
:10539000882321F00E941C87F801F6CFC090590D98
:1053A000D0905A0DE0905B0DF0905C0D20910905B6
:1053B00030910A0540910B0550910C05C701B601CB
:1053C0000E944EEC0E9493ED97FF07C09095809548
:1053D000709561957F4F8F4F9F4F693C7105810597
:1053E000910504F1C0920905D0920A05E0920B05DF
:1053F000F0920C05E8E3F4E484918F010F5F1F4FF6
:10540000882321F00E941C87F801F6CFE9EDF1E036
:1054100084918F010F5F1F4F882321F00E941C870A
:10542000F801F6CF20914D0D30914E0D40914F0D6A
:105430005091500D6091FD047091FE048091FF0425
:10544000909100050E942CE881111DC02091510D02
:105450003091520D4091530D5091540D60910105C2
:105460007091020580910305909104050E942CE83B
:10547000811109C0609100027091010280910202C5
:10548000909103021AC06091230270912402072EAA
:10549000000C880B990B0E9432E820910002309199
:1054A000010240910202509103020E9491E82AE019
:1054B00037ED43E25CE30E9491E80E94E6BD0E9462
:1054C000DCBD0C946840882311F40C94684011E012
:1054D000A2E0EA16F10409F010E00E94EAAB82E5CE
:1054E0000E9453BE882309F452C10E9415BF6B016C
:1054F0007C014090FD045090FE046090FF04709089
:10550000000520910105309102054091030550915D
:1055100004052BAF3CAF4DAF5EAF80914D0D909128
:105520004E0DA0914F0DB091500D23968CAF9DAFB5
:10553000AEAFBFAF23972091510D3091520D4091E6
:10554000530D5091540D2B962CAF3DAF4EAF5FAF26
:105550002B9720E030E0A901C701B6010E942CE89A
:10556000882309F4F4C4A301920123966CAD7DADA8
:105570008EAD9FAD23970E942CE881110FC02BADFB
:105580003CAD4DAD5EAD2B966CAD7DAD8EAD9FADA2
:105590002B970E942CE8882309F4D9C420E030E03E
:1055A000A901C701B6010E942CE8881F8827881F1F
:1055B00018130BC080E090E0A0E8BFE367968CAFC3
:1055C0009DAFAEAFBFAF67970AC020E030E040E8C4
:1055D0005FEB67962CAF3DAF4EAF5FAF6797A30110
:1055E000920123966CAD7DAD8EAD9FAD23970E9449
:1055F0004EEC2F966CAF7DAF8EAF9FAF2F972BAD3C
:105600003CAD4DAD5EAD2B966CAD7DAD8EAD9FAD21
:105610002B970E944EEC63966CAF7DAF8EAF9FAF21
:1056200063972F962CAD3DAD4EAD5FAD2F97CA0160
:10563000B9010E9491E84B015C0163962CAD3DAD30
:105640004EAD5FAD6397CA01B9010E9491E89B011D
:10565000AC01C501B4010E944FEC0E94BAEE27963E
:105660006CAF7DAF8EAF9FAF279720E030E040E07A
:105670005FE30E9491E84B015C01A7019601C7011D
:10568000B6010E9491E86B017C01A5019401C5015E
:10569000B4010E9491E89B01AC01C701B6010E94D0
:1056A0004EEC0E94BAEE9B01AC0167966CAD7DADED
:1056B0008EAD9FAD67970E9491E84B015C012396E8
:1056C0002CAD3DAD4EAD5FAD2397C301B2010E943D
:1056D0004FEC20E030E040E05FE30E9491E86B0196
:1056E0007C0163966CAD7DAD8EAD9FAD6397905898
:1056F00027962CAD3DAD4EAD5FAD27970E942BEDAB
:105700009B01AC01C501B4010E9491E89B01AC0171
:10571000C701B6010E944FECA30192010E944EEC1A
:105720006B017C012B962CAD3DAD4EAD5FAD2B9743
:105730006BAD7CAD8DAD9EAD0E944FEC20E030E0B6
:1057400040E05FE30E9491E82B013C0127962CADDD
:105750003DAD4EAD5FAD27972F966CAD7DAD8EAD57
:105760009FAD2F970E942BED9B01AC01C501B401A9
:105770000E9491E89B01AC01C301B2010E944FEC71
:105780002BAD3CAD4DAD5EAD0E944EEC14C089E436
:105790000E9453BE882329F00E9415BF6B017C0133
:1057A00003C0C12CD12C76018AE40E9453BE882309
:1057B000F9F00E9415BF2B966CAF7DAF8EAF9FAFF7
:1057C0002B9720E030E0A901C701B6010E942CE828
:1057D00081111EC020E030E0A9012B966CAD7DAD9B
:1057E0008EAD9FAD2B970E942CE8811111C0AFC3E5
:1057F00020E030E0A901C701B6010E942CE888230F
:1058000009F4A5C32B961CAE1DAE1EAE1FAE2B9782
:10581000D701C601B0588BAF9CAFADAFBEAF2B96D2
:105820002CAD3DAD4EAD5FAD2B97505823962CAFB0
:105830003DAF4EAF5FAF23979C01AD01BC01CD01E1
:105840000E9491E84B015C0123962CAD3DAD4EAD1D
:105850005FAD2397CA01B9010E9491E89B01AC0199
:10586000C501B4010E944FEC0E94BAEEA7966CAF3E
:105870007DAF8EAF9FAFA7978091FD049091FE04FE
:10588000A091FF04B091000527968CAF9DAFAEAFFD
:10589000BFAF2797A7019601BC01CD010E944FEC35
:1058A00067966CAF7DAF8EAF9FAF67972091010574
:1058B0003091020540910305509104052F962CAFBD
:1058C0003DAF4EAF5FAF2F972B962CAD3DAD4EAD9C
:1058D0005FAD2B972F966CAD7DAD8EAD9FAD2F97A5
:1058E0000E944FEC6B966CAF7DAF8EAF9FAF6B9706
:1058F00080914D0D90914E0DA0914F0DB091500D96
:105900006F968CAF9DAFAEAFBFAF6F9767962CAD64
:105910003DAD4EAD5FAD6797BC01CD010E944EEC31
:105920006B017C012091510D3091520D4091530D2E
:105930005091540DA3962CAF3DAF4EAF5FAFA397E0
:105940006B962CAD3DAD4EAD5FAD6B97A3966CAD38
:105950007DAD8EAD9FADA3970E944EEC4B015C01D7
:105960008091050590910605A0910705B091080565
:10597000AF968CAF9DAFAEAFBFAFAF979C01AD01FF
:105980006091550D7091560D8091570D9091580D65
:105990000E944EEC63966CAF7DAF8EAF9FAF639766
:1059A0002091590D30915A0D40915B0D50915C0D35
:1059B000AB962CAF3DAF4EAF5FAFAB978091090573
:1059C00090910A05A0910B05B0910C05E3968CAF60
:1059D0009DAFAEAFBFAFE397A70196016BAD7CADB6
:1059E0008DAD9EAD0E9491E82B013C01A501940173
:1059F00023966CAD7DAD8EAD9FAD23970E9491E84F
:105A00009B01AC01C301B2010E944FEC2B013C0190
:105A1000A50194016BAD7CAD8DAD9EAD0E9491E86A
:105A20004B015C01A701960123966CAD7DAD8EAD57
:105A30009FAD23970E9491E89B01AC01C501B40181
:105A40000E944EECA30192010E94C2EC6B017C010A
:105A500020E030E0A9010E942CE887FF0AC02BED6E
:105A60003FE049EC50E4C701B6010E944FEC6B01E6
:105A70007C01112351F02BED3FE049EC50E4C701CC
:105A8000B6010E944EEC6B017C0120E030E0A901E0
:105A9000C701B6010E942CE881112AC06F962CAD77
:105AA0003DAD4EAD5FAD6F9727966CAD7DAD8EADC4
:105AB0009FAD27970E942CE881111AC0A3962CADA8
:105AC0003DAD4EAD5FADA3972F966CAD7DAD8EAD68
:105AD0009FAD2F970E942CE881110AC02BED3FE06B
:105AE00049EC50E4C701B6010E944FEC6B017C0108
:105AF000A7962CAD3DAD4EAD5FADA797C701B601E2
:105B00000E9491E89B01AC010E9491E84B015C016D
:105B100063962CAD3DAD4EAD5FAD6397CA01B90143
:105B20000E9491E89B01AC01C501B4010E944FECB9
:105B30000E94BAEE4B015C012FE632E143E85AE3E2
:105B40000E942CE887FDFFC1C501B4010E94C4ED8D
:105B50000E9498ED2D967FAF6EAF2D97DB01AB2B9A
:105B600031F4E1E0F0E02D96FFAFEEAF2D972D96EA
:105B70002EAD3FAD2D97B90180E090E00E9430E856
:105B80004B015C019B01AC01C701B6010E942BEDEA
:105B900027966CAF7DAF8EAF9FAF2797A50194017D
:105BA00063966CAD7DAD8EAD9FAD63970E942BED7E
:105BB000A7966CAF7DAF8EAF9FAFA797E3962CAD46
:105BC0003DAD4EAD5FADE397AB966CAD7DAD8EADAB
:105BD0009FADAB970E944EECA50194010E942BED66
:105BE000AB966CAF7DAF8EAF9FAFAB9727962CADCA
:105BF0003DAD4EAD5FAD2797CA01B9010E9491E856
:105C000020E030E040E05FE30E9491E89B01AC01BE
:105C100060E070E080E89FE30E944EEC63966CAF1A
:105C20007DAF8EAF9FAF6397AF968CAD9DADAEADA0
:105C3000BFADAF9789879A87AB87BC87E3962CADBA
:105C40003DAD4EAD5FADE3972D873E874F87588BB7
:105C50006091230270912402072E000C880B990B8F
:105C60000E9432E82091000230910102409102022C
:105C7000509103020E9491E82AE037ED43E25CE391
:105C80000E9491E86F966CAF7DAF8EAF9FAF6F971C
:105C90000E94975B9B01AC0128533F4F4F4F5F4FD2
:105CA000A3962CAF3DAF4EAF5FAFA3974BAC5CACB0
:105CB0006DAC7EAC22242394312CD12C2D968EAD4C
:105CC0009FAD2D972816390609F429C10E9448D3A3
:105CD0000E94975BDC01CB01A3962CAD3DAD4EAD90
:105CE0005FADA397821B930BA40BB50BB7FD10C040
:105CF0000E94975B9B01AC0128533F4F4F4F5F4F72
:105D0000A3962CAF3DAF4EAF5FAFA3970E94DF8A43
:105D1000D39438E13D150CF44BC063962CAD3DADEA
:105D20004EAD5FAD639723966CAD7DAD8EAD9FADEF
:105D300023970E9491E84B015C0127962CAD3DAD65
:105D40004EAD5FAD2797B201C3010E9491E8A50156
:105D500094010E944FEC7B018C0163962CAD3DAD0C
:105D60004EAD5FAD6397B201C3010E9491E84B0154
:105D70005C0127962CAD3DAD4EAD5FAD27972396C8
:105D80006CAD7DAD8EAD9FAD23970E9491E89B01D8
:105D9000AC01C501B4010E944EEC2B013C01C701CE
:105DA000D80123968CAF9DAFAEAFBFAF239756C03F
:105DB000B10180E090E00E9430E827962CAD3DAD27
:105DC0004EAD5FAD27970E9491E84B015C010E94A8
:105DD00028ED6B017C01C501B4010E94B0EE4B01BE
:105DE0005C01A70196016BAD7CAD8DAD9EAD0E94AF
:105DF00091E82B013C01A50194012B966CAD7DAD82
:105E00008EAD9FAD2B970E9491E89B01AC01C30121
:105E1000B2010E944FEC2B013C01A50194016BAD36
:105E20007CAD8DAD9EAD0E9491E84B015C01A70158
:105E300096012B966CAD7DAD8EAD9FAD2B970E94DC
:105E400091E89B01AC01C501B4010E944EEC239680
:105E50006CAF7DAF8EAF9FAF2397D12C9201A30182
:105E600067966CAD7DAD8EAD9FAD67970E944FEC90
:105E700069837A838B839C8323962CAD3DAD4EAD95
:105E80005FAD23976B966CAD7DAD8EAD9FAD6B977F
:105E90000E944FEC6D837E838F839887A7962CADED
:105EA0003DAD4EAD5FADA79769857A858B859C85A5
:105EB0000E944FEC69877A878B879C87AB962CADC5
:105EC0003DAD4EAD5FADAB976D857E858F85988975
:105ED0000E944FEC6D877E878F87988B809131026F
:105EE000882321F0CE0101960E945A88C0906A044E
:105EF0006F96ECACFDAC0EAD1FAD6F979E01235FAE
:105F00003F4FAE01475F5F4FBE016B5F7F4FCE01DA
:105F100001960E9477984FEF241A340ACFCEC09092
:105F20006A046F96ECACFDAC0EAD1FAD6F9729E522
:105F30003DE045E55DE061E57DE08DE49DE00E94AA
:105F400077980E94DCBD0E940D490C946840E3EDF7
:105F5000F3E384918F010F5F1F4F882321F00E948C
:105F60001C87F801F6CFE3E1F2E084918F010F5F27
:105F70001F4F882311F40C9468400E941C87F8017D
:105F8000F4CF80E50E9453BE882329F00E940ABF07
:105F90006B017C0103C0C12CD12C760183E50E94EA
:105FA00053BE882321F00E943EBF6B017C010E94FA
:105FB000A3D40E940D4980912D0D90912E0DA0919A
:105FC0002F0DB091300DC80ED91EEA1EFB1E809118
:105FD0006702811105C060E089E292E00E94F7D873
:105FE0000E94975BDC01CB018C199D09AE09BF09AA
:105FF000B7FD02C00C9468400E94DF8AF1CF0E9476
:10600000A3D40E949FBA81E080930B0288E50E948E
:1060100053BEE82E89E50E9453BE082F8AE50E94F0
:1060200053BEF82EE11005C0011105C011E018277C
:1060300005C0011102C010E001C0182F80E1EDEF92
:10604000F4E0ADE4BDE001900D928A95E1F7111105
:1060500005C0E11003C0002309F444C020E030E093
:1060600040EA50E460913D0D70913E0D80913F0DEE
:106070009091400D0E944FEC6093550D7093560D1A
:106080008093570D9093580D20910505309106058A
:1060900040910705509108050E9475EE18167CF492
:1060A00019821A821B821C829E012F5F3F4F45E599
:1060B0005DE061E075E08DEF94E00E94BFBA1111E0
:1060C00005C0E11003C0011107C00CC080E090E0E2
:1060D0000E94EC881123B9F381E090E00E94EC88E3
:1060E000111102C0FF2021F082E090E00E94EC88B4
:1060F0000E94FD488091680480930B020E9485BA3B
:106100000E9442CD0C94684088E50E9453BE8823CB
:1061100019F00E9415BF0EC020E030E040E251E4CB
:106120006091FD047091FE048091FF049091000540
:106130000E944FEC4B015C0189E50E9453BE88230D
:1061400019F00E9415BF0EC020E030E040E251E49B
:1061500060910105709102058091030590910405FD
:106160000E944FEC2B013C0120913D0D30913E0DE2
:1061700040913F0D5091400D2BAF3CAF4DAF5EAF06
:106180002091350D3091360D4091370D5091380DDD
:10619000C501B4010E944EEC2091390D30913A0DA9
:1061A00040913B0D50913C0D23962CAF3DAF4EAF2F
:1061B0005FAF239720E030E040E251E40E944EECD4
:1061C0006B017C0127E137EB41ED58EB0E9475EE46
:1061D00087FF02C00C94684023E030E046E953E4B6
:1061E000C701B6010E942CE8181614F40C946840FC
:1061F00023962CAD3DAD4EAD5FAD2397C301B201EB
:106200000E944EEC20E030E040E251E40E944EEC6F
:106210006B017C0127E137EB41ED58EB0E9475EEF5
:1062200087FF02C00C94684023E030E046E953E465
:10623000C701B6010E942CE8181614F40C946840AB
:1062400020E030E0A9016BAD7CAD8DAD9EAD0E942C
:106250004FEC2BAD3CAD4DAD5EAD0E944EEC6B01F5
:106260007C0127E137EB41ED58EB0E9475EE87FF8B
:1062700002C00C94684023E030E046E953E4C701D3
:10628000B6010E942CE8181614F40C9468400C9483
:10629000214010926F040C94684081E080936F0459
:1062A0000C94694085E40E9453BEB82E811102C04F
:1062B0000E94A3D4BCEB8B2EB2E09B2E1DEFC12E0F
:1062C00014E0D12E01E4E02E0DE0F02E00E010E00D
:1062D000A12CD4018D914D010E9453BE8823F1F170
:1062E000F6012081318142815381E4962FAFE497FA
:1062F000E5963FAFE597E6964FAFE697E7965FAF37
:10630000E7970E9415BFD6016D937D938D939C9363
:106310001397E4962FADE497E5963FADE597E696A3
:106320004FADE697E7965FADE79703301105B1F003
:106330000E944EEC9B01AC01F7016081718182816A
:1063400093810E944FECD7016D937D938D939C9325
:106350001397C8010E94FFBDAA24A3940F5F1F4F8B
:10636000B4E0CB0ED11CE4E0EE0EF11C04301105BC
:1063700009F0AFCFAA2019F00E94FD4837C0BB201A
:10638000A9F1C0900905D0900A05E0900B05F090A6
:106390000C0520912D0E30912E0E40912F0E509114
:1063A000300EC701B6010E9491E80E9480EE609312
:1063B0005611709357118093581190935911C7013A
:1063C000B6010E9493ED2FB7F89460932714709351
:1063D00028148093291490932A142FBF10924611E9
:1063E0001092471110924811109249110E9442CD0B
:1063F0000C946840F1E7EF16F10409F493C608F035
:10640000E6C030E3E316F10409F47CC508F077C078
:1064100058E1E516F10409F4C3C208F044C092E162
:10642000E916F10409F45AC7E8F4B2E0EB16F104F6
:1064300008F4EFC1E1E1EE16F10411F00C946840AC
:1064400060E08AE792E00E94F7D85F988A989FB749
:10645000F894809108018E7F809308019FBF129865
:106460000C946840F5E1EF16F10409F48FC248F48A
:1064700034E1E316F10411F00C946840E2E9F2E033
:1064800042C246E1E416F10409F484C257E1E5167C
:10649000F10411F00C94684040E061E0C8010E94F2
:1064A00070740C9468408CE1E816F10409F4CDC2D4
:1064B00068F4AAE1EA16F10409F47DC208F089C281
:1064C00010928A110E947B790C946840EFE1EE16DD
:1064D000F10409F429C438F42EE1E216F10409F4B8
:1064E000BBC20C94684030E2E316F10409F4CCC35B
:1064F0004AE2E416F10409F4BDC40C9468405CE57A
:10650000E516F10409F428C768F591E5E916F104E8
:1065100009F4C7C6A0F4BCE4EB16F10409F4F6C410
:10652000EDE4EE16F10409F4F5C4FBE4EF16F10412
:1065300011F00C9468400E943B790C94684023E56C
:10654000E216F10409F4C6C608F4C1C644E5E4162F
:10655000F10409F4C3C655E5E516F10409F4EBC6E8
:106560000C9468408CE6E816F10409F4D8C5C8F428
:10657000A9E6EA16F10409F412C638F4E8E6EE16C4
:10658000F10409F4CBC40C946840FAE6EF16F10468
:1065900009F453C62BE6E216F10409F472C60C9412
:1065A00068403EE6E316F10409F409C508F414C690
:1065B0005FE6E516F10409F415C580E7E816F10475
:1065C00011F00C94684088E893E00E94778A92EE7C
:1065D000E916F10411F40C947F3D08F080C0BEEB85
:1065E000EB16F10409F410C660F5F7E7EF16F104B5
:1065F00009F44CC798F433E7E316F10409F439C7FA
:1066000008F432C755E7E516F10411F00C94684020
:1066100060E0C8010E940CD90C94684089E7E81634
:10662000F10409F49FC708F497C7ACE8EA16F1042F
:1066300009F4A1C5B1E9EB16F10409F498C70C946B
:106640006840EDECEE16F10411F40C941D3CE0F4FE
:1066500029ECE216F10411F40C94733B38F448EC85
:10666000E416F10409F4F7C70C9468405BECE516F6
:10667000F10411F40C94953B8CECE816F10411F440
:106680000C94B33B0C94684093EDE916F10411F4BB
:106690000C94C13CB0F4BEECEB16F10411F00C9478
:1066A00068403CEBA32E32E0B32E4DEFC42E44E005
:1066B000D42E51EFE52E54E0F52E00E010E00C94BE
:1066C000883CECEDEE16F10411F40C94593DFDED0F
:1066D000EF16F10411F40C94663D0C94684022E925
:1066E000E21621E0F20611F40C94783E08F041C065
:1066F0004FE2E41641E0F40611F40C94723E98F473
:106700008DE2E81681E0F80611F40C94D03D10F00B
:106710000C946F3EACE2EA16A1E0FA0611F40C9478
:10672000AA3D0C946840B3E6EB16B1E0FB0611F409
:106730000C94DE3F58F4F0E3EF16F1E0FF0611F0A1
:106740000C9468400E94C3CC0C94684020E9E21687
:1067500021E0F20611F40C94753E31E9E31631E0C4
:10676000F30611F00C94684081E00E940DBC0C947B
:10677000684046EFE41641E0F40611F40C949C3FA7
:1067800040F58CEAE81681E0F80611F40C947C3EA2
:1067900058F4AAE9EA16A1E0FA0611F00C94684050
:1067A0000E94FBC70C946840B4EFEB16B1E0FB0607
:1067B00011F40C94833FE5EFEE16E1E0FE0611F0D4
:1067C0000C9468400E94B44D80E00E94C7490C942C
:1067D0006840F3E5EF16F3E0FF0611F40C94AB3FCD
:1067E00048F437EFE31631E0F30611F40C949F3FC1
:1067F0000C94684040EAE41643E0F40609F48AC2C7
:1068000057EEE51653E0F50611F40C94F73F0C949F
:10681000684080E50E9453BE882361F00E940ABF51
:106820006B017C01BB24B394672B682B692B31F47B
:10683000B12C04C0B12CC12CD12C760183E50E946F
:1068400053BE882399F00E943EBF6B017C01B110BA
:106850000FC0672B682B692B59F4D8018C918823C2
:1068600039F061E0C8010E940CD907C0BB20A9F330
:1068700060E087E692E00E94F7D883E090E0909392
:106880002A0D8093290D81E08093DA070E94A3D41A
:106890000E940D49C114D104E104F104E9F0809192
:1068A0002D0D90912E0DA0912F0DB091300DC80E91
:1068B000D91EEA1EFB1E0E94975BDC01CB018C19DE
:1068C0009D09AE09BF09B7FF1AC08091DA07882376
:1068D000B1F00E94DF8AEFCF8091DA07882319F0A8
:1068E0000E94DF8AF9CF80918A1160E0882319F035
:1068F00088E592E002C084E492E00E94F7D810920A
:10690000DA070C94684084918F010F5F1F4F882332
:1069100021F00E941C87F801F6CF109210141092FB
:106920000F1440E050E0BA018BEB91E10E94F08E31
:106930008BE1EBEBF1E1DE01159601900D928A956A
:10694000E1F78091B9119091BA119C838B8380E813
:1069500093E09A83898340E050E0BE016F5F7F4FF0
:106960008AE094E00E9410C6CE0101960E946F4F0B
:10697000E3E8F2E084918F010F5F1F4F882311F449
:106980000C9468400E941C87F801F4CF0E94A27703
:106990000C94684010928A1110928B110C946840EC
:1069A00080918B11882319F081E080938A110E94D5
:1069B0003B790C94684080918B11882311F40C94DE
:1069C000684083E50E9453BE81110C948E400C9464
:1069D000684080918B11882351F1E3EAF2E08491C1
:1069E0008F010F5F1F4F882321F00E941C87F80141
:1069F000F6CF60910614709107148091081490915D
:106A000009144AE00E9423878FE20E941C8760914C
:106A100002147091031480910414909105144AE0BB
:106A20000E9423878AE00E941C870C946840E5EB53
:106A3000F2E084918F010F5F1F4F882311F40C94B3
:106A400068400E941C87F801F4CF40E060E0C80174
:106A50000E9470740C94684080918B11882311F40B
:106A60000C94684085E593E10E94AD8E85E593E145
:106A70000E944C911092891110928811E09070043C
:106A8000F090710480918B11882311F40C9468406C
:106A90000E9425741D8218861C821B8280E893E068
:106AA0009A83898387EB91E19093D7118093D611D4
:106AB000F70180818F3209F068C06FE270E0C70192
:106AC0000E9488EF8C010F5F1F4F9E012F5F3F4F89
:106AD00049010115110509F45EC06FE270E0C801BB
:106AE0000E9488EF6C01009709F456C00817190737
:106AF00008F052C05C01A01AB10AA501B801CE018C
:106B000080960E94B1EFE0E2F0E0EC0FFD1FEA0D8D
:106B1000FB1D10828E01005E1F4FD8018D918D01EB
:106B2000882319F00E941C87F8CF8AE00E941C87F6
:106B30006091D6117091D7116115710511F06C5FDC
:106B40007F4F21E0AE01405E5F4FCE0105960E946F
:106B5000D293811112C0BE01605E7F4F8CEE92E035
:106B60000E9415828EE20E941C878AE00E941C8788
:106B7000C4010E946F4F0C9468409092D71180928C
:106B8000D61186010F5F1F4FA4CF88ED91E190933E
:106B9000D7118093D61187016091D6117091D711CA
:106BA0006115710511F06C5F7F4F18A21BA222E0E6
:106BB000A801CE0180960E94D293811102C0F12CCF
:106BC0001EC0CE0180960E947EC58823C1F36CA5AD
:106BD0007DA58EA59FA541E00E947B82882379F345
:106BE000E8A9B0E2EB9FF0011124E551F14F309795
:106BF00031F385EE80831BA20E943B82F82ECE01EA
:106C000080960E94694FFF2009F1E6ECF2E0849142
:106C10007F012FEFE21AF20A882321F00E941C87DD
:106C2000F701F5CFD8018D918D01882319F00E94CD
:106C30001C87F8CF8AE00E941C87109206141092DD
:106C40000714109208141092091418C0E4EDF2E031
:106C500084917F01BFEFEB1AFB0A882321F00E9489
:106C60001C87F701F5CFF80181918F01882319F076
:106C70000E941C87F8CF8EE20E941C87CE010196ED
:106C80000E946F4F0C94684080918A1181110E947C
:106C9000A3D4009170041091710461E270E0C80106
:106CA0000E9488EF009719F08C010F5F1F4F80E55D
:106CB0000E9453BE882349F0FF24F3948091660418
:106CC000909167048017910708F0F12C80918B1147
:106CD000882311F40C9468404F2D61E0C8010E9494
:106CE000707483E50E9453BE882349F08091660446
:106CF000909167048017910710F40C949F40809145
:106D00008B11882319F081E080938A11F1100C9483
:106D100068404DCE81E08093891140E060E0C80179
:106D20000E9470740C9468400E9429C5ACE3CA2E7E
:106D3000D12CE12CF12CA70196010E94F1EB762ECB
:106D4000672ECA01B901A70196010E94F1EB6B0100
:106D50007C01CA01B90128E130E040E050E00E9426
:106D6000F1EB4B015C01C9016DE671E00E9413EF8C
:106D70008E010F5F1F4F6115710599F06F927F9221
:106D8000DF92CF929F928F929F938F937F936F9377
:106D900088E293E09F938F931F930F930E94C5E720
:106DA00012C00097B1F06F927F92DF92CF929F92C4
:106DB0008F929F938F9388E193E09F938F931F937C
:106DC0000F930E94C5E70FB6F894DEBF0FBECDBF8C
:106DD00036C081149104A104B10479F06F927F92BE
:106DE000DF92CF929F928F928CE093E09F938F934C
:106DF0001F930F930E94C5E7E6CFC114D104E104AD
:106E0000F10469F06F927F92DF92CF9284E093E079
:106E10009F938F931F930F930E94C5E7D4CF6F92D8
:106E20007F9280E093E09F938F931F930F930E9434
:106E3000C5E70F900F900F900F900F900F9060E0AC
:106E4000C8010E940CD9E8E3F4E484917F01BFEF0C
:106E5000EB1AFB0A882321F00E941C87F701F5CF6B
:106E6000B8018CE393E00E9415828AE00E941C879F
:106E70000C94684083E50E9453BE882311F40C945F
:106E800068400E94FDBE7C018F3F910519F010F013
:106E90000C94684080E50E9453BE882339F00E941C
:106EA000FDBE8C0197FF04C00C9468400DE010E01B
:106EB000D02EE0ECF2E0C8019927219131912817FA
:106EC000390731F023E0E031F207B9F70C94B14013
:106ED000E3EDF3E384918F010F5F1F4F882321F0CF
:106EE0000E941C87F801F6CFE9E4F3E084918F015A
:106EF0000F5F1F4F882311F40C9468400E941C8779
:106F0000F801F4CF0E94F7A50C9468400E947B79A9
:106F10000C9468400E9410C50C94684088E690E08C
:106F20000E9495BE81110C9468408091EE0D83FF04
:106F300002C00C94684083E50E9453BE8823D9F1B7
:106F40000E94FDBE909312088093110880E00E9479
:106F5000D3D00E94FDBE863591053CF40E9410C539
:106F600060E08FE593E00E94F7D80E94FDBE8C019F
:106F7000609198047091990480919A0490919B0477
:106F80000E9493ED60177107B4F48BE993E09F932F
:106F90008F938091690490E001969F938F9388E589
:106FA00093E09F938F931F920E9420790FB6F894DD
:106FB000DEBF0FBECDBF0E94E2E10C9468408EE4BC
:106FC0000E9453BE882311F40C9468400E942DE265
:106FD0006093190D70931A0D80931B0D90931C0DE7
:106FE0000C94684083E50E9453BE882319F00E94E8
:106FF00066BE01C080E08093EE0DE8E3F4E4849186
:107000008F010F5F1F4F882321F00E941C87F8011A
:10701000F6CFE1E8F3E084918F010F5F1F4F8823E3
:1070200021F00E941C87F801F6CF8091EE0D882395
:10703000A1F1F3E7CF2EF3E0DF2EE12CF12C20E0DD
:107040008091EE0D90E00E2C02C0959587950A94E4
:10705000E2F780FF17C0BB24B394B20E222319F0CD
:107060008CE20E941C87F60125913491F9018491EC
:1070700089010F5F1F4F882321F00E941C87980110
:10708000F5CF2B2DFFEFEF1AFF0A32E0C30ED11C14
:1070900045E0E416F104A1F63EC0EDE7F3E084918B
:1070A0008F010F5F1F4F8823B1F10E941C87F801E9
:1070B000F6CF8AE50E9453BE882309F472C70E9466
:1070C00015BF6B017C0120E030E040EA51EC0E94EA
:1070D00075EE87FD59C720E030E040EA51E4C70172
:1070E000B6010E942CE818160CF44EC7C092750E1B
:1070F000D092760EE092770EF092780EC0925F02F8
:10710000D0926002E0926102F092620242E0C70116
:10711000B6010E94A3878AE00E941C87D9C71092FB
:107120000402D6C783E50E9453BE882359F00E940B
:1071300066BE80933A028D3308F4CAC78CE380930D
:107140003A02C6C7E8E3F4E484918F010F5F1F4F52
:10715000882321F00E941C87F801F6CF40913A0263
:1071600050E060E070E081E993E00E94AD818AE048
:107170000E941C87ADC78091EE0D83FF01C0A8C798
:1071800083E50E9453BE882309F4A2C70E94FDBE76
:1071900090931608809315080E94A0D099C789E69D
:1071A00090E00E9495BE811111C0E8E9F3E084915E
:1071B0008F010F5F1F4F882321F00E941C87F80169
:1071C000F6CF0E946BA58AE00E941C8710922A0DC0
:1071D0001092290D0C942C448DE690E00E9495BEEF
:1071E000811176C78091EE0D83FD72C783E50E9401
:1071F00053BE28968FAF28978111C8C782E50E9499
:1072000053BE8111C3C764C78091EE0D83FD60C773
:1072100060E08CED93E00E94F7D883E50E9453BEB6
:1072200028968FAF289781110C94684282E50E94BE
:1072300053BE81110C9468424BC783E50E9453BE34
:10724000882321F00E9421E28C0102C00FEF10E0A0
:1072500080E50E9453BE882319F00E9421E202C0FB
:1072600080E090E098010F3F110519F010F02FEF2A
:1072700030E0892B09F02CC73093140820931308B1
:1072800027C780E50E9453BE811105C010921408E3
:10729000109213081DC70E9421E2892B09F018C71C
:1072A000F5CF0E9406D10E94A3D40E94668A109254
:1072B00014081092130868EE73E080E090E00E94DA
:1072C0003AD860E089EE93E00E94F7D801C71092A7
:1072D0006E04FEC681E080936E04FBC683E50E94C7
:1072E00053BE882359F00E943EBF60933B027093C7
:1072F0003C0280933D0290933E02EAC688E50E94DC
:1073000053BE81110C94D84389E50E9453BE81116C
:107310000C94D8438AE50E9453BE81110C94D84343
:1073200085E40E9453BE81110C94D8430E94A3D4DB
:107330000E94668ACDC683E50E9453BE882309F465
:10734000C7C60E943EBF6093310D7093320D80938B
:10735000330D9093340DBCC63CEBC32E32E0D32EDC
:1073600041E2E42E4EE0F42E10E0D6018D916D0145
:107370000E9453BE882309F46DC0133009F063C026
:107380000E9415BF4B015C0120E030E040EA51E46F
:107390000E942CE887FF4EC0A501940160912D0E3C
:1073A00070912E0E80912F0E9091300E0E942BED39
:1073B0002B013C019B01AC0160916D0E70916E0E32
:1073C00080916F0E9091700E0E9491E860936D0E07
:1073D00070936E0E80936F0E9093700EA3019201C6
:1073E00060915D0E70915E0E80915F0E9091600EC7
:1073F0000E9491E860935D0E70935E0E80935F0E25
:107400009093600E6091FB0D7091FC0D8091FD0DCD
:107410009091FE0D0E9430E8A30192010E9491E834
:107420000E9498ED6093FB0D7093FC0D8093FD0D11
:107430009093FE0D80922D0E90922E0EA0922F0E04
:10744000B092300E07C00E9415BFF70160837183B0
:10745000828393831F5FF4E0EF0EF11C143009F078
:1074600084CF0E944D9834C60E94A3D40E9442CD7E
:107470002FC6EBEFF3E084918F010F5F1F4F88233E
:1074800009F426C60E941C87F801F5CFE5EFF4E069
:1074900084918F010F5F1F4F882321F00E941C876A
:1074A000F801F6CFEDEEF4E084918F010F5F1F4FEE
:1074B000882321F00E941C87F801F6CF659B03C04A
:1074C0000CE813E002C001E913E0D8018D918D01B1
:1074D000882319F00E941C87F8CF8AE00E941C873D
:1074E000E5EEF4E084918F010F5F1F4F882321F0B8
:1074F0000E941C87F801F6CF8091030181FF03C031
:107500000CE813E002C001E913E0F80181918F015A
:10751000882319F00E941C87F8CF8AE00E941C87FC
:10752000EDEDF4E084918F010F5F1F4F882321F070
:107530000E941C87F801F6CF4B9B03C00CE813E0B8
:1075400002C001E913E0D8018D918D01882309F46F
:10755000E2CD0E941C87F7CF81E080930B028093DD
:107560006804B7C510920B0210926804B1C583E598
:107570000E9453BE8823F1F00E94FDBE182F823076
:10758000D0F0E3EDF3E384918F010F5F1F4F882369
:1075900021F00E941C87F801F6CFEFE0F5E084911E
:1075A0008F010F5F1F4F882309F492C50E941C872B
:1075B000F801F5CF10E088E40E9453BE8823B1F0B3
:1075C0000E94FDBEE12FF0E08A3A91053CF0853043
:1075D000B1E09B072CF084E091E002C08AEA90E0E1
:1075E000EE0FFF1FE35FF14F9183808386E40E94DB
:1075F00053BE8823A1F00E94FDBEE12FF0E0EE0F04
:10760000FF1FEF5EF14F8F3F910519F014F08FEFE0
:1076100090E097FF02C080E090E09183808382E455
:107620000E9453BE882309F453C50E94FDBEE12F7A
:10763000F0E08530910534F0883891052CF087E82A
:1076400090E002C085E090E0EE0FFF1FE75FF14F92
:10765000918380833DC588EC90E00E9495BE8111A6
:1076600037C584E40E9453BE8823D1F10E9415BF20
:1076700011E020E030E0A9010E942CE8811101C056
:1076800010E01093790E112359F10091690410E074
:107690000E9415BF000F111F000F111FF801ED59B7
:1076A000FD4F608371838283938320E030E0A901E2
:1076B000609163027091640280916502909166020C
:1076C0000E942CE881110CC080E090E0A0E4B0E4BE
:1076D0008093630290936402A0936502B093660264
:1076E0000E948D84F5C4E9E3EE2EEEE0FE2E0CEB55
:1076F00012E0F4E0DF2ED00EF80181918F010E949C
:1077000053BE882351F00E9415BF0E9498EDD70107
:107710006D937D938D939C931397B4E0EB0EF11CC6
:10772000D012EACF0E942097D3C461E5E62E6EE026
:10773000F62E0CEB12E074E0D72ED00EF8018191FA
:107740008F010E9453BE882341F00E9415BFD701CC
:107750006D937D938D939C931397B4E0EB0EF11C86
:10776000D012ECCFB5C483E50E9453BE8823D9F074
:107770000E9415BFAB01BC014093710E5093720E75
:107780006093730E7093740E4093310E5093320ECB
:107790006093330E7093340E8BE895E00E94E38182
:1077A0008AE00E941C8780E50E9453BE882399F0DE
:1077B0000E9415BFAB01BC014093710E5093720E35
:1077C0006093730E7093740E8EE695E00E94E381D1
:1077D0008AE00E941C8782E50E9453BE882399F0AC
:1077E0000E9415BFAB01BC014093350E5093360E7D
:1077F0006093370E7093380E8FE495E00E94E3811A
:107800008AE00E941C8784E50E9453BE882309F405
:107810005FC40E9415BFAB01BC014093310E509371
:10782000320E6093330E7093340E81E395E00E9424
:10783000E3818AE00E941C874BC483E50E9453BE0B
:10784000882351F00E9415BF60934D0E70934E0E29
:1078500080934F0E9093500E84E50E9453BE882370
:1078600051F00E9415BF6093490E70934A0E8093A9
:107870004B0E90934C0E82E40E9453BE882351F02D
:107880000E940ABF6093EA0D7093EB0D8093EC0D9C
:107890009093ED0D88E50E9453BE882351F00E941D
:1078A00015BF6093610E7093620E8093630E909388
:1078B000640E89E50E9453BE882351F00E9415BFD3
:1078C0006093650E7093660E8093670E9093680EBA
:1078D0008AE50E9453BE882351F00E9415BF609331
:1078E000690E70936A0E80936B0E90936C0E85E414
:1078F0000E9453BE882309F4EBC30E9415BF609316
:107900006D0E70936E0E80936F0E9093700EE0C3A9
:10791000F50181915F010E9453BE882311F10E94FD
:1079200015BF2B013C01D7012D913D914D915C91EB
:107930000E944EEC9B01AC01F60160817181828155
:1079400093810E944FECD6016D937D938D939C9310
:107950001397F7014082518262827382C8010E94AC
:10796000FFBD0F5F1F4FF4E0CF0ED11C24E0E20EED
:10797000F11C0330110561F60E94FD480E9442CDC2
:10798000A7C3E8E3F4E484918F010F5F1F4F8823BE
:1079900021F00E941C87F801F6CF83E50E9453BEB8
:1079A000882321F00E94D2BE80933102EBEDF5E0F6
:1079B00084918F010F5F1F4F882321F00E941C8745
:1079C000F801F6CF80913102811103C0E7EDF5E0B7
:1079D00002C0E3EDF5E084918F010F5F1F4F882314
:1079E00021F00E941C87F801F6CFEBECF5E08491C2
:1079F0008F010F5F1F4F882321F00E941C87F80121
:107A0000F6CF4091E8075091E9076091EA0770913D
:107A1000EB0789EC95E00E94E3814091EC075091DF
:107A2000ED076091EE077091EF0786EC95E00E94FC
:107A3000E3814091F0075091F1076091F207709156
:107A4000F30783EC95E00E94E381EBEBF5E0849192
:107A50008F010F5F1F4F882321F00E941C87F801C0
:107A6000F6CF409125025091260260912702709135
:107A7000280289EB95E00E94E38140912902509110
:107A80002A0260912B0270912C0286EB95E00E94F5
:107A9000E38140912D0250912E0260912F0270914E
:107AA000300283EB95E00E94E3818AE00E941C870C
:107AB0000FC383E50E9453BE882309F409C30E94C3
:107AC000FDBE909324028093230202C38DED90E0CB
:107AD0000E9495BE8111FCC283E50E9453BE88239B
:107AE00009F4F6C20091690410E00E94FDBE000F87
:107AF000111FF801EF5DFD4F91838083E9C280E59E
:107B00000E9453BE882309F4E3C20E94FDBE8C018B
:107B100083E50E9453BE882321F00E94FDBE7C01B4
:107B200003C0EE24EA94FE2CC7010196039708F0E7
:107B3000CFC217FDCDC2E0ECF2E0C8019927219138
:107B400031912817390709F4C3C233E0E031F30754
:107B5000B1F75AC683E50E9453BE882319F00E94EC
:107B600021E202C084E091E099A388A380E50E940D
:107B700053BE882349F00E9421E2893843E19407EB
:107B800028F088E893E102C088EE93E09A83898325
:107B9000BE01605E7F4FCE0101960E94EC7898C2D4
:107BA00085E40E9453BE811110C080E50E9453BE3F
:107BB000882399F00E9415BF609347027093480292
:107BC0008093490290934A0208C00E94FDBE181695
:107BD00019065CF7E3EDF3E371C089E40E9453BE3C
:107BE000882381F00E9415BF2CEA35EC47E25EE362
:107BF0000E9491E860934F0270935002809351026B
:107C00009093520284E40E9453BE882381F00E9424
:107C100015BF2CEA35EC47E25EE30E942BED609342
:107C20004B0270934C0280934D0290934E02E8E316
:107C3000F4E484918F010F5F1F4F882321F00E948D
:107C40001C87F801F6CF409147025091480260919D
:107C5000490270914A0283EF95E00E94E3812CEA89
:107C600035EC47E25EE360914F02709150028091E3
:107C70005102909152020E942BEDAB01BC018FEE9C
:107C800095E00E94C8812CEA35EC47E25EE3609102
:107C90004B0270914C0280914D0290914E020E94D5
:107CA00091E8AB01BC018BEE95E00E94C8818AE0AF
:107CB0000E941C870DC20E941C87F80184918F01CD
:107CC0000F5F1F4F8111F7CF06EA13E0D8018D91A6
:107CD0008D01882309F41FCA0E941C87F7CF0E94D8
:107CE0004ACCF6C10E9432C8F3C10E94A3D4F0C1AD
:107CF00080E00E940DBCECC1E1EFF4E0FCAFEBAF23
:107D00008DEF282E84E0382E20EA34E021963FAF14
:107D10002EAF219700E010E021964EAD5FAD219788
:107D2000405A544029965FAF4EAF29972196AEAD89
:107D3000BFAD21978D912196BFAFAEAF219788231C
:107D400009F4ACC0F801EB5DFD4F20813181428127
:107D50005381F801E851F84F6081718182819381EC
:107D60000E944FEC20E030E040E05FE30E9491E8A9
:107D70009B01AC01F10160817181828193810E943C
:107D800075EE181634F4C8018851934C0E940749C7
:107D900003C060E070E0CB01D1018D909D90AD906B
:107DA000BC90F801EB5CF24F20813181428153811C
:107DB0000E944FEC9B01AC01C501B4010E944EEC46
:107DC0006B017C0120E030E040EA51EC0E9475EE4E
:107DD00087FD35C020E030E040EA51E4C701B6013C
:107DE0000E942CE818165CF1EBADFCAD4080518090
:107DF00062807380A7019601C301B2010E944EEC1C
:107E00006B017C01A30192010E944EEC9B01AC012D
:107E1000C501B4010E944FECD1016D937D938D9308
:107E20009C931397EBADFCADC082D182E282F382CA
:107E300029968EAD9FAD29970E94FFBD2FC0E3ED1F
:107E4000F3E384918F010F5F1F4F882321F00E947D
:107E50001C87F801F6CFE5E1F6E084918F010F5F12
:107E60001F4F882321F00E941C87F801F6CF61E0A4
:107E700087E096E00E94F7D80E94075888E290E0D9
:107E80009A83898388EC90E099A388A3BE016F5FF1
:107E90007F4FCE0180960E94EC781AC12BAD3CAD8D
:107EA0002C5F3F4F3CAF2BAF0C5F1F4F34E0230ED6
:107EB000311C0C30110509F02FCF0E94FD480E94A3
:107EC00042CD60E087EF95E00E94F7D883E992E029
:107ED00099A388A304E610E01A830983BE01605EBB
:107EE0007F4FCE0101960E94EC788AEB92E099A335
:107EF00088A31A830983BE01605E7F4FCE0101967D
:107F00000E94EC78E5C0E3EDF3E384918F010F5F0D
:107F10001F4F882321F00E941C87F801F6CFE3E36E
:107F2000F6E084918F010F5F1F4F882309F4D0C0C2
:107F30000E941C87F801F5CF0E94B44DC9C083E5AB
:107F40000E9453BE882321F00E94D2BE91E089276F
:107F50000E94C749BDC0E8E3F4E484918F010F5F3C
:107F60001F4F882321F00E941C87F801F6CFEEE511
:107F7000F6E084918F010F5F1F4F882309F499C8A1
:107F80000E941C87F801F5CFE7E4F6E084918F01A9
:107F90000F5F1F4F882309F4BEC80E941C87F80199
:107FA000F5CF4091750E5091760E6091770E7091DD
:107FB000780E84E496E00E94E381ADC8E3EDF3E33C
:107FC00084918F010F5F1F4F882321F00E941C872F
:107FD000F801F6CFE8E6F6E084918F010F5F1F4FBE
:107FE000882309F475C00E941C87F801F5CF81E051
:107FF0008093AA021092210883E50E9453BE882331
:1080000009F4FFC30E94D2BE811162C0FAC3E0929C
:108010006A04E8E3F4E484918F010F5F1F4F882323
:1080200021F00E941C87F801F6CFB701772787E778
:1080300096E00E94FE818AE00E941C8749C080E091
:1080400048C00E949FBA83E50E9453BE882309F46A
:1080500063C00E94D2BEEE24E394F12C082FA3014A
:108060009201C501B4010E9456BC6B017C012CEA4F
:1080700035EC47E257E3C501B4010E944FECAB0178
:10808000BC018CE392E00E94C8812CEA35EC47E207
:1080900057E3C301B2010E944FECAB01BC0187E37F
:1080A00092E00E94C8812CEA35EC47E257E3C70111
:1080B000B6010E944FECAB01BC0182E392E00E944A
:1080C000C8818AE00E941C870E9485BA0E9442CD26
:1080D00081E010922A0D1092290D81111AC00C9482
:1080E000012984918F010F5F1F4F882321F00E9487
:1080F0001C87F801F6CF60912B0D70912C0D89E84B
:1081000096E00E94158282E20E941C878AE00E940B
:108110001C870E94648DA0C381E09DCF0E942DE248
:10812000AB01BC01409306145093071460930814EC
:108130007093091485E593E10E94F08EC9CF0E94E7
:108140002DE2AB01BC0140930614509307146093D9
:1081500008147093091485E593E10E94F08E0C9445
:108160007F3661E08D2D0E945C5A6E2D8D2D0E9410
:108170002D5AB7018D2D0E94985A0930110509F02A
:10818000A7CFF0921408E0921308A2CF0E94FDBE80
:10819000909312088093110880E00E94D3D00E942F
:1081A000FDBE8635910544F40E9410C560E087EB62
:1081B00093E00E94F7D802C00E943B7960911108B9
:1081C00070911208072E000C880B990B0E9432E860
:1081D000209198043091990440919A0450919B0405
:1081E0000E9475EE1816B4F48BE993E09F938F9379
:1081F0008091690490E001969F938F9380EB93E0C8
:108200009F938F931F920E9420790FB6F894DEBF40
:108210000FBECDBF0E94E2E181E080930402109284
:108220002A0D1092290D23961CAE1DAE1EAE1FAE58
:10823000239727961CAE1DAE1EAE1FAE27971BAE12
:108240002C961FAE2C979CE360969FAF6097ACE195
:108250006496AFAF6497B6E46896BFAF6897C12CD9
:10826000D12C70E8E72EEFEBFE2E812C912C5401DF
:108270006091110870911208072E000C880B990B61
:108280000E9432E8162F072F782E692E262F372FBF
:10829000482F592FB601C7010E942CE8882311F1FD
:1082A000209198043091990440919A0450919B0434
:1082B000612F702F872D962D0E942CE8881F88270C
:1082C000881F8BAF2896EFAD2897EE2379F088238F
:1082D00069F080910402882309F4FACE60E08BE90A
:1082E00093E06DC11C2D0D2D7E2C6F2C0E94975B91
:1082F0006B017C01DC01CB0127962CAD3DAD4EAD71
:108300005FAD2797821B930BA40BB50BB7FD47C03E
:10831000D701C60188519C4FAF4FBF4F27968CAFF6
:108320009DAFAEAFBFAF27970E946BA5ECEAF3E01D
:1083300084912F019FEF491A590A882321F00E9446
:108340001C87F201F5CF81149104A104B104D1F08E
:10835000D501C401805F984DAF4FBF4FBC01CD0127
:108360006C197D098E099F0928EE33E040E050E04A
:108370000E94F1EBCA01B9010E9489878AE00E943C
:108380001C870DC0E9EAF3E084912F01AFEF4A1A90
:108390005A0A882321F00E941C87F201F5CF0E941F
:1083A000DF8A3BD7609198047091990480919A0478
:1083B00090919B040E9493ED072E000C880B990B63
:1083C0000E9432E81B012C019B01AC01612F702F30
:1083D000872D962D0E944EEC9F7781149104A10465
:1083E000B10449F420E030E040E85FE30E942CE86B
:1083F00087FF0BC008C020E030E040E450E40E945A
:1084000075EE181614F446015701BBADBB2309F4F1
:1084100043C023962CAD3DAD4EAD5FAD23972115E6
:1084200031054105510541F0D701C601821B930B6F
:10843000A40BB50BB7FD30C09101A2012C966FAD16
:108440002C9760967FAD609764968FAD6497689621
:108450009FAD68970E944EEC20E030E040EC5FE377
:108460000E942CE887FD35CFD701C601805A95417F
:10847000AF4FBF4F23968CAF9DAFAEAFBFAF23972B
:108480002C962FAE2C9760963FAE609764964FAEB9
:10849000649768965FAE689780910402882309F418
:1084A00018CF81149104A104B10429F4C12ED02E57
:1084B000E72CF62CDDCE90E1C91A97E2D90AE10843
:1084C000F108C818D908EA08FB08F7FE02CFEECF7A
:1084D0000E94FDBE90931608809315080E94A0D0BC
:1084E0000E94FDBE069714F00E943B7981E08093C4
:1084F000040210922A0D1092290D80916A04809333
:10850000690423961CAE1DAE1EAE1FAE23972796A0
:108510001CAE1DAE1EAE1FAE27971BAE2C961FAE17
:108520002C97ACE36096AFAF6097BCE16496BFAFA9
:108530006497E6E46896EFAF6897C12CD12C50E8B9
:10854000E52E6FEBF62E812C912C540160911508CD
:1085500070911608072E000C880B990B0E9432E8C8
:10856000162F072F782E692E262F372F482F592F99
:10857000B601C7010E942CE8882321F120919C04B8
:1085800030919D0440919E0450919F04612F702F63
:10859000872D962D0E942CE8881F8827881F8BAF77
:1085A0002896FFAD2897FF2389F0882379F08091E2
:1085B0000402882309F48CCD60E08BEC93E00E94E8
:1085C000F7D886CD1C2D0D2D7E2C6F2C0E94975B2D
:1085D0006B017C01DC01CB0127962CAD3DAD4EAD8E
:1085E0005FAD2797821B930BA40BB50BB7FD47C05C
:1085F000D701C60188519C4FAF4FBF4F27968CAF14
:108600009DAFAEAFBFAF27970E946BA5E8EDF3E03B
:1086100084912F019FEF491A590A882321F00E9463
:108620001C87F201F5CF81149104A104B104D1F0AB
:10863000D501C401805F984DAF4FBF4FBC01CD0144
:108640006C197D098E099F0928EE33E040E050E067
:108650000E94F1EBCA01B9010E9489878AE00E9459
:108660001C870DC0E5EDF3E084912F01AFEF4A1AAE
:108670005A0A882321F00E941C87F201F5CF0E943C
:10868000DF8ACBD560919C0470919D0480919E04FB
:1086900090919F040E9493ED072E000C880B990B7C
:1086A0000E9432E81B012C019B01AC01612F702F4D
:1086B000872D962D0E944EEC9F7781149104A10482
:1086C000B10449F420E030E040E85FE30E942CE888
:1086D00087FF0BC008C020E030E040E450E40E9477
:1086E00075EE181614F446015701BBADBB2309F40F
:1086F00043C023962CAD3DAD4EAD5FAD2397211504
:1087000031054105510541F0D701C601821B930B8C
:10871000A40BB50BB7FD30C09101A2012C966FAD33
:108720002C9760967FAD609764968FAD649768963E
:108730009FAD68970E944EEC20E030E040EC5FE394
:108740000E942CE887FD33CFD701C601805A95419E
:10875000AF4FBF4F23968CAF9DAFAEAFBFAF239748
:108760002C962FAE2C9760963FAE609764964FAED6
:10877000649768965FAE689780910402882309F435
:1087800016CF81149104A104B10429F4C12ED02E76
:10879000E72CF62CDBCE90E1C91A97E2D90AE10862
:1087A000F108C818D908EA08FB08F7FE00CFEECF99
:1087B0000E94A3D488E50E9453BE882319F05F9AD3
:1087C0001092ED0489E50E9453BE882319F08A9A1D
:1087D0001092EE048AE50E9453BE882351F09FB7A1
:1087E000F894809108018160809308019FBF1092E6
:1087F000EF0485E40E9453BE882309F469CC129AE1
:1088000067CC0E94818D64CC0E94A3D4D02E60E0FE
:10881000802F0E945C5A4FEFE416F40659F4802F23
:108820000E94E9D931E020E0892B09F030E0032FE4
:10883000122F05C0EA94EF2861F000E010E08D2DC2
:108840000E94E9D98017910709F442CC0E94DF8A7F
:10885000F6CF01E010E0F3CFCA58DF4F0FB6F8941F
:10886000DEBF0FBECDBFDF91CF911F910F91FF9063
:10887000EF90DF90CF90BF90AF909F908F907F90C0
:108880006F905F904F903F902F9008950895FC0156
:10889000A681B7818281481B8581483018F0A80FD6
:1088A000B11D4770382F369536953695562F57702F
:1088B00080E890E002C0959587955A95E2F7439F2E
:1088C000402D1124669566956695E62FF0E0E40F3D
:1088D000F11DEA0FFB1F3081222311F0832B02C010
:1088E0008095832380830895FB014181DC011296EA
:1088F0002C911297421760F013962C91139724171E
:1089000038F0608115962C91621710F42481BFCF46
:108910000895FC0180819281980F928321819217A2
:1089200060F494819F5F94839381890F821710F084
:108930008FEF820F838381E0089580E00895FC012A
:1089400012828081815083831482089580E008958B
:108950000B96FC01849108950A96FC018491089578
:10896000FC0184910895FCDF882321F0823011F00E
:1089700083E0089586E00895FC01E60FF11D8491DF
:1089800090E0982F88273196E4918E0F911D0895DD
:1089900068E0F2CF66E0F0CF81E008952F923F9239
:1089A0004F925F926F927F928F929F92AF92BF92FF
:1089B000CF92DF92EF92FF920F931F93CF93DF93AB
:1089C00000D000D0CDB7DEB78C010E94975BF801D4
:1089D000C680D780E084F184C114D104E104F1049D
:1089E00009F0F6C22485222309F460C332852150A0
:1089F000248721E0230F22874585241301C0128696
:108A0000F80124E0329FE00DF11D1124C684D784C3
:108A1000E088F188F801C282D382E482F582DC0129
:108A2000CB018C0D9D1DA11DB11D86839783A08751
:108A3000B18784819581892B09F438C3FFB7FD8301
:108A4000F894F80122803380048115818091B70267
:108A5000853221F08F3F09F0B8C205C0E3E6F0E5AA
:108A600024912E83EDC085E28093B702E3E6F0E522
:108A7000E491EF3F09F4A9C2E23009F474C054F55F
:108A8000EE2309F453C0E13009F0D9C01092800000
:108A90001092810080918100886080938100809194
:108AA0008100816080938100EBEDFCE0E491F0E0D7
:108AB000EE0FFF1FEE57F34F8591949190937F0433
:108AC00080937E04E1E2FDE0E491E0937D0481E0A7
:108AD0008E83B9C0E43009F48EC00CF468C0E53070
:108AE00009F0ADC010922001109221018091210166
:108AF0008860809321018091210181608093210110
:108B0000EBEDFCE0E491F0E0EE0FFF1FEE57F34FCA
:108B1000859194919093760480937504E1E2FDE051
:108B2000E491E093740425E02E838DC014BC15BC41
:108B300084B5826084BD85B5816085BDEBEDFCE0C8
:108B4000E491F0E0EE0FFF1FEE57F34F8591949103
:108B50009093820480938104E1E2FDE0E491E0934C
:108B600080041E8270C01092B0001092B1008091FB
:108B7000B00082608093B0008091B10081608093EA
:108B8000B100EBEDFCE0E491F0E0EE0FFF1FEE57DB
:108B9000F34F859194919093871480938614E1E22A
:108BA000FDE0E491E093881492E09E834CC0109223
:108BB00090001092910080919100886080939100C4
:108BC00080919100816080939100EBEDFCE0E49155
:108BD000F0E0EE0FFF1FEE57F34F859194919093C5
:108BE0007C0480937B04E1E2FDE0E491E0937A046D
:108BF000E3E0EE8328C01092A0001092A1008091C3
:108C0000A10088608093A1008091A1008160809381
:108C1000A100EBEDFCE0E491F0E0EE0FFF1FEE575A
:108C2000F34F859194919093790480937804E1E2D5
:108C3000FDE0E491E0937704F4E0FE8304C0EE836A
:108C40008E8187FDC2C12101612C712C61E085E21A
:108C50000E945C5A4801A12CB12C8E818D7F09F0B5
:108C6000BDC060E072E18AE790E0A50194010E9436
:108C700013EC29833A834B835C8369017A0191E089
:108C8000C91AD108E108F108EFEFCE16D104E104CA
:108C9000F10409F008F44DC060E472E48FE090E064
:108CA000A50194010E9413EC69017A01F1E0CF1A49
:108CB000D108E108F1082E81223001F58FEFC816A6
:108CC000D104E104F10409F008F4EEC160E970EDAB
:108CD00083E090E0A50194010E9413EC69017A0100
:108CE00091E0C91AD108E108F108EFEFCE16D104DE
:108CF000E104F10409F0E0F583E069C0FFEFCF166D
:108D0000D104E104F104B9F0B0F068E478EE81E058
:108D100090E0A50194010E9413EC69017A0181E0C1
:108D2000C81AD108E108F1089E81992309F49AC173
:108D300090C181E001C082E09E819923A1F047C0EB
:108D400089819A81AB81BC812AE0B595A7959795D9
:108D500087952A95D1F76C017D01E1E0CE1AD10803
:108D6000E108F10885E095B5987F892B85BDA1C004
:108D700068E478EE81E090E0A50194010E9413EC94
:108D800069017A01F1E0CF1AD108E108F1082FEF6B
:108D9000C216D104E104F10409F008F428C164E228
:108DA00074EF80E090E0A50194010E9413EC69014A
:108DB0007A01E1E0CE1AD108E108F108FFEFCF1601
:108DC000D104E104F10411F008F013C185E09091A1
:108DD000B100987F892B8093B1006BC060E072E195
:108DE0008AE790E0A50194010E9413EC69017A01E1
:108DF000E1E0CE1AD108E108F108C114D104F1E094
:108E0000EF06F10488F068E478EE81E090E0A501D7
:108E100094010E9413EC69017A0181E0C81AD1081B
:108E2000E108F10883E001C081E09E81913071F496
:108E300090918100987F892B809381004528462856
:108E40004728D9F52FEF3FEFA90168C0EE81E33045
:108E500071F490919100987F892B8093910045281F
:108E60004628472851F52FEF3FEFA90179C0FE8131
:108E7000F43071F49091A100987F892B8093A10028
:108E8000452846284728C9F42FEF3FEFA9017AC0AB
:108E90002E81253071F490912101987F892B809348
:108EA000210145284628472841F42FEF3FEFA9012B
:108EB0007BC045284628472869F09801220F331FB8
:108EC000D1010E943FEC28EE33E040E050E00E94E8
:108ED000F1EB03C02FEF3FEFA9018E81823081F1CA
:108EE0002CF4882361F08130C9F06FC09E819430EA
:108EF00009F448C0ACF1953009F456C066C0C7BC4F
:108F000020939304309394044093950450939604D3
:108F100080916E00826080936E0057C0D09289006D
:108F2000C092880020938F04309390044093910462
:108F30005093920480916F00826080936F0045C0CF
:108F4000C092B3002093891430938A1440938B14F9
:108F500050938C148091700082608093700035C0B3
:108F6000D0929900C092980020938B0430938C0487
:108F700040938D0450938E048091710082608093A1
:108F8000710023C0D092A900C092A800209387044A
:108F9000309388044093890450938A04809172002E
:108FA00082608093720011C0D0922901C092280182
:108FB0002093830430938404409385045093860463
:108FC00080917300826080937300ED81EFBF6EC06B
:108FD000DC01CB018C199D09AE09BF09B7FD66C044
:108FE0004098F80116821782108611865FC084E0CF
:108FF000EECE62E17AE780E090E0A50194010E9464
:1090000013EC69017A0181E0C81AD108E108F1087E
:109010009FEFC916D104E104F104C9F0C0F08981C1
:109020009A81AB81BC815AE0B595A79597958795B4
:109030005A95D1F76C017D0121E0C21AD108E108EF
:10904000F1088E81882309F48DCE87E0C0CE86E0BA
:1090500073CEEFEFCE16D104E104F10409F048F627
:1090600084E06ACE8FEFC816D104E104F104D1F098
:10907000C8F062E17AE780E090E0A50194010E94E7
:1090800013EC69017A01F1E0CF1AD108E108F10887
:109090002FEFC216D104E104F10411F008F050CE14
:1090A00084E061CE83E05FCE82E091CE26960FB65B
:1090B000F894DEBF0FBECDBFDF91CF911F910F910E
:1090C000FF90EF90DF90CF90BF90AF909F908F90E8
:1090D0007F906F905F904F903F902F9008952091D8
:1090E000A30430E0F901E35FFA4F80832F5F3F4F25
:1090F000237033272093A3048091AF068F5F809362
:10910000AF060895CF93FC0180818B33A1F080914D
:10911000AF06843080F4C62FBF018091A30420E6FF
:10912000829FC0011124825D9A4F0E949CEF8C2F78
:10913000D6DF81E001C080E0CF910895DF92EF9209
:10914000FF920F931F93CF93DF93CDB7DEB76E9748
:109150000FB6F894DEBF0FBECDBF609122087091AC
:1091600023086115710501F14DE150E0CE01019632
:109170007C010E949CE71E8EF7018F010E191F09CA
:10918000D190DD2019F09AE0D912F7CFF701E00F66
:10919000F11F108260E0C701B5DF882329F0C70105
:1091A0000E94488A811109C081E0209122083091F3
:1091B0002308232BA1F480E012C0DD2049F00F5FCB
:1091C0001F4F8091220890912308080F191F02C099
:1091D00000E010E01093230800932208E5CF6E967C
:1091E0000FB6F894DEBF0FBECDBFDF91CF911F91B8
:1091F0000F91FF90EF90DF90089529E035E045E072
:1092000055E061E075E08DEF94E00C948A97FC01E5
:10921000659175918591949108950E94975B6093F3
:109220002D0D70932E0D80932F0D9093300D08957A
:109230000F931F93CF93DF93E0911914F0911A14B9
:10924000428153816481758114161506160617062E
:1092500004F52091F40C20FF1CC03CB12091730454
:1092600032953695377041E03427832F81702E7FF9
:10927000822B80937304909172049170892349F03A
:1092800080912D05816080932D0580E090E00E9403
:1092900062D4E0911914F0911A1486819781A08507
:1092A000B185181619061A061B0654F58091F40CA0
:1092B00081FF26C08091030120917304422F50E06A
:1092C000869591E08927082F017010E02227332727
:1092D000201B310B242735272270332724273527DD
:1092E00020937304809172048270282349F0809146
:1092F0002D05826080932D0581E090E00E9462D46C
:10930000E0911914F0911A1482859385A485B5858E
:10931000181619061A061B068CF58091F40C82FFAC
:109320002DC08091F004882349F199B18091730494
:10933000282F30E0892F86958695869591E089279C
:109340008170C82F80E0D82F882799278C1B9D0B10
:109350008227932784709927822793278093730409
:10936000909172049470892349F080912D05846056
:1093700080932D0582E090E00E9462D48091730476
:1093800080937204DF91CF911F910F910895AF9256
:10939000BF92CF92DF92EF92FF920F931F93CF93E2
:1093A000C82F882319F0E7EFF8E00CC0E8E3F4E4F5
:1093B00084918F010F5F1F4F8823A9F30E941C87A0
:1093C000F801F6CF84918F010F5F1F4F882321F0A2
:1093D0000E941C87F801F6CF8AE00E941C87C11109
:1093E0002CC0E8E3F4E484918F010F5F1F4F8823C2
:1093F00021F00E941C87F801F6CFE4EEF8E084919A
:109400008F010F5F1F4F882321F00E941C87F801F6
:10941000F6CF8091790E882321F08AE00E941C8784
:109420003AC0E9EDF8E084918F010F5F1F4F882368
:1094300091F10E941C87F801F6CF40916302509190
:109440006402609165027091660280ED98E00E946E
:10945000E3818AE00E941C878091790E811127C0E8
:10946000CC2319F0E5ECF8E00CC0E8E3F4E48491D7
:109470008F010F5F1F4F8823A9F30E941C87F801FB
:10948000F6CF84918F010F5F1F4F882381F00E94D8
:109490001C87F801F6CFE8E3F4E484918F010F5FB5
:1094A0001F4F882351F20E941C87F801F6CFC1118B
:1094B00024C0E8E3F4E484918F010F5F1F4F8823F9
:1094C00021F00E941C87F801F6CFE4EBF8E08491CC
:1094D0008F010F5F1F4F882321F00E941C87F80126
:1094E000F6CFE8E3F4E484918F010F5F1F4F8823E8
:1094F00021F00E941C87F801F6CF4091210E509177
:10950000220E6091230E7091240E8CEA98E00E9446
:10951000E3814091250E5091260E6091270E7091A7
:10952000280E89EA98E00E94E3814091290E50912B
:109530002A0E60912B0E70912C0E86EA98E00E9404
:10954000E38140912D0E50912E0E60912F0E70915F
:10955000300E83EA98E00E94E3818AE00E941C8733
:10956000C11124C0E8E3F4E484918F010F5F1F4F21
:10957000882321F00E941C87F801F6CFE5E8F8E087
:1095800084918F010F5F1F4F882321F00E941C8759
:10959000F801F6CFE8E3F4E484918F010F5F1F4FE9
:1095A000882321F00E941C87F801F6CF4091510ECC
:1095B0005091520E6091530E7091540E8CE798E0CA
:1095C0000E94E3814091550E5091560E6091570EC6
:1095D0007091580E89E798E00E94E3814091590EFE
:1095E00050915A0E60915B0E70915C0E86E798E088
:1095F0000E94E38140915D0E50915E0E60915F0E7E
:109600007091600E83E798E00E94E3818AE00E94F7
:109610001C87C11124C0E8E3F4E484918F010F5F3B
:109620001F4F882321F00E941C87F801F6CFE1E547
:10963000F8E084918F010F5F1F4F882321F00E9473
:109640001C87F801F6CFE8E3F4E484918F010F5F03
:109650001F4F882321F00E941C87F801F6CF40910C
:10966000390E50913A0E60913B0E70913C0E88E499
:1096700098E00E94AD8140913D0E50913E0E609168
:109680003F0E7091400E85E498E00E94AD814091BC
:10969000410E5091420E6091430E7091440E82E44F
:1096A00098E00E94AD814091450E5091460E609128
:1096B000470E7091480E8FE398E00E94AD818AE0DA
:1096C0000E941C87C11124C0E8E3F4E484918F0157
:1096D0000F5F1F4F882321F00E941C87F801F6CFEF
:1096E000E5EFF7E084918F010F5F1F4F882321F092
:1096F0000E941C87F801F6CFE8E3F4E484918F011F
:109700000F5F1F4F882321F00E941C87F801F6CFBE
:109710004091710E5091720E6091730E7091740EA3
:109720008CEE97E00E94E3814091350E5091360E09
:109730006091370E7091380E89EE97E00E94E381B8
:109740004091310E5091320E6091330E7091340E73
:1097500086EE97E00E94E3818AE00E941C87C11197
:1097600024C0E8E3F4E484918F010F5F1F4F882346
:1097700021F00E941C87F801F6CFE2E7F7E0849120
:109780008F010F5F1F4F882321F00E941C87F80173
:10979000F6CFE8E3F4E484918F010F5F1F4F882335
:1097A00021F00E941C87F801F6CF40914D0E509198
:1097B0004E0E60914F0E7091500E89E697E00E9418
:1097C000E3814091490E50914A0E60914B0E709189
:1097D0004C0E86E697E00E94E3814091EA0D50919D
:1097E000EB0D6091EC0D7091ED0D83E697E00E941A
:1097F000AD814091610E5091620E6091630E709147
:10980000640E80E697E00E94E3814091650E5091DE
:10981000660E6091670E7091680E8DE597E00E946C
:10982000E3814091690E50916A0E60916B0E7091C8
:109830006C0E8AE597E00E94E38140916D0E509195
:109840006E0E60916F0E7091700E87E597E00E942A
:10985000E3818AE00E941C87C11124C0E8E3F4E49C
:1098600084918F010F5F1F4F882321F00E941C8776
:10987000F801F6CFE9E4F7E084918F010F5F1F4F05
:10988000882321F00E941C87F801F6CFE8E3F4E476
:1098900084918F010F5F1F4F882321F00E941C8746
:1098A000F801F6CF4091F1045091F2046091F30475
:1098B0007091F40480E497E00E94E3814091F50404
:1098C0005091F6046091F7047091F8048DE397E0ED
:1098D0000E94E3814091F9045091FA046091FB04E5
:1098E0007091FC048AE397E00E94E3818AE00E9481
:1098F0001C87CC2379F08DE0A82E8EE0B82E99E05D
:10990000C92E9EE0D92E21E1E22E2EE0F22E00E0BB
:1099100010E024C0E8E3F4E484918F010F5F1F4F4F
:10992000882321F00E941C87F801F6CFEDE1F7E0D3
:1099300084918F010F5F1F4F882321F00E941C87A5
:10994000F801F6CFE8E3F4E484918F010F5F1F4F35
:10995000882389F20E941C87F801F6CFB80184E1C0
:1099600097E00E94FE81F501619171915F0181E1B3
:1099700097E00E94FE81F601619171916F018EE086
:1099800097E00E94FE81F701619171917F018BE068
:1099900097E00E94FE818AE00E941C870130110539
:1099A00019F001E010E0DACFC11124C0E8E3F4E4DB
:1099B00084918F010F5F1F4F882321F00E941C8725
:1099C000F801F6CFECEFF6E084918F010F5F1F4FA7
:1099D000882321F00E941C87F801F6CFE8E3F4E425
:1099E00084918F010F5F1F4F882321F00E941C87F5
:1099F000F801F6CF40914702509148026091490228
:109A000070914A0283EF96E00E94E3812CEA35ECE4
:109A100047E25EE360914F027091500280915102E3
:109A2000909152020E942BEDAB01BC0180EF96E0B9
:109A30000E94C8812CEA35EC47E25EE360914B025C
:109A400070914C0280914D0290914E020E9491E8DB
:109A5000AB01BC018DEE96E00E94C8818AE00E94B5
:109A60001C87C1110CC0E8E3F4E484918F010F5FFF
:109A70001F4F882321F00E941C87F801F6CF4091E8
:109A8000B3025091B4026091B5027091B60284EEB7
:109A900096E00E94E3812CEA35EC47E25EE36091B8
:109AA000AF027091B0028091B1029091B2020E9417
:109AB0002BEDAB01BC0181EE96E00E94C8812CEA3F
:109AC00035EC47E25EE36091AB027091AC028091AD
:109AD000AD029091AE020E9491E8AB01BC018EED07
:109AE00096E00E94C8818AE00E941C87C11124C0B0
:109AF000E8E3F4E484918F010F5F1F4F882321F086
:109B00000E941C87F801F6CFE8ECF6E084918F0103
:109B10000F5F1F4F882321F00E941C87F801F6CFAA
:109B2000E8E3F4E484918F010F5F1F4F882321F055
:109B30000E941C87F801F6CF4091750E5091760E69
:109B40006091770E7091780E8FEB96E00E94E38122
:109B50008AE0CF911F910F91FF90EF90DF90CF900F
:109B6000BF90AF900C941C87AF92BF92CF92DF92C0
:109B7000EF92FF920F931F93CF93DF93CDB7DEB792
:109B8000E0970FB6F894DEBF0FBECDBF80E1E0E1F5
:109B9000F3E0DE01919601900D928A95E1F780E164
:109BA000E0E2F3E0DE01519601900D928A95E1F733
:109BB00080E1E0E3F3E0DE01119601900D928A95D9
:109BC000E1F7DE01919661E27EE0AE014F5E5F4F0C
:109BD00021E53EE0CE0101965C0189E39EE08E0125
:109BE0000F5C1F4FCD90DD90ED90FD90FB01C19279
:109BF000D192E192F192BF01FA01C190D190E1902E
:109C0000F190AF01F901C192D192E192F1929F01DD
:109C1000F501C190D190E190F1905F01FC01C192FA
:109C2000D192E192F192CF01A017B107D9F680E06D
:109C300090E8ABEBB4E48093710E9093720EA09316
:109C4000730EB093740E8093350E9093360EA093DE
:109C5000370EB093380E80E090E8ABE3B5E4809324
:109C6000310E9093320EA093330EB093340E1092B7
:109C70004D0E10924E0E10924F0E1092500E80E22A
:109C80009EE4A0E0B0E08093EA0D9093EB0DA093EA
:109C9000EC0DB093ED0D1092490E10924A0E1092F9
:109CA0004B0E10924C0E80E090E0A0E0B1E4809367
:109CB000610E9093620EA093630EB093640E809336
:109CC000650E9093660EA093670EB093680E8DECB0
:109CD0009CECACECBEE38093690E90936A0EA0936B
:109CE0006B0EB0936C0E80E090E0A0EAB0E480933D
:109CF0006D0E90936E0EA0936F0EB093700E8CE06D
:109D0000E1EFF4E0DF011D928A95E9F71092750EFC
:109D10001092760E1092770E1092780E87ED90E0EA
:109D200090930E0E80930D0E80EF90E09093100EA6
:109D300080930F0E86E490E090930A0E8093090EB4
:109D40008EE690E090930C0E80930B0E1092120E04
:109D50001092110E1092140E1092130E86EF98E2CC
:109D6000A1E0B2E48093470290934802A093490295
:109D7000B0934A0284E795EDA7E1BFE380934F02D9
:109D800090935002A0935102B093520280E590E06C
:109D9000ACEDB3E480934B0290934C02A0934D0240
:109DA000B0934E0286EF98EAA0EBB3E48093B3023F
:109DB0009093B402A093B502B093B60283EA9FE5F4
:109DC000A6E3B1E48093AF029093B002A093B102F6
:109DD000B093B20286E893E2ABE2B5E48093AB02C3
:109DE0009093AC02A093AD02B093AE021092790EA4
:109DF00080E090E0A0E4B0E480936302909364027A
:109E0000A0936502B093660210920B021092680450
:109E10000E9420970E944D980E948D8480E090E0DF
:109E20000E94FFBD81E090E00E94FFBD82E090E0D3
:109E30000E94FFBD8091750E9091760EA091770ED5
:109E4000B091780E80935F0290936002A0936102BC
:109E5000B0936202E8E3F4E484918F010F5F1F4F37
:109E6000882321F00E941C87F801F6CFECE9F6E088
:109E700084918F010F5F1F4F882321F00E941C8760
:109E8000F801F6CFE0960FB6F894DEBF0FBECDBF57
:109E9000DF91CF911F910F91FF90EF90DF90CF90C6
:109EA000BF90AF900895FC0120E03EE2DB014C91B1
:109EB000403241F0283011F430833196DB014C916F
:109EC000408331962F5F6F5F7F4F2B3079F7108281
:109ED0000895FC01238121110C944C91089520E8F0
:109EE00033E0FC01318320830496F3CFCF92DF92DD
:109EF000FF920F931F93CF93DF931F921F92CDB7C3
:109F0000DEB76901DB0112960D911C911397423364
:109F100009F471C0B8F4453109F47AC0473109F445
:109F20008BC0443109F0A1C0D80115962C9115972A
:109F30001696ED91FC911797CF01820F911D820F1C
:109F4000911D5EC0463409F487C0473409F488C0C7
:109F50004B3309F08AC0F90181819381913029F056
:109F6000933031F4482F885004C048E0480F01C0B6
:109F7000482F21E0D80113963C91381708F420E0CF
:109F800031E0F8015281451708F430E051E04817FC
:109F900008F050E0822F852B382319F4252309F48B
:109FA00064C0D6011296FC90913051F030F092309E
:109FB00049F0933051F42FEF09C020E031E007C0A1
:109FC00021E004C020E03FEF02C020E030E0F7FED7
:109FD00008C0B601C8012A8339830E9474443981BC
:109FE0002A81F6018081830F80838181820F8183A2
:109FF000FF0C69F73AC0B901C8010E94744435C02A
:10A000001192E817F907E1F7C8010E949F442DC09B
:10A01000C8010E948944882349F1F80125810680FE
:10A02000F781E02DCF01820F911D820F911D1192BA
:10A03000E817F907E1F719C0D9011C92F8018281EC
:10A0400011968C9311978581815012968C9312975B
:10A05000838113968C9309C0D80115968C9103C007
:10A06000D80111968C91F601808381E00F900F90BA
:10A07000DF91CF911F910F91FF90DF90CF900895C6
:10A08000DB01ED91FC9119948F929F92BF92CF9238
:10A09000DF92EF92FF920F931F93CF93DF931F9264
:10A0A000CDB7DEB74C01062FF42E122F522FE62E1D
:10A0B000E20EBB24BA946C018CE1C80ED11C8E2D2B
:10A0C000851B583078F0F40162817381848FF58E9E
:10A0D000178EB68E96014BE3C4015983D1DF5981A7
:10A0E0005850EDCF812F887F080F212F277019F14D
:10A0F00087E02827F40162817381048FF58E178E23
:10A100002F5F27708FEF90E001C0880F2A95EAF744
:10A11000868F9401245E3F4F4BE3C4010F90DF9183
:10A12000CF911F910F91FF90EF90DF90CF90BF9054
:10A130009F908F90A5CF0F90DF91CF911F910F919E
:10A14000FF90EF90DF90CF90BF909F908F900895F9
:10A15000EF92FF920F931F93CF93DF937C01D62F43
:10A16000122FC42F040F212F4C2F6D2FC7018CDF0E
:10A17000CF5F0C13F8CFDF91CF911F910F91FF901C
:10A18000EF900895EF92FF920F931F93CF93DF9379
:10A190001F92CDB7DEB78C01DC011296ED90FC90DA
:10A1A0001397D196ED91FC91D29782E0199520E01A
:10A1B00030E04AE0B701C80163DFF82ED801D1963C
:10A1C000ED91FC91D29783E01995D801D196ED914C
:10A1D000FC91D29780E01995FF2081F1F80162810E
:10A1E00073819E012F5F3F4F46E4C80149DF89819B
:10A1F000D8018C9312966D917C9113979E012F5FDD
:10A200003F4F47E4C8013CDF8981F80181836281C7
:10A21000738120E030E048E4C80132DFD8011B96AA
:10A220008C931B9798012D5C3F4F12966D917C91FA
:10A23000139747E1C80124DF81E001C080E00F905F
:10A24000DF91CF911F910F91FF90EF90089588E2D9
:10A2500090E00197F1F708952EE93FE0009729F08B
:10A26000F9013197F1F70197F9CF08950F93FC01A8
:10A270000150040F84A996A9941718F0081728F420
:10A2800002C0081750F0041740F42150260F83A98C
:10A2900095A9961720F4281720F480E007C0281706
:10A2A00020F481E0261710F0F8CF81E00F91089597
:10A2B000DF92EF92FF920F931F93CF93DF93EC0106
:10A2C000162FF42EE22ED2DF882329F02E2D4F2DCB
:10A2D000612FCE013DDFDF91CF911F910F91FF9054
:10A2E000EF90DF9008952F923F925F926F927F924E
:10A2F0008F929F92AF92BF92CF92DF92EF92FF9296
:10A300000F931F93CF93DF931F92CDB7DEB71C013E
:10A31000C62E142FD22EDC011496ED90FC901597CA
:10A32000C7010E94B044082FF101848195810E94E9
:10A33000B344982E013019F48FE0A82E02C0AA244D
:10A34000AA94D10114968D919C9115970E94AC44CA
:10A35000082FF101848195810E94A844B82ED10173
:10A3600014968D919C9115970E94C844B0E6BD1536
:10A3700030F4009721F0E80EF91E01E611C0F1015A
:10A38000848195810E94CA44F0E4FD1530F4009761
:10A3900021F0E80EF91E01E403C021E1E20EF11CF8
:10A3A000BD1480F4D10150961C92509753961C9284
:10A3B000539754961C92549751961C9251975296CB
:10A3C0001C92C5C0B01670F3892D90E0F70124915E
:10A3D0002F3F21F4FFEFEF1AFF0A5AC00D114FC0B3
:10A3E000D10114968D919C9115970E94B0449701CC
:10A3F0002F5F3F4FF701882311F08230E1F4849101
:10A40000D10153968C935397F901249154962C9330
:10A410005497F7013396E4915096EC935097F701D7
:10A420003496E4915196EC935197F7013596E49167
:10A430005296EC9320C08491982F9F709250D10136
:10A4400052969C93529782958F7051968C93519708
:10A45000F9012491822F8F7054968C9354972295F2
:10A460002F7053962C935397F7013296E491E2950F
:10A47000EF705096EC93E114F10479F468C0F701A1
:10A480003296E491EA219C012E0F311DE20EF31E5B
:10A490000B1509F487CF0F5F99CFF1018481958166
:10A4A0000E94B344B82ED10153969C905397549672
:10A4B000DC90549751968C915197C80E52969C916E
:10A4C0009D0D512E591A0D2D292D452D6C2DC10193
:10A4D000CDDE8823C9F1C7018B0D911D5C0187E09A
:10A4E000890DF82EF694F694F694D50C41019CE172
:10A4F000890E911C6F2C712C5D1431F15C2D85013E
:10A50000802F8A198F15E0F4F8018491D1011296F9
:10A510006D917C9113975C965C935C975D965C92D1
:10A520005D975F961C925F975E968C9394014BE3C8
:10A53000C1015983A5DD0F5F1F4F5981585FE0CFDF
:10A54000A60CB71C5394D8CFF101808901C080E0DC
:10A550000F90DF91CF911F910F91FF90EF90DF90BF
:10A56000CF90BF90AF909F908F907F906F905F90B3
:10A570003F902F9008954F925F926F927F928F92AB
:10A580009F92AF92BF92CF92DF92EF92FF920F9382
:10A590001F93CF93DF93CDB7DEB762970FB6F894D2
:10A5A000DEBF0FBECDBF1092D7070E94975B009110
:10A5B000C9041091CA042091CB043091CC046B01E2
:10A5C0007C01C01AD10AE20AF30AF7FC13C02091F9
:10A5D000C80420952093C804DC01CB018A549C4F09
:10A5E000AF4FBF4F8093C9049093CA04A093CB048C
:10A5F000B093CC04FF24F3948091C804811101C06E
:10A60000F12C0E949BD880913011853198F4FF2065
:10A6100049F08091130890911408892B19F003E5F3
:10A620001AE002C006E319E023E14FE061E089E0AF
:10A630000E944DC2809130118D3108F091C1883057
:10A64000D0F56091110870911208072E000C880B4C
:10A65000990B0E9432E820E030E040E05FE30E9486
:10A660004FEC0E9493ED7C876B87643671052CF468
:10A670006A30710524F426E003C022E101C02CE019
:10A6800082E190E0821B910997FD0196959587954F
:10A690009195819591098B5F8093331187E0809329
:10A6A0003411CE010B960E9401D80E94E85E83E32C
:10A6B00099E00E94DB5E809130118D3108F044C03A
:10A6C00080913211853108F43FC0609198047091F7
:10A6D000990480919A0490919B040E9493ED072E17
:10A6E000000C880B990B0E9432E820E030E040E03B
:10A6F0005FE30E944FEC0E9493ED9B017E876D8784
:10A70000643671050CF066C32A3031050CF060C365
:10A7100026E082E190E0821B910997FD01969595D4
:10A7200087959195819591098B5F809333118CE189
:10A7300080933411CE010D960E9401D80E94E85EEC
:10A7400083E399E00E94DB5E80913011853138F51A
:10A7500080913211813118F16091110870911208C5
:10A76000072E000C880B990B0E9432E82091980468
:10A770003091990440919A0450919B040E9475EE87
:10A7800018160CF029C310921C1102E022E041E1DE
:10A790006DE08CEF90E18CDD81E080931C11809165
:10A7A00030118830D0F56091150870911608072E89
:10A7B000000C880B990B0E9432E820E030E040E06A
:10A7C0005FE30E944FEC0E9493ED788B6F876436B5
:10A7D00071052CF46A30710524F426E003C022E1EF
:10A7E00001C02CE082E190E0821B910997FD019667
:10A7F000959587959195819591098F5A80933311FD
:10A8000087E080933411CE010F960E9401D80E94F8
:10A81000E85E83E399E00E94DB5E809130118D3128
:10A8200008F044C080913211853108F43FC0609136
:10A830009C0470919D0480919E0490919F040E94BD
:10A8400093ED072E000C880B990B0E9432E820E054
:10A8500030E040E05FE30E944FEC0E9493ED9B01EB
:10A860007A8B698B643671050CF0C0C22A303105D1
:10A870000CF0BAC226E082E190E0821B910997FDBC
:10A880000196959587959195819591098F5A809319
:10A8900033118CE180933411CE0141960E9401D88E
:10A8A0000E94E85E83E399E00E94DB5E80913011B4
:10A8B000853138F580913211813118F16091150898
:10A8C00070911608072E000C880B990B0E9432E835
:10A8D00020919C0430919D0440919E0450919F04CE
:10A8E0000E9475EE18160CF083C210921C1102E043
:10A8F00022E042E168E58CEF90E1DADC81E08093D0
:10A900001C11809130118C3158F5809132118431B5
:10A9100038F120911308309114082F5F3F4F44E61F
:10A92000429FC001439F900D112497FF02C08150A8
:10A930009F4F292F392F330F330B3A832983232B32
:10A9400079F088E6809333118BE180933411CE0146
:10A9500001960E9401D80E94E85E85E20E94307450
:10A9600080913011843328F4809132118A3208F0BA
:10A9700047C280913011853328F4809132118133A0
:10A9800008F063C280918A11882309F44AC080913B
:10A990003011843308F045C080913211823308F4BD
:10A9A00040C020915813222319F1809102149091F4
:10A9B0000314A0910414B09105140097A105B105EA
:10A9C00009F44AC2BC01CD016D597F4F8F4F9F4F93
:10A9D00024E630E040E050E00E94F1EB6091061484
:10A9E0007091071480910814909109140E94F1EB62
:10A9F00048E4249FB0011124072E000C880B990B0A
:10AA00000E9432E82AE037ED43E25CE30E9491E8DD
:10AA10000E9498ED262F02E042E367E38CEF90E17D
:10AA200047DC80913011813308F060C08091321191
:10AA3000893208F45BC00E9429C52B013C018CE3DC
:10AA4000882E912CA12CB12CC301B201A501940137
:10AA50000E94F1EBCA01B901A50194010E94F1EB3A
:10AA6000CA01962E872E59018E010F5F1F4F41E8B4
:10AA7000441641E5540641E06406710408F4EEC151
:10AA8000B90128E130E040E050E00E94F1EB2901FB
:10AA90003A018F929F92C50168E170E00E9413EF26
:10AAA0009F938F935F924F928FE199E09F938F9343
:10AAB0001F930F930E94C5E70FB6F894DEBF0FBE39
:10AAC000CDBF9AE0491651046104710408F0F5C144
:10AAD00097E0892F880F980F9195955A909333118D
:10AAE00080E380933411C8010E94E85EE091F61083
:10AAF000F091F71084818111D4C06091FD047091B0
:10AB0000FE048091FF04909100050E9493ED7A83EA
:10AB10006983CE0101960E9495D7BC0189ED94E02E
:10AB20000E949CEF609101057091020580910305E0
:10AB3000909104050E9493ED7A836983CE0101967A
:10AB40000E9495D7BC0184ED94E00E949CEF2CEA12
:10AB500035EC47E257E36091050570910605809159
:10AB60000705909108050E944FEC20E030E048EC8A
:10AB700052E40E9491E80E9493ED4B015C0197FD25
:10AB800019C090E1891697E29906A104B104E4F096
:10AB9000C501B40120E137E240E050E00E9413EC2F
:10ABA000CA01B9012AE030E040E050E00E9413EC15
:10ABB000605D0BC0B094A09490948094811C911C13
:10ABC000A11CB11C6DE201C060E260931A0828EE7E
:10ABD000821623E09206A104B10494F0C501B401E9
:10ABE00028EE33E040E050E00E9413ECCA01B901C6
:10ABF0002AE030E040E050E00E9413EC605D01C0CC
:10AC000060E260931B08C501B40124E630E040E037
:10AC100050E00E9413EC9AE0492E512C612C712CCB
:10AC2000CA01B901A30192010E9413EC605D609317
:10AC30001C08C501B401A30192010E9413EC4B0151
:10AC40005C01672B682B692B79F08EE280931D08DD
:10AC5000CA01B901A30192010E9413EC605D6093E7
:10AC60001E0880E3880D15C0CA01B901A301920135
:10AC70000E9413EC662339F08EE280931D08605D1C
:10AC800060931E0805C080E280931E0880931D0813
:10AC900080E280931F086AE178E08DEC94E00E94E6
:10ACA0009CEF80913011883298F4809132118D316F
:10ACB00078F02BE040E86DE180E00E9478C380915D
:10ACC0003011873228F4809132118F3108F0F7C0AB
:10ACD00080913011823328F4809132118B3208F048
:10ACE00053C180913011803428F48091321188331F
:10ACF00008F064C18091D907882339F098D740E0E3
:10AD000050E0BA0182E298E526D7209123023091E3
:10AD100024024091FF075091000860910108709152
:10AD20000208C901840F951F2436310524F48536A5
:10AD300091053CF416C02436310531F08436910576
:10AD400084F484E690E00DC04B3051056105710537
:10AD500014F00A9706C0463F5F4F6F4F7F4F6CF469
:10AD60000A9690932402809323021092FF07109278
:10AD7000000810920108109202088091230290911D
:10AD800024028A3091053CF0883E43E094072CF081
:10AD900087EE93E002C08AE090E0909324028093D3
:10ADA000230262960FB6F894DEBF0FBECDBFDF91CF
:10ADB000CF911F910F91FF90EF90DF90CF90BF90B8
:10ADC000AF909F908F907F906F905F904F9008957D
:10ADD0002CE09FCC22E19DCC02E022E041E16DE03D
:10ADE0008CEF90E165DADBCC2CE045CD22E143CD60
:10ADF00002E022E042E168E58CEF90E159DA81CD92
:10AE000007E028E04AE26AE28CEF90E151DA05E0DF
:10AE100022E04CE262E38CEF90E14ADA24E04AE07F
:10AE200061E38AE20E9478C36091FE107091FF1086
:10AE300082E3809318118BE28093191128E131E1AC
:10AE400042E38CEF90E11CD994CD24E04AE461E325
:10AE500086E30E9478C396CD20E0CACD44E6A416CE
:10AE6000B104C0F48F929F92C50168E170E00E9426
:10AE700013EF9F938F9385E199E09F938F931F9397
:10AE80000F930E94C5E70FB6F894DEBF0FBECDBF8B
:10AE900095E01FCE8F929F923F932F938DE099E084
:10AEA0009F938F931F930F930E94C5E70FB6F8945B
:10AEB000DEBF0FBECDBF96E00CCE98E00ACE83E099
:10AEC0008093331186E280933411FF2021F081E3D7
:10AED00099E071D70DC08091A004811102C08FE369
:10AEE00005C08091ED048111F2CF80E20E943074A0
:10AEF0008BE08093331116E21093341189ED94E0C6
:10AF000067D78BE28093331110933411FF2021F027
:10AF10008FE299E050D70DC08091A104811102C049
:10AF20008FE305C08091EE048111F2CF80E20E9490
:10AF3000307483E38093331116E21093341184ED5F
:10AF400094E046D783E58093331110933411FF20AA
:10AF500021F08DE299E02FD70DC08091A2048111DC
:10AF600002C08FE305C08091EF048111F2CF80E22F
:10AF70000E9430748BE58093331186E28093341104
:10AF80008DEC94E025D7A4CE84E037D683E080937F
:10AF9000331112E31093341186E0F9D60E949BD846
:10AFA0008CE0809333111093341183E292E00E947D
:10AFB00001D80ED785E20E94307493CE10923311DF
:10AFC0008FE38093341187E692E002D793CE80918D
:10AFD00097048630D8F496E0899FF0011124EC554F
:10AFE000FB4F209132023091330231832083409114
:10AFF000FF07509100086091010870910208428398
:10B000005383648375838F5F80939704089540E032
:10B0100050E0BA018BEB92E59EC5E0919704EE23D8
:10B0200081F0E150E093970486E0E89FF00111245D
:10B03000EC55FB4F42815381648175818081918100
:10B040008AC5E5CF0F931F93CF93DF931092D70755
:10B050008091FF0790910008A0910108B09102082B
:10B0600081309048A105B10540F01092FF07109281
:10B0700000081092010810920208C091FF07809109
:10B08000DE041816DCF4282F082E000C330B215098
:10B0900031094C2F0C2E000C550B4217530774F03E
:10B0A000CFEFC80F8C2F90E0A0E0B0E08093FF07B7
:10B0B00090930008A0930108B09302081092C9076A
:10B0C0008091C807C81714F4C093C8078091C807B7
:10B0D000082E000C990B04962C2F0C2E000C330B11
:10B0E0008217930724F48CEF8C0F8093C80710917C
:10B0F000C807D0E001E0112341F080915A119091EE
:10B100005B11891B8F70B9F519C0809134028823B7
:10B1100049F081E0C11180E024E040ED5BE06D2F5B
:10B120000E945CD88091D907882339F3C111E5CFFB
:10B1300074DF8091C907882301F30FC180918A11C0
:10B14000811119C01130D1F480913402882351F05B
:10B1500081E0C13009F080E023E043EC5BE06D2F3B
:10B160000E945CD88091D907882331F1C13021F544
:10B170008DEA9DE61BC0113009F4D6C01230E1F40F
:10B1800080913402882351F081E0C23009F080E0E0
:10B1900023E04BEB5BE06D2F0E945CD88091D907D8
:10B1A000882351F0C23041F482EC90EB0E94AA6BEC
:10B1B0008091C9078111D1C080918B11882309F436
:10B1C0008BC080915813882309F476C080918A112E
:10B1D0008823E9F01330D9F580913402882351F0A7
:10B1E00081E0C33009F080E020E24FEA5BE06D2FA0
:10B1F0000E945CD88091D907882309F48CC0C330A1
:10B2000009F089C010928A110E947B7950C01330D6
:10B21000F1F480913402882351F081E0C33009F0C9
:10B2200080E020E242EA5BE06D2F0E945CD88091D2
:10B23000D907882309F46FC0C33009F06CC080912E
:10B240008B11811100938A110E943B7930C0143018
:10B2500009F061C080913402882351F081E0C4304C
:10B2600009F080E020E247E95BE06D2F0E945CD8A6
:10B270008091D907882309F44EC0C43009F04BC02F
:10B280000E9425748091A3048093AE061092AF06AD
:10B290000E94FBC70E9410C5109214081092130858
:10B2A0001092040260E080E79BE00E94F7D8809152
:10B2B000C907882381F151C0133011F084E02CC0FC
:10B2C000809134028823C1F081E0C33009F080E02E
:10B2D00023E049E85BE00DC0133081F78091340230
:10B2E000882351F081E0C33009F080E023E04EE78D
:10B2F0005BE06D2F0E945CD88091D9078823F1F222
:10B30000C330E1F684ED96E60E94AA6B8091C907EE
:10B310008823A1F222C085E0DF5F1F5FD53009F0EE
:10B32000EACE8093DE0419C080913402882351F064
:10B3300081E0C13009F080E023E04BEC5BE06D2F51
:10B340000E945CD88091D907882309F435CFC13099
:10B3500009F032CF89EF90E729CFDF91CF911F918C
:10B360000F91089590E0FC013197E231F10508F06A
:10B370004EC08827EE58FF4F8F4F0C943AEF8091C4
:10B3800080008F7703C0809180008F7D8093800044
:10B39000089580918000877FF9CF84B58F7702C0B0
:10B3A00084B58F7D84BD08958091B0008F7703C0F0
:10B3B0008091B0008F7D8093B000089580919000BF
:10B3C0008F7707C0809190008F7D03C0809190009F
:10B3D000877F8093900008958091A0008F7707C0A9
:10B3E0008091A0008F7D03C08091A000877F809313
:10B3F000A0000895809120018F7707C080912001DF
:10B400008F7D03C080912001877F80932001089564
:10B410003FB7F8948091E3049091E404A091E5048F
:10B42000B091E60426B5A89B05C02F3F19F0019600
:10B43000A11DB11D3FBFBA2FA92F982F8827820FBA
:10B44000911DA11DB11DBC01CD0142E0660F771F0A
:10B45000881F991F4A95D1F708951F93CF93DF93C3
:10B46000282F30E0F901EE5BF24F8491F901E450AE
:10B47000F34FD491F901EA54F34FC491CC23C1F0B6
:10B48000162F81116FDFEC2FF0E0EE0FFF1FEE574C
:10B49000F34FA591B4918FB7F894111105C09C9109
:10B4A000ED2FE095E92302C0EC91ED2BEC938FBFDB
:10B4B000DF91CF911F910895CF93DF9390E0FC012E
:10B4C000E450F34F2491FC01EA54F34F8491882314
:10B4D00061F190E0880F991FFC01E859F34FC59185
:10B4E000D491FC01EE57F34FA591B491611109C0BD
:10B4F0009FB7F8948881209582238883EC912E232E
:10B500000BC0623061F49FB7F8943881822F809528
:10B5100083238883EC912E2B2C939FBF06C08FB77B
:10B52000F894E8812E2B28838FBFDF91CF91089567
:10B530001F93CF93DF93182FEB0161E0BDDF2097BE
:10B5400011F460E004C0CF3FD10531F461E0812FF8
:10B55000DF91CF911F9181CFE12FF0E0EE5BF24FB1
:10B56000E4914E2F50E0FA013197E231F10508F0F5
:10B570009DC08827EC57FF4F8F4F0C943AEF84B54E
:10B58000806884BDC7BD97C084B5806284BDC8BDD6
:10B5900092C080918000806880938000D093890061
:10B5A000C093880088C08091800080628093800072
:10B5B000D0938B00C0938A007EC080918000886009
:10B5C00080938000D0938D00C0938C0074C08091D4
:10B5D000B00080688093B000C093B3006CC08091CD
:10B5E000B00080628093B000C093B40064C08091CA
:10B5F0009000806880939000D0939900C093980049
:10B600005AC080919000806280939000D0939B00FC
:10B61000C0939A0050C08091900088608093900001
:10B62000D0939D00C0939C0046C08091A00080688C
:10B630008093A0008091A0008F7B8093A000D09386
:10B64000A900C093A80037C08091A00080628093B9
:10B65000A000D093AB00C093AA002DC08091A000A1
:10B6600088608093A000D093AD00C093AC0023C04D
:10B6700080912001806880932001D0932901C0939C
:10B68000280119C080912001806280932001D0930D
:10B690002B01C0932A010FC0809120018860809304
:10B6A0002001D0932D01C0932C0105C0C038D105D5
:10B6B0000CF04CCF46CFDF91CF911F9108958F9220
:10B6C0009F92AF92BF92CF92DF92EF92FF926B0167
:10B6D0007C019EDE4B015C01C114D104E104F10444
:10B6E000E9F096DEDC01CB0188199909AA09BB09AA
:10B6F000883E9340A105B10578F321E0C21AD10834
:10B70000E108F10888EE880E83E0981EA11CB11CA8
:10B71000C114D104E104F10421F7DECFFF90EF90D2
:10B72000DF90CF90BF90AF909F908F9008952FB7EC
:10B73000F8946091DF047091E0048091E1049091AD
:10B74000E2042FBF089511982FB787FD71C0F894B8
:10B75000909102019E7F909302012FBF119A0000E9
:10B760001198282F220F9FB786FD81C0F8948091F1
:10B7700002018E7F809302019FBF119A00001198F1
:10B78000922F990F26FD6DC02FB7F894809102017A
:10B790008E7F809302012FBF119A00001198892F8C
:10B7A000880F2FB796FD58C0F894909102019E7FA4
:10B7B000909302012FBF119A00001198982F990FB2
:10B7C0002FB786FD44C0F894809102018E7F80934C
:10B7D00002012FBF119A00001198892F880F2FB7EF
:10B7E00096FD30C0F894909102019E7F90930201E3
:10B7F0002FBF119A00001198982F990F2FB786FD2F
:10B800001CC0F894809102018E7F809302012FBFAB
:10B81000119A0000119896FD2FC09FB7F89480915F
:10B8200002018E7F809302019FBF119A000008954C
:10B83000F8949091020191608ECFF894809102016A
:10B840008160E3CFF894909102019160CFCFF8949A
:10B85000809102018160BBCFF894909102019160C8
:10B86000A7CF2FB7F89480910201816092CFF8940E
:10B870008091020181607ECF9FB7F8948091020190
:10B880008160D0CFFC011382128284E493E0918323
:10B89000808313AE14AE15AE9F012C5F3F4F11860F
:10B8A000108613861286158681E0848782E2868759
:10B8B000138A128ADF019796CF01C5964FEF4D93F9
:10B8C000A817B907E1F791E094A346EA54E4528F30
:10B8D000418F938F148E158E80E4868F178E86E4A9
:10B8E00094E496AB85AB77836683C9010C94C25010
:10B8F0006F927F928F929F92AF92BF92CF92DF9280
:10B90000EF92FF920F931F93CF93DF935C017B0124
:10B91000742E69018AE0481709F474C0A5E14A133E
:10B920004FC0DB011296ED91FC9113979280C68176
:10B93000D7819FB7F89480910201826080930201C1
:10B940009FBF0E94275180EE882E890C90E1692EBE
:10B95000690C88EFF8DE0E942751BFE1B91508F4A1
:10B9600043C0892D80778068EEDE892D8295807FA7
:10B97000EADE0E94275180E8E6DE80E0E4DE0E94F5
:10B9800027518AEFE0DE0E9427518E01005F1F4F92
:10B990008881807FD8DE89918295807FD4DEC01730
:10B9A000D107B1F70E942751939483949610D1CF79
:10B9B0009FB7F894809102018D7F809302019FBF11
:10B9C0009601472DB701C501DF91CF911F910F91CE
:10B9D000FF90EF90DF90CF90BF90AF909F908F90AF
:10B9E0007F906F900C94764F882D80778068ABDEC7
:10B9F000882D8295807FA7DE0E94275180E8A3DEF4
:10BA000080E8BCCF809101018260809301019FB7E3
:10BA1000F894809102018D7F809302019FBF8091F5
:10BA200001018160809301019FB7F8948091020128
:10BA30008E7F809302019FBF099A119A9FB7F89455
:10BA4000809102018260809302019FBF0E94275172
:10BA500088E790E00E942C5188EF75DE0E94275104
:10BA600080E071DE80E86FDE0E94275180E06BDEAF
:10BA700080E169DE0E9427518FE090E00E942C5106
:10BA800080E361DE80EE5FDE0E942751D0E08D2FE3
:10BA90008077806858DE8D2F8295807F54DE0E94EB
:10BAA000275180E850DE80E04EDE0E9427518AEF69
:10BAB0004ADE0E942751C0E280E045DE80E043DE9E
:10BAC0000E942751C150C1F788EF3DDE0E942751E7
:10BAD000DF5FD032E1F680E036DE80EC34DE0E94BB
:10BAE000275166CFCF92DF92EF92FF920F931F9371
:10BAF000CF93DF931F92CDB7DEB76C01DC01DC96EC
:10BB00001C91DC97DB960C917C01B4E0EB0EF11CF0
:10BB1000DC015996ED91FC915A97C70169831995FB
:10BB2000482F410F2981602FC7010E947351F601F0
:10BB300023AD082E000C990B820F911D83AF81E07D
:10BB400090E00F90DF91CF911F910F91FF90EF90B8
:10BB5000DF90CF9008952091320230913302281760
:10BB60003907D9F090933302809332024093FF0754
:10BB70005093000860930108709302088B5B924514
:10BB800021F41092D2071092970482E0809334023D
:10BB900081E08093C9071092D80708959CE0899F9F
:10BBA000802D112491E0980F909317082CE0280F16
:10BBB000209318084091301150E030E02E5F3F4F45
:10BBC00024173507CCF0292F30E04091321150E096
:10BBD000241735078CF4662341F08E5F0E945FC303
:10BBE000809118088E5F0E945FC3809118081092A0
:10BBF00033118093341108950895CF93C82F823064
:10BC000059F02CF4813089F4CF910C949BD8833077
:10BC100031F0843021F009C08CED9BE002C083E458
:10BC200096E40E94D8C2C0938314CF910895EF92F6
:10BC3000FF920F931F93CF93DF931F92CDB7DEB781
:10BC400080913511811107C081E0809335118CEF0F
:10BC500090E10E94C2506091FE107091FF10198215
:10BC60009E012F5F3F4F4FE08CEF90E10E944050CC
:10BC700080911E02882371F10E943B7406ED10E151
:10BC800020E440E160E080E00E944DC284E0B5DF46
:10BC90006091FD106E5147EB53E080E00E94A3C21B
:10BCA0006091FD1062514CEB53E080E00E94A3C212
:10BCB0006091FD10665043EC53E080E00E94A3C207
:10BCC0000E9425C38111DACF68EB7BE080E090E031
:10BCD0000E943AD8F090FC1080911E0281110AC097
:10BCE00010921E020F90DF91CF911F910F91FF9044
:10BCF000EF9008950E943B742F2D30E0C901C89742
:10BD000097FD019695958795E82E2E513109369528
:10BD10002795F22E01E510E123E147E06CE08E2D3E
:10BD20000E944DC284E069DF0091FC1010E00257D0
:10BD30001109169507956091FD10625141ED53E090
:10BD40008F2D0E94A3C26091FD10665047ED53E015
:10BD5000802F0E94A3C20E9425C38111DBCFC0CFD8
:10BD6000CF93C82F8FEF8C0F893058F48CED9BE068
:10BD70000E94D8C28C2F0E943074809183143DDFC2
:10BD800003C08C2F0E94307481E0CF910895CF932F
:10BD90009FEF980F993060F4C82F8CED9BE00E94C4
:10BDA000D8C28C2F0E94307480918314CF9125CFFC
:10BDB000CF910C943074CF93DF93EC01FE0184910A
:10BDC000882319F0E4DF2196F9CFDF91CF91089510
:10BDD0000F931F93CF938C01C0E0F801EC0FF11D7E
:10BDE0008081882319F0D3DFCF5FF7CFCF911F91E8
:10BDF0000F9108959F92AF92BF92CF92DF92EF92F0
:10BE0000FF920F931F93CF93DF931F92CDB7DEB7AF
:10BE10005C017B0120E030E0F501E20FF31FE491CB
:10BE2000EE2319F02F5F3F4FF7CFF7016F01CE18C8
:10BE3000DF0881918111FACFDD24332784E190E07E
:10BE40008C199D098217930714F001E001C002E0EC
:10BE500010E08091FD1090E0B8016F5F7F4F0E946D
:10BE600027EF86E0982E960E80913011981648F0B4
:10BE70002091321130E0892D90E00B972817390777
:10BE800094F5E114F104C1F101501109609F900C87
:10BE9000112480913011981678F12091321130E000
:10BEA000892D90E00B972817390734F18AE30E9417
:10BEB000307425E130E02C193D09822F880F280FBE
:10BEC000220F2093331190923411C7010F90DF910C
:10BED000CF911F910F91FF90EF90DF90CF90BF9087
:10BEE000AF909F9075CF1092331190923411C5018D
:10BEF000698361DF6981C5CF0F90DF91CF911F9179
:10BF00000F91FF90EF90DF90CF90BF90AF909F90F8
:10BF10000895CF93DF93EC0168E172E0B3DC8CE429
:10BF200093E099838883DF91CF9108952F923F9278
:10BF30004F925F926F927F928F929F92AF92BF9239
:10BF4000CF92DF92EF92FF920F931F93CF93DF93E5
:10BF5000EC0145EF5EE081E090E0FA01259134913B
:10BF6000C217D3070CF05DC09C0121503109220F8C
:10BF7000331F220F331FD901AD50B14FFD01659121
:10BF800074912F50314FF901A590B490FC01EE0F40
:10BF9000FF1FEE0FFF1FED50F14FE590F490FD01F4
:10BFA000C590D490FA0105911491F901259034902F
:10BFB000072E000C880B990B0E9432E82B013C01E4
:10BFC000CA19DB09BE01DD0F880B990B0E9432E80C
:10BFD0004B015C01B7016C197D09072E000C880B21
:10BFE000990B0E9432E89B01AC01C501B4010E948B
:10BFF00091E86B017C01B80162197309072E000CEE
:10C00000880B990B0E9432E89B01AC01C701B60175
:10C010000E942BED9B01AC01C301B2010E944FECC9
:10C0200011C001964C5F5F4F8034910509F095CFA8
:10C03000EFEEFFE065917491072E000C880B990BD1
:10C040000E9432E8DF91CF911F910F91FF90EF9006
:10C05000DF90CF90BF90AF909F908F907F906F9028
:10C060005F904F903F902F90089560919804709149
:10C07000990480919A0490919B040E9493EDCB01C6
:10C0800008951F920F920FB60F9211240BB60F92C4
:10C090002F933F934F935F936F937F938F939F93D0
:10C0A000AF93BF93CF93DF93EF93FF938091B70646
:10C0B000811156C181E08093B70680916E008B7F1D
:10C0C00080936E007894809117028F37B0F08F576D
:10C0D0009091B6069093C707992311F02C9A01C04E
:10C0E0002C989091B5069093C6072FB7992379F0B5
:10C0F000F8949091020190620EC09091C707891741
:10C1000008F02C989091C607891740F02FB7F89443
:10C11000909102019F7D909302012FBF8F5F8093CA
:10C1200017029091C50781E089278093C507811187
:10C130000E94A3D880911502909116028230910539
:10C14000A1F1A4F4009761F1019709F048C0809132
:10C150007800909179002091BA073091BB07820F47
:10C16000931F9093BB078093BA0739C08330910522
:10C1700041F10497A1F58091C407811103C086E0C5
:10C180008093C4078091C40781508093C40788239B
:10C1900031F183E090E090931602809315021FC066
:10C1A00088E080937B0085E404C088E080937B0076
:10C1B00086E480937C0080917A00806480937A008A
:10C1C0000EC080917800909179002091B80730914D
:10C1D000B907820F931F9093B9078093B807809196
:10C1E000150290911602892B09F060C0809114020B
:10C1F0008F5F80311CF48093140258C01092140297
:10C200008091B406811113C08091BA079091BB0749
:10C210009093B3068093B2068091B8079091B907C6
:10C220009093B1068093B00681E08093B4068AE0D3
:10C23000EAEBF7E0DF011D928A95E9F71092B90762
:10C240001092B807C091B206D091B306D195C195AE
:10C25000D1098091E9049091EA0491958195910921
:10C260008C179D07CCF1809107029091080291955F
:10C2700081959109C817D9070CF43FC02091B006E9
:10C280003091B1068091E7049091E80482179307FA
:10C290000CF044C020910502309106028091B00656
:10C2A0009091B106821793070CF049C08091150256
:10C2B00090911602019665E070E00E9427EF90933E
:10C2C000160280931502F8941092B70680916E00C2
:10C2D000846080936E0044C0809111089091120890
:10C2E000181619060CF0BFCF42E350E16FE370E17E
:10C2F00080E090E00E94EFD1B6CF8091110890913C
:10C300001208181619060CF0B9CF42E050E16FE0A0
:10C3100070E180E090E00E94EFD1B0CF80911508ED
:10C3200090911608181619060CF0B4CF41E250E1AE
:10C330006FE370E18FEF9FEF0E94EFD1ABCF809161
:10C34000150890911608181619060CF0AFCF41EF9A
:10C350005FE06FE070E18FEF9FEF0E94EFD1A6CF1B
:10C36000FF91EF91DF91CF91BF91AF919F918F910D
:10C370007F916F915F914F913F912F910F900BBEE5
:10C380000F900FBE0F901F9018950F931F93CF9390
:10C39000DF9300D01F92CDB7DEB78091FF07909159
:10C3A0000008A0910108B0910208B7FF08C01092E0
:10C3B000FF07109200081092010810920208809165
:10C3C000030890910408A0910508B09106084091D7
:10C3D000FF075091000860910108709102088417CE
:10C3E0009507A607B70744F48093FF0790930008CA
:10C3F000A0930108B093020880913402882371F160
:10C400004091FF0750910008609101087091020867
:10C410008091070890910808A0910908B0910A0836
:10C420008A019B01080F191F2A1F3B1FC901B80170
:10C430000E9430E820E030E048EC52E40E9491E8AD
:10C4400069837A838B839C83CE0101960E942DD6CB
:10C45000BC0180910D0890910E08CCDC8091D90729
:10C46000882399F14091FF075091000860910108DD
:10C47000709102088091070890910808A09109081E
:10C48000B0910A088A019B01080F191F2A1F3B1F40
:10C49000C901B8010E9430E820E030E048EC52E4E5
:10C4A0000E9491E80E9498EDE0910B08F0910C0831
:10C4B000309721F060837183828393830E940D58AB
:10C4C000E0910F08F091100819950F900F900F90C0
:10C4D0000F90DF91CF911F910F9108950F931F93AC
:10C4E000CF93DF9300D01F92CDB7DEB78091FF07C7
:10C4F00090910008A0910108B0910208B7FF08C010
:10C500001092FF0710920008109201081092020882
:10C510008091030890910408A0910508B091060845
:10C520004091FF0750910008609101087091020846
:10C5300084179507A607B70744F48093FF079093E5
:10C540000008A0930108B093020880913402882368
:10C5500071F14091FF0750910008609101087091BE
:10C5600002088091070890910808A0910908B091ED
:10C570000A088A019B01080F191F2A1F3B1FC901C6
:10C58000B8010E9432E820E030E048EC52E40E941A
:10C5900091E869837A838B839C83CE0101960E9404
:10C5A0002DD6BC0180910D0890910E0823DC80915E
:10C5B000D907882361F14091FF07509100086091ED
:10C5C0000108709102088091070890910808A091D5
:10C5D0000908B0910A088A019B01080F191F2A1F38
:10C5E0003B1FC901B8010E9432E820E030E048EC6E
:10C5F00052E40E9491E8E0910B08F0910C0830970A
:10C6000021F060837183828393830E940D580F9081
:10C610000F900F900F90DF91CF911F910F91089580
:10C620000F931F93CF93DF9300D01F92CDB7DEB748
:10C630008091FF0790910008A0910108B091020835
:10C64000B7FF08C01092FF0710920008109201086F
:10C65000109202088091030890910408A0910508A7
:10C66000B09106084091FF075091000860910108C1
:10C670007091020884179507A607B70744F48093C2
:10C68000FF0790930008A0930108B09302088091DF
:10C690003402882371F14091FF07509100086091A6
:10C6A0000108709102088091070890910808A091F4
:10C6B0000908B0910A088A019B01080F191F2A1F57
:10C6C0003B1FC901B8010E9432E82AE037ED43E27E
:10C6D0005CE30E9491E869837A838B839C83CE011B
:10C6E00001960E94F7D4BC0180910D0890910E082C
:10C6F00081DB8091D907882389F14091FF07509110
:10C7000000086091010870910208809107089091DB
:10C710000808A0910908B0910A088A019B01080F36
:10C72000191F2A1F3B1FC901B8010E9432E82AE0E5
:10C7300037ED43E25CE30E9491E8E0910B08F09151
:10C740000C08309721F060837183828393830E9469
:10C750000D58E0910F08F091100819950F900F9067
:10C760000F900F90DF91CF911F910F910895CF926D
:10C77000DF92EF92FF920F931F93CF93DF9300D03E
:10C780001F92CDB7DEB78091FF0790910008A0916E
:10C790000108B0910208B7FF08C01092FF0710927D
:10C7A00000081092010810920208809103089091ED
:10C7B0000408A0910508B09106084091FF07509128
:10C7C0000008609101087091020884179507A60778
:10C7D000B70744F48093FF0790930008A0930108E3
:10C7E000B093020880913402882371F14091FF07D1
:10C7F000509100086091010870910208809107082B
:10C8000090910808A0910908B0910A086A017B017B
:10C81000C80ED91EEA1EFB1EC701B6010E9432E8EF
:10C820002AE037ED43E25CE30E9491E869837A8372
:10C830008B839C83CE0101960E94ACD5BC01809174
:10C840000D0890910E08D6DA1091D907112361F1E5
:10C850008091FF0790910008A0910108B091020813
:10C8600040910708509108086091090870910A08E2
:10C870006C017D01C40ED51EE61EF71EC701B60170
:10C880000E9432E82AE037ED43E25CE30E9491E83F
:10C89000E0910B08F0910C08309721F060837183D0
:10C8A000828393830E940D58812F0F900F900F90D9
:10C8B0000F90DF91CF911F910F91FF90EF90DF903C
:10C8C000CF90089554DF882329F0E0910F08F0916C
:10C8D0001008199408954BCF0F931F93CF93DF93B4
:10C8E00000D01F92CDB7DEB78091FF07909100086E
:10C8F000A0910108B0910208B7FF08C01092FF078D
:10C90000109200081092010810920208809103080A
:10C9100090910408A0910508B09106084091FF0786
:10C9200050910008609101087091020884179507E2
:10C93000A607B70744F48093FF0790930008A093DD
:10C940000108B093020880913402882371F140916C
:10C95000FF075091000860910108709102088091D2
:10C96000070890910808A0910908B0910A088A0167
:10C970009B01080F191F2A1F3B1FC901B8010E9404
:10C9800032E82FE632E143E85AE30E9491E86983F6
:10C990007A838B839C83CE0101960E94A179BC018E
:10C9A00080910D0890910E0825DA8091D90788238F
:10C9B00089F14091FF075091000860910108709142
:10C9C00002088091070890910808A0910908B09189
:10C9D0000A088A019B01080F191F2A1F3B1FC90162
:10C9E000B8010E9432E82FE632E143E85AE30E94A0
:10C9F00091E8E0910B08F0910C08309721F06083EA
:10CA00007183828393830E940D58E0910F08F09107
:10CA1000100819950F900F900F900F90DF91CF9104
:10CA20001F910F910895CF92DF92EF92FF920F9393
:10CA30001F93CF93DF9300D01F92CDB7DEB78091C5
:10CA4000FF0790910008A0910108B0910208B7FF7C
:10CA500008C01092FF07109200081092010810926F
:10CA600002088091030890910408A0910508B091F4
:10CA700006084091FF0750910008609101087091ED
:10CA8000020884179507A607B70744F48093FF07A9
:10CA900090930008A0930108B0930208809134029B
:10CAA000882371F14091FF075091000860910108BF
:10CAB000709102088091070890910808A0910908D8
:10CAC000B0910A086A017B01C80ED91EEA1EFB1E3E
:10CAD000C701B6010E9432E82AE037ED43E25CE389
:10CAE0000E9491E869837A838B839C83CE010196AF
:10CAF0000E9417D7BC0180910D0890910E087AD939
:10CB00001091D907112361F18091FF0790910008DE
:10CB1000A0910108B09102084091070850910808BF
:10CB20006091090870910A086C017D01C40ED51E40
:10CB3000E61EF71EC701B6010E9432E82AE037ED73
:10CB400043E25CE30E9491E8E0910B08F0910C084D
:10CB5000309721F060837183828393830E940D5804
:10CB6000812F0F900F900F900F90DF91CF911F9119
:10CB70000F91FF90EF90DF90CF90089554DF8823BE
:10CB800029F0E0910F08F0911008199408954BCF07
:10CB90000F931F93CF93DF931F921F92CDB7DEB7F2
:10CBA0008091FF0790910008A0910108B0910208C0
:10CBB000B7FF08C01092FF071092000810920108FA
:10CBC000109202088091030890910408A091050832
:10CBD000B09106084091FF0750910008609101084C
:10CBE0007091020884179507A607B70744F480934D
:10CBF000FF0790930008A0930108B093020880916A
:10CC00003402882341F14091FF0750910008609160
:10CC10000108709102088091070890910808A0917E
:10CC20000908B0910A088A019B01080F191F2A1FE1
:10CC30003B1FC901B8010E9432E80E9493ED7A833C
:10CC40006983CE0101960E9401D8BC0180910D0834
:10CC500090910E08CFD88091D907882331F1409167
:10CC6000FF075091000860910108709102088091BF
:10CC7000070890910808A0910908B0910A088A0154
:10CC80009B01080F191F2A1F3B1FC901B8010E94F1
:10CC900032E8E0910B08F0910C08309721F06083A6
:10CCA0007183828393830E940D580F900F90DF91C0
:10CCB000CF911F910F910895CF93DF9300D0CDB7FF
:10CCC000DEB78091FF0790910008A0910108B09114
:10CCD0000208B7FF08C01092FF07109200081092D8
:10CCE0000108109202088091030890910408A09115
:10CCF0000508B09106084091FF0750910008609127
:10CD000001087091020884179507A607B70744F435
:10CD10008093FF0790930008A0930108B093020846
:10CD2000809134028823B1F02091070830910808DF
:10CD30008091FF0790910008820F931F9A83898347
:10CD4000CE0101960E9401D8BC0180910D089091FE
:10CD50000E0850D88091D9078823B1F04091070878
:10CD6000509108082091FF0730910008240F351FCB
:10CD7000E0910B08F0910C08309711F0318320837B
:10CD80008B830E940D588B810F900F900F90DF9135
:10CD9000CF91089591CF90DF882329F0E0910F087B
:10CDA000F091100819940895AF92BF92CF92DF923C
:10CDB000EF92FF920F931F93CF93DF93CDB7DEB720
:10CDC0006F970FB6F894DEBF0FBECDBF80913402CF
:10CDD000811105C08091D907882309F4CDC188ED60
:10CDE00091E19093D7118093D61181E090E09093D8
:10CDF000101480930F14109212141092111440E02A
:10CE000050E0BA018CED91E10E94F08E8091D61134
:10CE10009091D7112BE1FC013496DE01159601901B
:10CE20000D922A95E1F7FC01828193819C838B838B
:10CE300080E893E09A83898340E050E0BE016F5F11
:10CE40007F4F8AE094E00E9410C6CE0101960E94B6
:10CE50006F4FA0901114B09012141092D7078091C8
:10CE6000FF0790910008A0910108B091020881305D
:10CE70009048A105B10540F01092FF0710920008FC
:10CE800010920108109202081091FF078091DB07B1
:10CE90001816DCF4282F082E000C330B2150310912
:10CEA000412F012E000C550B4217530774F01FEF52
:10CEB000180F812F90E0A0E0B0E08093FF079093DF
:10CEC0000008A0930108B09302081092C90780914E
:10CED000C807181714F41093C8078091C807082EC4
:10CEE000000C990B0496212F012E000C330B821796
:10CEF000930724F48CEF810F8093C8070091C80733
:10CF0000F12C21E0A21AB108002359F06DE871E17B
:10CF10008CED91E10E94FC9080918D118F32D9F4BB
:10CF20001EC080913402882349F081E0111180E015
:10CF300024E040EF50E36F2D0E945CD88091D90728
:10CF4000882321F31111E2CF0E940D588091C90767
:10CF50008823E1F211C1013041F092E001C091E07B
:10CF60006501EE24E394E00E63C0809134028823CF
:10CF700051F081E0113009F080E020E24CEE50E306
:10CF80006F2D0E945CD88091D907882331F311302E
:10CF900021F780912D138823D1F0815080932D1398
:10CFA000EFE18E9FC0011124FC01E550FE4E2BE104
:10CFB000ACEDB1E101900D922A95E1F7FC01E95049
:10CFC000FE4E828193819093DB118093DA1110924F
:10CFD000C8070FC08AE00E941C87CE0101960E94FC
:10CFE0006F4F1092FF0710920008109201081092E4
:10CFF000020881E08093C90783E080933402BCC0BB
:10D000000913B1C060E070E0C6010E94D073909136
:10D010008C1180913402992309F489C081110DC0CB
:10D020008091D907811111C09E2DF1E0CF1AD1084E
:10D030002FEFC216D20621F798C081E0101380E0CE
:10D0400041E06F2D0E94167AEBCF1013EDCF1D82B9
:10D0500018861C821B8280E893E09A8389838091E2
:10D06000DF11882319F008ED11E102C007EB11E18F
:10D070007801F4E0EF0EF11C21E04DE851E1B70139
:10D08000CE0105960E94D293811124C0E8E3F4E416
:10D0900084918F010F5F1F4F882321F00E941C870E
:10D0A000F801F6CFE6EDF0E384918F010F5F1F4F9B
:10D0B000811103C00DE811E104C00E941C87F80132
:10D0C000F3CFF80181918F01882309F483CF0E9467
:10D0D0001C87F7CF80912D138A30C8F491E0980F08
:10D0E00090932D13FFE18F9FC0011124DC01A55007
:10D0F000BE4E2BE1F70101900D922A95E1F7F80160
:10D1000022813381FC01E950FE4E338322838BE17F
:10D11000FE013596ACEDB1E101900D928A95E1F7F3
:10D120008B819C819093DB118093DA1156CF8823F9
:10D1300039F081E0101380E040E06F2D0E94167AF4
:10D140008091D907882309F46FCF10136DCF8DE834
:10D1500091E10E948D760E9407588091C90788232B
:10D1600009F462CF09C09F5F60CFF3940F5F85E041
:10D17000F812CACE9093DB076F960FB6F894DEBF15
:10D180000FBECDBFDF91CF911F910F91FF90EF9018
:10D19000DF90CF90BF90AF9008954F925F926F92C3
:10D1A0007F928F929F92AF92BF92CF92DF92EF9237
:10D1B000FF920F931F93CF93DF9300D01F92CDB7B1
:10D1C000DEB710911F021F3FF9F00E94975BC090DD
:10D1D000CA07D090CB07E090CC07F090CD07DC01D8
:10D1E000CB018C199D09AE09BF09B7FD0DC0209177
:10D1F0005B1180915A1130E090E001968F70992771
:10D200002817390709F018C20E94A3D880917E140C
:10D2100082FF40C08091E70781113EC081E080938A
:10D22000E7079091DA0789278093D9071092DA07E8
:10D2300083E08093340210927E140E94975BDC019D
:10D24000CB018C509E4FAF4FBF4F80937F14909374
:10D250008014A0938114B093821480ED97E09C8396
:10D260008B8382E390E09A838983BE016D5F7F4F59
:10D27000CE0101960E94EC7816E0115069F08CE521
:10D2800091E10E94CE4462E070E080E090E00E9474
:10D290005F5BF3CF1092E7071091090110951170B1
:10D2A0008091E6071817A9F0112309F4E6C10E943E
:10D2B000A2778091E607823029F060E082E091E376
:10D2C0000E94F7D81093E60783E0809334020E940F
:10D2D000175E0E94975B6B017C018091E207909141
:10D2E000E307A091E407B091E507A7019601281B89
:10D2F000390B4A0B5B0B57FF05C08091D807882379
:10D3000009F4F6C1D701C6018C599F4FAF4FBF4FEB
:10D310008093E2079093E307A093E407B093E507B7
:10D3200080917D1418162CF480917D14843074F44F
:10D3300008C080917D14992781950CF490950497ED
:10D340002CF48091D90781119FC0AFC08091D7077D
:10D35000882309F472C080917D14181664F48091BA
:10D360007D14082E000C990B97FD039695958795D3
:10D37000959587950EC080917D14082E000C990B11
:10D3800097FD0396959587959595879591958195A8
:10D3900091098090D3079090D407A090D507B090C2
:10D3A000D60781149104A104B104D1F1BC01990FF5
:10D3B000880B990B0E9432E82B013C01C701B60192
:10D3C000681979098A099B090E9430E89B01AC0120
:10D3D000C301B2010E942BED20E030E04AE754E4A3
:10D3E0000E9491E84B015C0120E030E040E253E410
:10D3F0000E9475EE87FF0FC020E030E046E952E45E
:10D40000C501B4010E9475EE87FD0AC02AE030E034
:10D4100040E050E009C024E630E040E050E004C0C5
:10D4200021E030E040E050E0C092D307D092D40732
:10D43000E092D507F092D60704C021E030E040E04A
:10D4400050E0A0917D140A2E000CBB0B0E9439EC19
:10D4500024E030E040E050E00E9413EC8091FF07B0
:10D4600090910008A0910108B0910208820F931FCB
:10D47000A41FB51F8093FF0790930008A093010895
:10D48000B093020810927D14D701C6018856954CBE
:10D49000AF4FBF4F8093DE079093DF07A093E00765
:10D4A000B093E10782E08093340280913202909140
:10D4B00033028B5B924541F480912002882309F46A
:10D4C000E7C08150809320022FB7F8948091CE0757
:10D4D0009091CF07A091D007B091D1072FBF3AE02C
:10D4E000B695A795979587953A95D1F7009741E01E
:10D4F000A407B10520F08FEF9FEFA0E0B0E0969574
:10D50000879520913402211105C03091D80731113F
:10D51000EBC055C0009741F04091DC075091DD070A
:10D520004817590708F04BC08091D807811111C0E6
:10D53000223050F0243028F0243031F4109234029C
:10D5400003C081E0809334020E943B7481E08093A9
:10D55000D80784E00E94FD5D81E080931C11E0917A
:10D560003202F091330219951092D9078091D807B1
:10D57000882351F00E9425C391E0811101C090E001
:10D580009093D807911194C08090DC079090DD07AC
:10D59000A12CB12C0E94975BDC01CB018C199D0959
:10D5A000AE09BF0988169906AA06BB0640F40E9478
:10D5B000975B6C197D097093DD076093DC078091A0
:10D5C0003202909133028B5B924521F08091D20719
:10D5D000882379F088E9C80E8AE3D81EE11CF11C83
:10D5E000C092DE07D092DF07E092E007F092E107F9
:10D5F0000FC08091DE079091DF07A091E007B09106
:10D60000E107C81AD90AEA0AFB0AF7FE0E9407587E
:10D610008091D80781116CC080913402813049F02B
:10D6200008F466C0843008F063C081E0809334025F
:10D630005FC0109234025CC024E01202F001112499
:10D64000E05BFC4F20E030E040E752E46081718114
:10D65000828193810E942BEDC12C7B018C0129E0FA
:10D6600035E045E055E061E075E08DEF94E00E9423
:10D6700077988FEF80931F02C7CD10928A11109276
:10D680008B11823009F41ECE60E085EF90E318CE56
:10D690008CE0809320028091DC079091DD07019758
:10D6A0009093DD078093DC0781E0809334020CCFF8
:10D6B0008090DC079090DD07A12CB12C0E94975B35
:10D6C000DC01CB018C199D09AE09BF0988169906AA
:10D6D000AA06BB0668F40E94975B6C197D097093DB
:10D6E000DD076093DC0704C0009709F432CF14CF44
:10D6F0000F900F900F900F90DF91CF911F910F918E
:10D70000FF90EF90DF90CF90BF90AF909F908F9061
:10D710007F906F905F904F9008950E94175E3E98A3
:10D72000469A3C98449A3A98429AEAE0F1E080811D
:10D730008E7F80839FB7F894EBE0F1E08081816079
:10D7400080839FBF82E08093E6070E94A3D8109257
:10D750007D140895CF93DF931F921F92CDB7DEB74C
:10D7600089839A830E94E75740E050E0BA0189819B
:10D770009A810F900F90DF91CF910C94AB5D80E078
:10D7800090E0A0E2B1E48093F8079093F907A093AA
:10D79000FA07B093FB0740E050E0BA018091FD0723
:10D7A0009091FE070C94AB5D80E090E0A0E8BFE3B1
:10D7B0008093F8079093F907A093FA07B093FB07BB
:10D7C00040E050E0BA018091FD079091FE070C9473
:10D7D000AB5D8DEC9CECACECBDE38093F8079093D3
:10D7E000F907A093FA07B093FB0740E050E0BA01B5
:10D7F0008091FD079091FE070C94AB5DCF92DF9274
:10D80000EF92FF92CF93C82F0E94975B6B017C0130
:10D8100024EA30E74DE75FE36091F8077091F9077C
:10D820008091FA079091FB070E942CE887FD05C0C4
:10D8300046E950E060E070E003C040E050E0BA012B
:10D84000C40ED51EE61EF71EC092CA07D092CB07A3
:10D85000E092CC07F092CD07C0931F02CF91FF90CA
:10D86000EF90DF90CF9008958091D90781110C94AB
:10D870000D586091FF077091000880910108909108
:10D880000208611571058105910571F10E9432E868
:10D890002091F8073091F9074091FA075091FB0762
:10D8A0000E9491E89B01AC016091090570910A0505
:10D8B00080910B0590910C050E944FEC6093090537
:10D8C00070930A0580930B0590930C051092FF0747
:10D8D00010920008109201081092020883E090E074
:10D8E0008DDF81E08093340280913402882349F0F7
:10D8F00089E095E00E94CFD6BC018BE392E30C94C3
:10D90000FA5E08952F923F924F925F926F927F92AC
:10D910008F929F92AF92BF92CF92DF92EF92FF923F
:10D920000F931F93CF93DF9300D000D0CDB7DEB716
:10D930002091D9072223D1F026960FB6F894DEBFA6
:10D940000FBECDBFDF91CF911F910F91FF90EF9050
:10D95000DF90CF90BF90AF909F908F907F906F900F
:10D960005F904F903F902F900C940D588B011C01AD
:10D970008091FF0790910008A0910108B0910208E2
:10D98000892B8A2B8B2B09F497C00E940D49980193
:10D99000220F331F220F331F3E832D83F901E350E3
:10D9A000FB4F4080518062807380809131028111F1
:10D9B00015C020E030E04AE754E4C301B2010E9400
:10D9C0004EEC4B015C0120E030E04AE754E4C30137
:10D9D000B2010E944FEC6B017C0110C0ED81FE8111
:10D9E000E851F84F80809180A280B380ED81FE8164
:10D9F000EB5DFD4FC080D180E280F3808091FF0716
:10DA000090910008A0910108B091020889839A833F
:10DA1000AB83BC83BC01CD010E9432E82091F807A2
:10DA20003091F9074091FA075091FB070E9491E865
:10DA30009B01AC01C301B2010E944FECAD81BE81DC
:10DA4000A350BB4F3D01FD016083718382839383AB
:10DA500029813A814B815C8157FF0DC0A50194015A
:10DA60000E942CE887FF1BC0D3018D929D92AD923E
:10DA7000BC92139714C029813A814B815C81232B7E
:10DA8000242B252B61F0A70196010E9475EE181634
:10DA900034F4D301CD92DD92ED92FC921397C8013C
:10DAA000ADDE1092FF07109200081092010810924C
:10DAB000020881E08093340280913402882329F1A6
:10DAC000C801880F991F880F991F83509B4F0E9490
:10DAD000CFD6BC01C10126960FB6F894DEBF0FBEAB
:10DAE000CDBFDF91CF911F910F91FF90EF90DF900D
:10DAF000CF90BF90AF909F908F907F906F905F90EE
:10DB00004F903F902F900C94FA5E26960FB6F894A3
:10DB1000DEBF0FBECDBFDF91CF911F910F91FF9060
:10DB2000EF90DF90CF90BF90AF909F908F907F90BD
:10DB30006F905F904F903F902F90089562E070E05B
:10DB400084E392E3DFCE61E070E08DE292E3DACE2F
:10DB500060E070E086E292E3D5CEAF92BF92CF92C2
:10DB6000DF92EF92FF920F931F93CF93DF93109268
:10DB7000D7078091FF0790910008A0910108B0910C
:10DB8000020881309048A105B10540F01092FF07CE
:10DB9000109200081092010810920208C091FF072D
:10DBA0008091F7071816DCF4282F082E000C330B91
:10DBB000215031094C2F0C2E000C550B42175307E6
:10DBC00074F0CFEFC80F8C2F90E0A0E0B0E080930E
:10DBD000FF0790930008A0930108B09302081092E9
:10DBE000C9078091C807C81714F4C093C80780916B
:10DBF000C807082E000C990B04962C2F0C2E000C35
:10DC0000330B8217930724F48CEF8C0F8093C80793
:10DC1000D091C80710E083EEE82E81E3F82E9DEB4B
:10DC2000C92E91E3D92E29E0A22E22E3B22ED111E2
:10DC300017C080913402882349F081E0C11180E04F
:10DC400024E041E252E3612F0E945CD88091D90721
:10DC5000882309F47DC0C1117BC00E940D5874C097
:10DC6000D130D1F480913402882351F081E0C13069
:10DC700009F080E023E047E152E3612F0E945CD885
:10DC80008091D907882309F463C0C13009F060C0CE
:10DC90008CE89CEA5FDD58C0D230D9F48091340220
:10DCA000882351F081E0C23009F080E020E24DE0AD
:10DCB00052E3612F0E945CD88091D907882309F430
:10DCC00047C0C23009F044C0B0922308A092220895
:10DCD00039C0D330E9F480913402882351F081E0D7
:10DCE000C33009F080E020E248EF51E3612F0E9449
:10DCF0005CD88091D907882359F1C33049F5D09277
:10DD00002308C09222080E949E480E9407581CC007
:10DD1000D430F1F480913402882351F081E0C43092
:10DD200009F080E020E247EE51E3612F0E945CD8C9
:10DD30008091D907882361F0C43051F4F092230810
:10DD4000E09222080E949E488091C90781117EC0FE
:10DD500080911108909112082091150830911608B1
:10DD6000232B11F4892B31F1D53031F58091340218
:10DD7000882351F081E0C53009F080E020E24AEDCF
:10DD800051E3612F0E945CD88091D907882309F460
:10DD90005BC0C53009F058C01092140810921308E7
:10DDA0000E9406D10E9407588091C907882309F470
:10DDB0004BC04CC005E001C006E0D0131DC08091EF
:10DDC0003402882349F081E0CD1380E023E04EEC5B
:10DDD00051E3612F0E945CD88091D907882359F0C4
:10DDE000CD1309C085E190E7B5DC8091C9078111A9
:10DDF0002DC00C2F01C00D2F81E0800FD81749F0E6
:10DE00001F5FDF5F153009F012CF0E5F0093F70739
:10DE10001DC080913402882349F081E0CD1380E059
:10DE200023E042EC51E3612F0E945CD88091D90736
:10DE3000882331F3CD13E4CF81E39FE68BDC80911F
:10DE4000C9078823E9F202C006E0D6CFDF91CF915F
:10DE50001F910F91FF90EF90DF90CF90BF90AF9008
:10DE600008951F93CF93DF931092D7078091FF07F8
:10DE700090910008A0910108B0910208813090486B
:10DE8000A105B10540F01092FF0710920008109212
:10DE9000010810920208C091FF078091F60718163A
:10DEA000DCF4282F082E000C330B215031094C2FA5
:10DEB0000C2E000C550B4217530774F0CFEFC80F10
:10DEC0008C2F90E0A0E0B0E08093FF0790930008D3
:10DED000A0930108B09302081092C9078091C80767
:10DEE000C81714F4C093C8078091C807082E000C07
:10DEF000990B04962C2F0C2E000C330B82179307D2
:10DF000024F48CEF8C0F8093C8071091C807D0E0E1
:10DF1000111117C080913402882349F081E0C111AA
:10DF200080E024E045EB51E36D2F0E945CD88091A6
:10DF3000D907882309F46DC0C1116BC00E940D5828
:10DF400064C01130F9F480913402882351F081E0EB
:10DF5000C13009F080E020E249EA51E36D2F0E94D0
:10DF60005CD88091D907882309F453C0C13009F0E7
:10DF700050C04091130E5091140E60910B0E709191
:10DF80000C0E1CC01230F9F480913402882351F039
:10DF900081E0C23009F080E020E249E951E36D2FD1
:10DFA0000E945CD88091D907882399F1C23089F505
:10DFB0004091130E5091140E6FEF7FEF80910F0E72
:10DFC0009091100E20C0133021F5809134028823E7
:10DFD00051F081E0C33009F080E020E249E851E3EC
:10DFE0006D2F0E945CD88091D907882391F0C330AF
:10DFF00081F44091130E5091140E60910B0E7091AC
:10E000000C0E80E090E00E94597A8091C90781113E
:10E0100008C0DF5F1F5FD53009F07ACF84E08093BE
:10E02000F607DF91CF911F9108951F93CF93DF9350
:10E030001092D7078091FF0790910008A0910108E6
:10E04000B091020881309048A105B10540F01092CE
:10E05000FF07109200081092010810920208C09168
:10E06000FF078091F5071816DCF4282F082E000C06
:10E07000330B215031094C2F0C2E000C550B42173D
:10E08000530774F0CFEFC80F8C2F90E0A0E0B0E002
:10E090008093FF0790930008A0930108B0930208B3
:10E0A0001092C9078091C807C81714F4C093C80715
:10E0B0008091C807082E000C990B04962C2F0C2E6B
:10E0C000000C330B8217930724F48CEF8C0F809392
:10E0D000C8071091C807D0E0111117C08091340211
:10E0E000882349F081E0C11180E024E041E851E358
:10E0F0006D2F0E945CD88091D907882309F46DC0E8
:10E10000C1116BC00E940D5864C01130F9F48091A8
:10E110003402882351F081E0C13009F080E020E230
:10E1200045E751E36D2F0E945CD88091D907882381
:10E1300009F453C0C13009F050C04091110E509104
:10E14000120E6091090E70910A0E1CC01230F9F483
:10E1500080913402882351F081E0C23009F080E0E0
:10E1600020E245E651E36D2F0E945CD88091D907EB
:10E17000882399F1C23089F54091110E5091120E09
:10E180006FEF7FEF80910D0E90910E0E20C0133037
:10E1900021F580913402882351F081E0C33009F0E9
:10E1A00080E020E245E551E36D2F0E945CD880912C
:10E1B000D907882391F0C33081F44091110E50911A
:10E1C000120E6091090E70910A0E80E090E00E949C
:10E1D000597A8091C907811108C0DF5F1F5FD53070
:10E1E00009F07ACF84E08093F507DF91CF911F91FA
:10E1F0000895FF920F931F93CF93DF931092D70749
:10E200008091FF0790910008A0910108B091020849
:10E2100081309048A105B10540F01092FF0710929F
:10E2200000081092010810920208C091FF07809127
:10E23000F4071816DCF4282F082E000C330B21509D
:10E2400031094C2F0C2E000C550B4217530774F05C
:10E25000CFEFC80F8C2F90E0A0E0B0E08093FF07D5
:10E2600090930008A0930108B09302081092C90788
:10E270008091C807C81714F4C093C8078091C807D5
:10E28000082E000C990B04962C2F0C2E000C330B2F
:10E290008217930724F48CEF8C0F8093C80710919A
:10E2A000C807D0E0FF24F394111117C08091340205
:10E2B000882349F081E0C11180E024E040E551E38A
:10E2C0006D2F0E945CD88091D907882309F4E4C09F
:10E2D000C111E2C00E940D58DBC0113021F58091C0
:10E2E0003402882379F083E292E00E9401D89C01F5
:10E2F00081E0C13009F080E000E04AE451E36D2F95
:10E300000E944CDE8091D907882309F4C5C0C13032
:10E3100009F0C2C027EE33E04AE050E063E272E069
:10E3200084E491E3B3C0123071F580913402882304
:10E3300079F081E198E00E9401D89C0181E0C2302F
:10E3400009F080E000E04DE351E36D2F0E944CDEC8
:10E350008091D907882309F49FC0C23009F09CC07E
:10E36000F092D7071092D3071092D4071092D507D6
:10E370001092D6072AE532E744E051E061E178E007
:10E3800086E391E32FC0133081F580913402882316
:10E3900079F085E198E00E9401D89C0181E0C330CA
:10E3A00009F080E000E042E351E36D2F0E944CDE73
:10E3B0008091D907882309F46FC0C33009F06CC07D
:10E3C000F092D7071092D3071092D4071092D50776
:10E3D0001092D6072DE532E747E850E065E178E096
:10E3E0008EE291E30E942DE053C0143061F58091DC
:10E3F0003402882379F083E198E00E9401D89C01DF
:10E4000081E0C43009F080E000E044E251E36D2F88
:10E410000E944CDE8091D9078823F1F1C430E1F5E8
:10E42000F092D7071092D3071092D4071092D50715
:10E430001092D6072FEF30E040E050E063E178E043
:10E440008AE191E323C0153039F5809134028823A5
:10E4500079F081E292E00E9401D89C0181E0C53010
:10E4600009F080E000E045E151E36D2F0E944CDEB1
:10E470008091D907882381F0C53071F427EE33E00D
:10E480004AE050E061E272E080E191E30E94D7DF70
:10E490008091C907811108C0DF5F1F5FD53009F087
:10E4A00003CF86E08093F407DF91CF911F910F9106
:10E4B000FF90089580E00C94D3D00C94A0D0EF92FC
:10E4C000FF921F93CF93DF937C017093FE076093BD
:10E4D000FD071092D7078091FF0790910008A09147
:10E4E0000108B091020881309048A105B10540F0C3
:10E4F0001092FF0710920008109201081092020873
:10E50000C091FF078091FC071816DCF4282F082E15
:10E51000000C330B215031094C2F0C2E000C550BE5
:10E520004217530774F0CFEFC80F8C2F90E0A0E094
:10E53000B0E08093FF0790930008A0930108B09388
:10E5400002081092C9078091C807C81714F4C09335
:10E55000C8072091C807022E000C330B2C5F3F4FD9
:10E560008C2F0C2E000C990B2817390724F48CEFF4
:10E570008C0F8093C8071091C807D0E091E081E02C
:10E58000E816F10459F122E0E216F10409F448C05A
:10E59000E114F10409F066C0111189C09923B1F0AA
:10E5A0001C16A4F08091FF0790910008A09101082B
:10E5B000B09102080196A11DB11D8093FF079093B1
:10E5C0000008A0930108B0930208CF5F8091340245
:10E5D000882309F4D7C063E872E365C0111167C0EE
:10E5E0009923B1F01C16A4F08091FF0790910008C8
:10E5F000A0910108B09102080196A11DB11D809360
:10E60000FF0790930008A0930108B0930208CF5F22
:10E6100080913402882309F4B5C06CE772E343C0EB
:10E62000111145C09923B1F01C16A4F08091FF0789
:10E6300090910008A0910108B09102080196A11DD7
:10E64000B11D8093FF0790930008A0930108B09339
:10E650000208CF5F80913402882309F493C065E7F4
:10E6600072E321C0111123C09923B1F01C16A4F04C
:10E670008091FF0790910008A0910108B0910208D5
:10E680000196A11DB11D8093FF0790930008A093F0
:10E690000108B0930208CF5F80913402882309F407
:10E6A00071C06CE672E38D2F0E9417E36BC01130CE
:10E6B000C9F480913402882351F081E0C13009F01F
:10E6C00080E024E042E652E36D2F0E945CD8809106
:10E6D000D907882309F456C0C13009F053C00E94FD
:10E6E0000D584CC01230B9F480913402882351F097
:10E6F00081E0C23009F080E023E048E552E36D2F6D
:10E700000E945CD88091D9078823E1F1C230D1F50D
:10E710008FEB9BE631C01330B9F48091340288232B
:10E7200051F081E0C33009F080E023E04FE452E390
:10E730006D2F0E945CD88091D907882319F1C330CE
:10E7400009F584ED9BE618C01430E1F480913402A1
:10E75000882351F081E0C43009F080E023E044E4F4
:10E7600052E36D2F0E945CD88091D907882351F025
:10E77000C43041F489EE9BE60E94AA6B8091C907E0
:10E78000811108C0DF5F1F5F90E0D53009F0F7CE40
:10E79000D093FC07DF91CF911F91FF90EF900895E8
:10E7A000EF92FF920F931F93CF93DF93CDB7DEB716
:10E7B0006F970FB6F894DEBF0FBECDBF7B0106ED9D
:10E7C00011E128ED31E1F8013183208322E030E0CE
:10E7D0003093101420930F149093121480931114FB
:10E7E00040E050E0BA018CED91E10E94F08EF8011A
:10E7F000808191812BE1FC013496DE011596019018
:10E800000D922A95E1F7FC01828193819C838B8391
:10E8100080E893E09A838983A701BE016F5F7F4FF1
:10E820008AE094E00E9410C6CE0101960E946F4FCC
:10E830006F960FB6F894DEBF0FBECDBFDF91CF91BC
:10E840001F910F91FF90EF90089510928A1180917F
:10E850005813882321F085E593E10C944C91089599
:10E86000E091F810F091F9100190F081E02D682FFF
:10E8700088EF90E11994CF93DF9380913511811146
:10E8800007C081E0809335118CEF90E10E94C25067
:10E89000C091FE10D091FF10E0912D11F0912E113A
:10E8A00082E01995E0912D11F0912E1181E01995DA
:10E8B00020E030E044E1BE018CEF90E10E94405046
:10E8C0002FE231E147E1BE018CEF90E10E94405020
:10E8D000E0912D11F0912E1180E0DF91CF911994EC
:10E8E0006F927F928F929F92AF92BF92DF92EF9240
:10E8F000FF920F931F93CF93DF93CDB7DEB7AD9702
:10E900000FB6F894DEBF0FBECDBF20918B1122232E
:10E9100009F4EFC1D62E7C0180915813882309F4A5
:10E920009FC0442309F4BAC180917013882329F150
:10E93000E3EDF3E384918F010F5F1F4F882321F0F4
:10E940000E941C87F801F6CFE0E9F3E384918F0180
:10E950000F5F1F4F882321F00E941C87F801F6CF1C
:10E9600061E070E080E090E00E9489878AE00E9488
:10E970001C8787E893E30E94778A8FE28093751360
:10E98000B12C21E006E713E19FE1A92E80912D1320
:10E99000B816B8F4AB9CC0011124B80185509E4E46
:10E9A0002DA70E94FC90C8012DA58C010196F801AD
:10E9B0003081332321F02D3811F02F5FF6CFB3943F
:10E9C000E5CF27FD08C0B80185E593E10E94FC90E2
:10E9D000E8E3F4E403C0F8011082FACF84918F01D8
:10E9E0000F5F1F4F882321F00E941C87F801F6CF8C
:10E9F000B7018EE693E30E94158260917013FDE8E3
:10EA00006F9FB00111246B587C4E83E693E30E9404
:10EA1000158240910614509107146091081470916A
:10EA200009148DE593E30E94AD818AE00E941C8762
:10EA30008091701394E0899FF0011124EF58FC4EEF
:10EA400040910614509107146091081470910914B4
:10EA500040835183628373838F5F809370130DC0F3
:10EA60001092701382E0B82E1BC1B70180E593E3CA
:10EA70000E9415828AE00E941C87E7DE1D821886AC
:10EA80001C821B8280E893E09A83898387EB91E163
:10EA90009093D7118093D611F70180818F3209F0BE
:10EAA00067C087010F5F1F4FCE0101963C01011522
:10EAB000110509F463C06FE270E0C8010E9488EF9D
:10EAC0005C01009709F45BC00817190708F057C0EC
:10EAD0004C01801A910AA401B801CE0180960E94CF
:10EAE000B1EFE0E2F0E0EC0FFD1FE80DF91D108240
:10EAF000FE01B0964F018F01F80181918F018823AB
:10EB000019F00E941C87F8CF8AE00E941C87609150
:10EB1000D6117091D7116115710511F06C5F7F4F9F
:10EB200021E0AE01405E5F4FCE0105960E94D29378
:10EB3000811116C0ECE3F3E384918F010F5F1F4F47
:10EB4000882321F00E941C87F801F6CFF4018191FF
:10EB50004F01882319F00E941C87F8CF8EE287C0EE
:10EB60007092D7116092D61185010F5F1F4F9FCF12
:10EB700088ED91E19093D7118093D6118701909100
:10EB8000D6118091D711692F782FDD2009F459C053
:10EB90006115710511F06C5F7F4F21E0A80185E5DB
:10EBA00093E10E94D293882309F447C080916613B1
:10EBB00090916713A0916813B09169138093021428
:10EBC00090930314A0930414B0930514B8018EE23B
:10EBD00093E30E94158240910214509103146091B6
:10EBE00004147091051486E293E30E94AD818AE0DB
:10EBF0000E941C8710920614109207141092081499
:10EC000010920914E7E1F3E384917F019FEFE91A81
:10EC1000F90A882321F00E941C87F701F5CFB8017B
:10EC200080E090E0BDDD80919A11882319F08AE997
:10EC300091E101C0C80160E02AC0B80183E093E31C
:10EC400010C06115710511F06C5F7F4F26E5A801BA
:10EC500085E593E10E94D29381110CC0B8018FEE3B
:10EC600092E30E9415828EE20E941C878AE00E9435
:10EC70001C870FC081E080938811B7018DED92E36E
:10EC80000E9415828AE00E941C8760E0C8010E94F1
:10EC90000CD9CE0101960E946F4F2BC0BB24B394B8
:10ECA000E8E3F4E484918F010F5F1F4F882321F084
:10ECB0000E941C87F801F6CFE8E5F3E384918F0109
:10ECC0000F5F1F4F882321F00E941C87F801F6CFA9
:10ECD000E1E0BE1619F00BEE13E002C001EF13E005
:10ECE000F80181918F01882309F4BFCE0E941C870F
:10ECF000F7CFAD960FB6F894DEBF0FBECDBFDF9154
:10ED0000CF911F910F91FF90EF90DF90BF90AF9048
:10ED10009F908F907F906F900895CF92DF92EF92A7
:10ED2000FF920F931F93CF93DF93CDB7DEB7EDB66E
:10ED3000FEB6DC010D900020E9F79D01281B390B80
:10ED40002C5F3F4F4DB75EB7421B530B0FB6F89485
:10ED50005EBF0FBE4DBF0DB71EB70F5F1F4F9F9316
:10ED60008F9386ED92E39F938F931F930F930E944F
:10ED7000C5E7680154E0C50ED11C0F900F900F90AD
:10ED80000F900F900F90F6018081882349F0082E94
:10ED9000000C990B0E944CEFF60181936F01F3CFA9
:10EDA00060E0C8010E948248882319F0C8010E94CF
:10EDB000488A82ED92E390932308809322080E9470
:10EDC0009E480FB6F894FEBE0FBEEDBEDF91CF9108
:10EDD0001F910F91FF90EF90DF90CF900895AF9229
:10EDE000BF92CF92DF92EF92FF920F931F93CF9338
:10EDF000DF93CDB7DEB7AA970FB6F894DEBF0FBE8C
:10EE0000CDBF8091B6118F938091B5118F9389EC0E
:10EE100092E39F938F937E0181E2E80EF11CFF92B3
:10EE2000EF920E94C5E70F900F900F900F900F90F8
:10EE30000F9010E0F70101900020E9F73197EE19EB
:10EE4000FF091E1784F46701C10ED11C17FDDA9467
:10EE5000F6018081082E000C990B0E944CEFF60100
:10EE600080831F5FE7CF40E050E0BA018BEB91E178
:10EE70000E94F08E00E0CE0101966C018091BE11DF
:10EE8000823028F4011114C08FEF9FEF16C08091DB
:10EE9000C3119091C411A091C511B091C6118F7189
:10EEA0009927AA27BB27892B8A2B8B2B59F71AC0A6
:10EEB0008091B5119091B61101969093B6118093FF
:10EEC000B511AA960FB6F894DEBF0FBECDBFDF9185
:10EED000CF911F910F91FF90EF90DF90CF90BF9057
:10EEE000AF90089540E050E0B6018BEB91E10E94B5
:10EEF0002B8418163CF6F60101900020E9F73197B3
:10EF00001E2F1C19115068F05601A10EB11C17FDDF
:10EF1000BA94F501808190E00E944CEFF501808366
:10EF2000F1CF8A858E3709F4A9CF45E050E0B701CB
:10EF3000C6010E94A3EF892B09F0A0CFC701EDDE27
:10EF400001E09CCFCF92DF92EF92FF921F93CF937D
:10EF5000DF9310928B118091BE11882321F08BEBEF
:10EF600091E10E944C911092321310922F1385E37D
:10EF700080932E130E94975BEB01A89561E080912E
:10EF80002E130E945C5A8EE293E10E9445962398CC
:10EF9000229A219A209A289A85E08093301382E55C
:10EFA0008CBD1DBC1AE08FEF0E944A961150D9F714
:10EFB00020E030E0A90160E08EE293E10E945696E5
:10EFC000182F80933113813049F00E94975B6C1B9E
:10EFD0007D0B613D774060F381E054C02AEA31E067
:10EFE00040E050E068E08EE293E10E94569682FF96
:10EFF00003C0109332130EC014E00E944F9680930A
:10F0000031131150D1F78A3A11F082E03BC082E00F
:10F010008093321380913213823021F0C12CD12C95
:10F02000760105C0C12CD12CE12C80E4F82E20E023
:10F0300030E0A90167E38EE293E10E945696A701B2
:10F04000960169E28EE293E10E9456968093311315
:10F05000882349F00E94975B6C1B7D0B613D7740D4
:10F0600030F38AE00FC080913213823011F520E036
:10F0700030E0A9016AE38EE293E10E94569688236C
:10F0800051F088E080932F138EE293E10E94459621
:10F09000E8E3F4E41AC00E944F96807C803C19F4A7
:10F0A00083E0809332130E944F960E944F960E94F5
:10F0B0004F968EE293E10E9445961092301381E0C4
:10F0C0000E94B0C3811132C015C08491EF01219616
:10F0D000882321F00E941C87FE01F7CFEBEBF2E3BF
:10F0E0008491EF012196882309F457C00E941C8760
:10F0F000FE01F6CF80E00E94B0C3811117C0E3ED9E
:10F10000F3E38491EF012196882321F00E941C876C
:10F11000FE01F7CFE7EAF2E38491EF01219688231D
:10F1200009F43BC00E941C87FE01F6CF63E373E144
:10F130008BEB91E10E94A990811116C0E3EDF3E3FE
:10F140008491EF012196882321F00E941C87FE0103
:10F15000F7CFE6E9F2E38491EF0121968823E9F005
:10F160000E941C87FE01F7CF81E080938B11E8E3BA
:10F17000F4E48491EF012196882321F00E941C87FA
:10F18000FE01F7CFEAE8F2E38491EF0121968823AC
:10F1900021F00E941C87FE01F7CF8BE1EBEBF1E140
:10F1A000ACEDB1E101900D928A95E1F78091B91132
:10F1B0009091BA119093DB118093DA1187EB91E172
:10F1C0009093D7118093D611DF91CF911F91FF902B
:10F1D000EF90DF90CF9008950F931F93CF93DF931D
:10F1E0008C01EB019091681120916911921307C075
:10F1F0008CE591E10E94CE440E9448D3F3CFF80100
:10F20000A081B181488159818091671134E0839F49
:10F21000F0011124E05AFE4EB387A2875587448738
:10F220009F5F909368118F5F821719F08093671129
:10F2300002C010926711DF91CF911F910F91089535
:10F24000CF93DF93CDB7DEB780912108811110C035
:10F250009E01275F3F4F4F81588562E470E087E64B
:10F2600092E00E94F4E70E945FC583E0809334023D
:10F27000DF91CF91089580917A1190917B11813027
:10F280009105B9F1029759F40E9429C560937C1148
:10F2900070937D1180937E1190937F1118C010920E
:10F2A000801110928111109282111092831110928C
:10F2B000841110928511109286111092871110926C
:10F2C0007C1110927D1110927E1110927F1181E0BD
:10F2D00090E090937B1180937A110E94975B6093EA
:10F2E000801170938111809382119093831181E03A
:10F2F000089580E0089580917A1190917B11019793
:10F3000091F482E090E090937B1180937A110E94B7
:10F31000975B60938411709385118093861190930D
:10F32000871181E0089580E00895BC0180E090E0BD
:10F330004AE00E9423878DE00E941C878AE00C949B
:10F340001C878F929F92AF92BF92CF92DF92EF92E3
:10F35000FF92CF9320E030E04AE754E4FC01608163
:10F360007181828193810E9491E80E9493ED6B01EB
:10F370007C01611571058105910561F097FF0AC057
:10F38000F094E094D094C094C11CD11CE11CF11CF9
:10F390008DE201C080E280931A08C701B60128EE11
:10F3A00033E040E050E00E9413EC8AE0882E912C7C
:10F3B000A12CB12CCA01B901A50194010E9413EC42
:10F3C000605D60931B088EE280931C08C701B60144
:10F3D00024E630E040E050E00E9413ECCA01B9019D
:10F3E000A50194010E9413EC605D60931D08C701A4
:10F3F000B601A50194010E9413ECC62FCA01B90100
:10F40000A50194010E9413EC605D60931E08C05D2D
:10F41000C0931F088AE198E0CF91FF90EF90DF90B2
:10F42000CF90BF90AF909F908F900895FF920F93D1
:10F430001F93CF93DF931F92CDB7DEB7982F862F00
:10F44000692F49830E94CE5D9091301180911808F8
:10F450004981891738F190913211809117089817D6
:10F4600008F180919A118823D1F01092AF110AE926
:10F4700011E1442319F082E00E94C75E85E1F82E75
:10F48000F80181918F01882321F00E94B05EF81A63
:10F49000F7CFFF2039F080E2E3D9FA94FACF0DE8F4
:10F4A00011E1E7CF0F90DF91CF911F910F91FF9066
:10F4B00008950F931F93CF93DF93EB018A011816E2
:10F4C00019066CF4843121E0920714F083E191E095
:10F4D000909312088093110880E00E94D3D0D7FD4A
:10F4E00006C0D0931608C09315080E94A0D01093B0
:10F4F000140800931308DF91CF911F910F910C9482
:10F500000758CF93DF931F92CDB7DEB7698341E0F1
:10F5100050E0BE016F5F7F4F04960E94C3940F902E
:10F52000DF91CF9108958091F40C80FF03C0899AF8
:10F530008FEF02C0899881E0809335028091F40CAE
:10F5400081FF03C08F988FEF02C08F9A81E0809374
:10F5500036028091F40C9FB782FF09C0F894809125
:10F560000B01826080930B019FBF8FEF08C0F8945E
:10F5700080910B018D7F80930B019FBF81E0809371
:10F5800037028091F40C83FF03C016988FEF02C0FE
:10F59000169A81E080933802089590915A118091D3
:10F5A0005B11981731F080915B118F5F8F708093A2
:10F5B0005B1108951F920F920FB60F9211240BB694
:10F5C0000F92BF92CF92DF92EF92FF920F931F9311
:10F5D0002F933F934F935F936F937F938F939F935B
:10F5E000AF93BF93EF93FF93CF93DF9300D01F921E
:10F5F000CDB7DEB780916E008B7F80936E008091D7
:10F600006F008D7F80936F007894C090150DD0901F
:10F61000160DE090170DF090180DC114D104E104FF
:10F62000F10409F442C080910B02811104C0809161
:10F63000F0048823D1F10E941849F9EBCF16FBE0C2
:10F64000DF06E104F10488F008EBC01A0BE0D00AF1
:10F65000E108F108C092150DD092160DE092170D39
:10F66000F092180D88EB9BE009C0C6011092150DB1
:10F670001092160D1092170D1092180D909389008C
:10F6800080938800209188003091890080918400C7
:10F690009091850040962817390708F06DC0809139
:10F6A00084009091850040961FC08091F50C909148
:10F6B000F60C009709F493C08C01015011091093C6
:10F6C000F60C0093F50C10921A141092191465DFC1
:10F6D000012B41F48AED9BE3909323088093220849
:10F6E0000E949E4888EC90E0909389008093880067
:10F6F00043C0C8011ADE24E630E080910B02882363
:10F7000009F4B9C4C901293BBBE03B0708F0ECC5CB
:10F7100090938900809388008091070D9091080D47
:10F72000A091090DB0910A0D820F931FA11DB11D6B
:10F730008093070D9093080DA093090DB0930A0DC7
:10F7400020918800309189008091840090918500FB
:10F7500040962817390748F48091840090918500DD
:10F7600040969093890080938800BB2029F01092E6
:10F770001A141092191411DFF8948091B706882397
:10F7800021F080916E008B7F03C080916E008460B9
:10F7900080936E0080916F00826080936F000F9065
:10F7A0000F900F900F90DF91CF91FF91EF91BF914C
:10F7B000AF919F918F917F916F915F914F913F9109
:10F7C0002F911F910F91FF90EF90DF90CF90BF90FE
:10F7D0000F900BBE0F900FBE0F901F901895E091E9
:10F7E0001914F0911A14309709F0B1C190915A117F
:10F7F00080915B11981751F1E0915B111DE4E19F3D
:10F80000F0011124EC5DF74FC090CE07D090CF07E8
:10F81000E090D007F090D1079F01275B3F4FD901BF
:10F820004D915D916D917C91D701C601841B950B23
:10F83000A60BB70B8093CE079093CF07A093D0076A
:10F84000B093D1078081886080830BC08FB7F89414
:10F850001092CE071092CF071092D0071092D107C6
:10F860008FBFF0931A14E0931914309709F46CC108
:10F8700052A18091F40C418158130AC0242F30E02A
:10F8800080913902082E000C990B2817390729F0AE
:10F890005093F40C4093390246DE1092110D1092F1
:10F8A000120D1092130D1092140DE0911914F09195
:10F8B0001A1487A990AD8134BCE99B0728F48132E2
:10F8C000EEE49E0748F002C080E49CE99695879597
:10F8D0009695879524E007C08131F7E29F0730F0C5
:10F8E0009695879522E02093100D08C021E0209383
:10F8F000100D8032910510F480E290E07C0100E26E
:10F90000E01AF108E11418E0F106E0F0EF2DFF270E
:10F91000EE0FFF1FEE0FFF1FCF018652984CFC0128
:10F920003296459154916E2DAA27659F9001649F50
:10F93000210D3A1F06942A1F3A1F1124FC018591BC
:10F9400094911CC09701369527952C7F26523C4CEC
:10F95000F90185919491F901329665917491A7010D
:10F9600047705527649F9001659F300D749F300D3F
:10F970001124B3E036952795BA95E1F7821B930BD6
:10F980008436910570F407EF13E0D8018D918D0155
:10F99000882319F00E941C87F8CFC701C6DC84E6D3
:10F9A00090E090930F0D80930E0D8091100D809339
:10F9B0000D0DE0911914F0911A1483AD94AD90934C
:10F9C0000C0D80930B0D8134BCE99B0728F4813228
:10F9D000EEE49E0748F002C080E49CE99695879586
:10F9E0009695879524E007C08131F7E29F0730F0B4
:10F9F0009695879522E02093100D08C021E0209372
:10FA0000100D8032910510F480E290E07C0100E25C
:10FA1000E01AF108E11418E0F106E0F0EF2DFF27FD
:10FA2000EE0FFF1FEE0FFF1FCF018652984CFC0117
:10FA30003296459154916E2DAA27659F9001649F3F
:10FA4000210D3A1F06942A1F3A1F1124FC018591AB
:10FA500094911CC09701369527952C7F26523C4CDB
:10FA6000F90185919491F901329665917491A701FC
:10FA700047705527649F9001659F300D749F300D2E
:10FA8000112453E0369527955A95E1F7821B930B85
:10FA90008436910570F407EF13E0D8018D918D0144
:10FAA000882319F00E941C87F8CFC7013EDC84E64A
:10FAB00090E0AC0160E070E04093070D5093080DBA
:10FAC0006093090D70930A0D9093890080938800CC
:10FAD000E0911914F0911A1482899389A489B58947
:10FAE000B695A79597958795B095A0959095819592
:10FAF0009F4FAF4FBF4F8093030D9093040DA09382
:10FB0000050DB093060D8093FF0C9093000DA0930C
:10FB1000010DB093020D8093FB0C9093FC0CA0930D
:10FB2000FD0CB093FE0C8093F70C9093F80CA0930F
:10FB3000F90CB093FA0C109215141092161410923E
:10FB400017141092181403C080ED97E0CDCD80916A
:10FB50000B028111C6C38091F0048111C2C32091B0
:10FB6000100D222309F4AFC1E0911914F0911A1479
:10FB70004091F70C5091F80C6091F90C7091FA0CCF
:10FB800082819381A481B581840F951FA61FB71F21
:10FB90008093F70C9093F80CA093F90CB093FA0CA7
:10FBA000181619061A061B060CF4889AE091191407
:10FBB000F0911A144091FB0C5091FC0C6091FD0CDB
:10FBC0007091FE0C86819781A085B185840F951F69
:10FBD000A61FB71F8093FB0C9093FC0CA093FD0C09
:10FBE000B093FE0C181619061A061B060CF48E9A12
:10FBF000E0911914F0911A144091FF0C5091000DEE
:10FC00006091010D7091020D82859385A485B58563
:10FC1000840F951FA61FB71F8093FF0C9093000DB4
:10FC2000A093010DB093020D181619061A061B06B3
:10FC300044F49FB7F89480910B01886080930B0186
:10FC40009FBFE0911914F0911A144091030D509147
:10FC5000040D6091050D7091060D86859785A0892C
:10FC6000B189840F951FA61FB71F8093030D909332
:10FC7000040DA093050DB093060D181619061A066B
:10FC80001B060CF4149A8091F70C9091F80CA0913B
:10FC9000F90CB091FA0C181619061A061B0684F511
:10FCA000E0911914F0911A14428953896489758975
:10FCB000841B950BA60BB70B8093F70C9093F80C55
:10FCC000A093F90CB093FA0C8091350240911B146B
:10FCD00050911C1460911D1470911E14082E000C7C
:10FCE000990BAA0BBB0B840F951FA61FB71F809300
:10FCF0001B1490931C14A0931D14B0931E14889889
:10FD00008091FB0C9091FC0CA091FD0CB091FE0C2D
:10FD1000181619061A061B0684F5E0911914F091BD
:10FD20001A144289538964897589841B950BA60B23
:10FD3000B70B8093FB0C9093FC0CA093FD0CB0933D
:10FD4000FE0C8091360240911F1450912014609156
:10FD5000211470912214082E000C990BAA0BBB0BD6
:10FD6000840F951FA61FB71F80931F149093201414
:10FD7000A0932114B09322148E988091FF0C90913F
:10FD8000000DA091010DB091020D181619061A066A
:10FD90001B06BCF5E0911914F0911A14428953899D
:10FDA00064897589841B950BA60BB70B8093FF0C98
:10FDB0009093000DA093010DB093020D8091370236
:10FDC00040912314509124146091251470912614AD
:10FDD000082E000C990BAA0BBB0B840F951FA61FB6
:10FDE000B71F8093231490932414A0932514B093E9
:10FDF00026149FB7F89480910B01877F80930B01A5
:10FE00009FBF8091030D9091040DA091050DB091BD
:10FE1000060D181619061A061B0684F5E09119142A
:10FE2000F0911A144289538964897589841B950B52
:10FE3000A60BB70B8093030D9093040DA093050DB3
:10FE4000B093060D809138024091271450912814E8
:10FE50006091291470912A14082E000C990BAA0B9A
:10FE6000BB0B840F951FA61FB71F80932714909379
:10FE70002814A0932914B0932A141498809115146F
:10FE800090911614A0911714B09118140196A11D09
:10FE9000B11D8093151490931614A0931714B0936A
:10FEA00018142150E0911914F0911A1442895389C1
:10FEB0006489758984179507A607B70708F451CE9A
:10FEC000BB24B39401C0B12C409115145091161469
:10FED0006091171470911814E0901914F0901A148E
:10FEE000F70186899789A08DB18D84179507A6079C
:10FEF000B70708F4C6C04091070D5091080D6091F6
:10FF0000090D70910A0D068D178D20A131A1AA2728
:10FF1000419FB12D529FC001629F900D619F800D46
:10FF2000911D429FB00D811D9A1F519FB00D811DE3
:10FF30009A1F609FB00D811D9A1F509FB10D8A1F9F
:10FF40009A1FB6958A1F9A1F349F800D911D359F69
:10FF5000900D112423AD34AD820F931F90930C0D9F
:10FF600080930B0D47A950AD61AD72ADA0E0B0E03C
:10FF7000481759076A077B0720F450930C0D4093EC
:10FF80000B0D80910B0D90910C0D8134BCE99B07FA
:10FF900028F48132EEE49E0748F002C080E49CE938
:10FFA000969587959695879524E007C08131F7E26D
:10FFB0009F0730F09695879522E02093100D08C09A
:10FFC00021E02093100D8032910510F480E290E042
:10FFD0008C0100521109011528E01207E8F0E12F09
:10FFE000FF27EE0FFF1FEE0FFF1FCF018652984C29
:10FFF000FC01329625913491AA27039FA001029F0C
:020000021000EC
:10000000410D5A1F06944A1F5A1F1124FC012591C5
:100010003491241B350B1FC09801369527952C7FF2
:1000200026523C4CF90145915491F9013296659163
:100030007491980127703327629FC001639F900DD0
:10004000729F900D1124F3E096958795FA95E1F74C
:100050009A01281B390B2436310508F04ECB77EF77
:10006000E72E73E0F72ED7018D917D01882309F4E7
:1000700040CBE2D6F8CF8091F004811143CBC90187
:1000800047CB40911514509116146091171470913C
:100090001814F701828D938DA48DB58D8417950763
:1000A000A607B70708F0EAC00091110D1091120DD4
:1000B0002091130D3091140D09831A832B833C83F7
:1000C000468D578D60A171A1AA27059FB12D169F5E
:1000D0006001269FD00C259FC00CD11C069FB00D3F
:1000E000C11CDA1E159FB00DC11CDA1E249FB00D75
:1000F000C11CDA1E149FB10DCA1EDA1EB695CA1EA7
:10010000DA1E709FC00CD11C719FD00C11248091FD
:100110000B0D90910C0DFF96C816D90680F48C1922
:100120009D0940815181628173816C01E12CF12C28
:10013000C416D506E606F70620F4CA0102C080817F
:10014000918181341CE9910728F481322EE49207D1
:1001500048F002C080E49CE996958795969587952E
:1001600024E007C0813137E2930730F096958795F8
:1001700022E02093100D08C021E02093100D803262
:10018000910510F480E290E08C01005211090115F4
:1001900048E01407E8F0E12FFF27EE0FFF1FEE0FF6
:1001A000FF1FCF018652984CFC0132962591349165
:1001B000AA27039FA001029F410D5A1F06944A1FC0
:1001C0005A1F1124FC0125913491241B350B1FC0AB
:1001D0009801369527952C7F26523C4CF901459184
:1001E0005491F901329665917491980127703327E3
:1001F000629FC001639F900D729F900D112423E0B8
:10020000969587952A95E1F79A01281B390B243694
:10021000310578F487EFE82E83E0F82ED7018D9131
:100220007D01882311F008D6F9CFC8017ED824E6D5
:1002300030E080910B02811104C08091F00488238A
:1002400039F0C901293BBBE03B0708F068C001C099
:10025000C901909389008093880089819A81AB813C
:10026000BC81820F931FA11DB11D8093110D90932E
:10027000120DA093130DB093140D62CA20910E0DB0
:1002800030910F0D80910B02811104C08091F00418
:100290008823F1F0293BEBE03E07D0F0C90168EB81
:1002A0007BE00E9413EF883E43E0940708F052C0C1
:1002B0008854944FA901481B590B60E070E04093AB
:1002C000150D5093160D6093170D7093180D9C012A
:1002D000309389002093880080910D0D8093100D3C
:1002E0002FCA0E9418493BCC68EB7BE00E9413EFB9
:1002F000883E03E0900780F48854944FA901481B7E
:10030000590B60E070E04093150D5093160D60930B
:10031000170D7093180DFCC988EB9BE0EFCF68EBCD
:100320007BE00E9413EF883E13E0910780F488542D
:10033000944FA901481B590B60E070E04093150DE4
:100340005093160D6093170D7093180D82CF88EBA4
:100350009BE0EFCF88EB9BE0ADCFCF92DF92EF92A7
:10036000FF92CF93DF936A017B01FC018491EF013F
:100370002196882319F060D5FE01F8CF4AE0C70125
:10038000B601DF91CF91FF90EF90DF90CF905BC5EA
:10039000CF92DF92EF92FF92CF93DF936A017B01BE
:1003A000FC018491EF012196882319F045D5FE01C7
:1003B000F8CF42E0C701B601DF91CF91FF90EF90F7
:1003C000DF90CF90C0C5CF92DF92EF92FF92CF9394
:1003D000DF936A017B01FC018491EF012196882360
:1003E00019F02AD5FE01F8CF42E0C701B601DF912E
:1003F000CF91FF90EF90DF90CF90A5C50F931F9303
:10040000CF93DF938B01FC018491EF012196882328
:1004100019F012D5FE01F8CFB801110F880B990B16
:10042000DF91CF911F910F9174C50F931F93CF93BD
:10043000DF931F921F92CDB7DEB7FC0184918F012D
:100440000F5F1F4F811102C08B0107C069837A8340
:10045000F3D4F80169817A81F1CFF80181918F019C
:10046000882311F0E9D4F9CF0F900F90DF91CF914D
:100470001F910F910895CF938091F3108823B9F1C4
:100480004091EB105091EC106091ED107091EE10D6
:100490002BEE3EE08091F4109091F5100E946E9149
:1004A000C82F811102C0C0E023C04091EF105091CD
:1004B000F0106091F1107091F21041155105610535
:1004C000710591F02BEE3EE08091F4109091F510C3
:1004D0000E946E91882339F31092EF101092F01061
:1004E0001092F1101092F2101092F31001C0C1E0BE
:1004F0008C2FCF910895CF92DF92EF92FF92CF93FE
:100500006B017C01C42F8091EB109091EC10A091B5
:10051000ED10B091EE108C159D05AE05BF05C9F02C
:10052000AADF811102C080E018C02BEE3EE0B701C7
:10053000A6018091F4109091F5100E94C596882331
:1005400091F3C092EB10D092EC10E092ED10F0928B
:10055000EE1081E0C1118093F310CF91FF90EF90E6
:10056000DF90CF9008954F925F926F927F928F921B
:100570009F92AF92BF92CF92DF92EF92FF920F9332
:100580001F93CF93DF93EC016A017B0128013901AE
:10059000423051056105710510F480E064C0898521
:1005A0009A85AB85BC850196A11DB11D8417950761
:1005B000A607B70790F38F89803149F48D2C9E2CC4
:1005C000AF2CBB248B899C89AD89BE890FC080323A
:1005D00021F78B889C88AD88BE88DB01CA0157E073
:1005E000B695A795979587955A95D1F7880E991E38
:1005F000AA1EBB1E41E0C501B4017DDF882369F25C
:100600009F89903161F4DD24EE24FF249601220FAE
:10061000331FF901E551F14F5182408211C0E89436
:10062000C7F8DD24EE24FF249601220F331F220F8A
:10063000331FF901E551F14F40825182628273828A
:100640009A89923080F04D815E816F817885840E29
:10065000951EA61EB71E8092EF109092F010A092E9
:10066000F110B092F210DF91CF911F910F91FF9096
:10067000EF90DF90CF90BF90AF909F908F907F9042
:100680006F905F904F900895CF92DF92EF92FF921C
:100690000F931F93CF93DF93FC0181859285A385F0
:1006A000B4850196A11DB11D84179507A607B7074C
:1006B00010F480E061C08789803149F4BB27A72FFF
:1006C000962F852FC388D488E588F6880FC080329E
:1006D00081F783899489A589B6896A017B01C7E07E
:1006E000F694E794D794C794CA95D1F78C0D9D1DC5
:1006F000AE1DBF1DE9016A017B018F014091EB1026
:100700005091EC106091ED107091EE1084179507E8
:10071000A607B70799F4F80187898031B1F4B701CA
:10072000A601552766277727440F551FFA01E55183
:10073000F14F80819181A0E0B0E019C040E0BC01A0
:10074000CD01D9DE8111E7CFB4CFB701A6014F7734
:10075000552766277727440F551F440F551FFA0169
:10076000E551F14F80819181A281B381BF7088836F
:100770009983AA83BB8381E0DF91CF911F910F9171
:10078000FF90EF90DF90CF9008954F925F926F921D
:100790007F92AF92BF92CF92DF92EF92FF920F9330
:1007A0001F93CF93DF9300D01F92CDB7DEB78C019C
:1007B00049835A836B837C835901C12CD12C7601E8
:1007C000412C82E0582E612C712C49815A816B8119
:1007D0007C819E012F5F3F4FC80156DF882341F186
:1007E000D301C201F801058404C0880F991FAA1F14
:1007F000BB1F0A94D2F7C80ED91EEA1EFB1E498100
:100800005A816B817C818789803139F481E0483F4E
:100810005F4F6105710538F4D8CF81E0483F5F4FE5
:100820006F4F7F4090F2F501C082D182E282F38265
:100830000F900F900F900F90DF91CF911F910F911C
:10084000FF90EF90DF90CF90BF90AF907F906F9030
:100850005F904F900895DF92EF92FF920F931F9356
:10086000CF93DF937C01EB018A018DE0D82E40E22B
:1008700050E0BE01C7010E94868F8032910539F099
:1008800021E0892B09F420E0822F81953EC0288148
:10089000222399F1253E59F32E3249F30115110512
:1008A00041F13B853F733F3021F54A8D5B8D452BF0
:1008B00001F52F713FEF320F3230D8F430E0215084
:1008C0003109D29EC001D39E900D1124D801A80FEA
:1008D000B91FFE0120E0AD01253088F431813D9340
:1008E0002F5F32962D30C1F7288126FF02C0FA0112
:1008F00015862B8523FDBBCF08C080E006C02B30BA
:1009000010F43481ECCF3681EACFDF91CF911F9183
:100910000F91FF90EF90DF900895CF92DF92EF92CA
:10092000FF92C0906302D0906402E0906502F09064
:1009300066028091790E882321F120E030E0A90140
:10094000C701B6010E942CE88823D9F020E030E0EE
:1009500040E05FE3C701B6010E9491E89B01AC0152
:100960000E9491E82BED3FE049E450E40E9491E8B9
:100970009B01AC0160E070E080E89FE30E942BEDFA
:1009800004C060E070E080E89FE3609343027093EE
:1009900044028093450290934602FF90EF90DF90CF
:1009A000CF9008954F925F926F927F92AF92BF92D5
:1009B000CF92DF92EF92FF920F931F93CF93DF932B
:1009C000009709F456C0FC01208121FD52C0EB01C3
:1009D0008C0147A050A461A472A4AFA0B8A4C9A47C
:1009E000DAA49501A601C301B2010E942CE887FF99
:1009F00040C0A3019201C301B2010E9491E82B0102
:100A00003C01F80183A994A9A5A9B6A9BC01CD010F
:100A100090589B01AC010E944FECF80127A530A92A
:100A200041A952A90E9491E89B01AC01C301B20106
:100A30000E944EEC0E94BAEE7B018C019B01AC013E
:100A4000B501C6010E942CE887FF02C0750186012E
:100A50009701A801B501C6010E942CE8882349F03E
:100A6000A701B8014FA358A769A77AA78881816019
:100A70008883DF91CF911F910F91FF90EF90DF90CE
:100A8000CF90BF90AF907F906F905F904F90089500
:100A90002F923F924F925F926F927F928F929F928E
:100AA000AF92BF92CF92DF92EF92FF920F931F937C
:100AB000CF93DF93CDB7DEB768970FB6F894DEBF5C
:100AC0000FBECDBF1C015B018A01DC01D7966D9181
:100AD0007D918D919C91DA970E9430E86B017C01A9
:100AE000F50120813181428153810E9491E80E9469
:100AF00015ED0E9498ED69877A878B879C87D801CE
:100B00002D913D914D915C91C701B6010E9491E8F4
:100B10000E9415ED0E9498ED6D877E878F87988BD8
:100B200029853A854B855C85283731054105510576
:100B300040F488E790E0A0E0B0E089879A87AB872F
:100B4000BC872D853E854F8558892837310541055D
:100B5000510540F488E790E0A0E0B0E08D879E87E3
:100B6000AF87B88B91012D5B3F4FD9018D919D913E
:100B70000D90BC91A02D8D839E83AF83B887BC015F
:100B8000CD010E9432E869837A838B839C836985D7
:100B90007A858B859C850E9430E8698B7A8B8B8B5C
:100BA0009C8B20E030E0A90169817A818B819C8156
:100BB0000E942CE8882339F1A7019601C701B601EC
:100BC0000E9491E84B015C0129893A894B895C8933
:100BD000CA01B9010E9491E89B01AC01C501B401B1
:100BE0000E944EEC4B015C0129813A814B815C8172
:100BF000CA01B9010E944FEC9B01AC01C501B401CF
:100C00000E942BED03C060E070E0CB010E9415ED67
:100C10000E9493ED2B013C016D817E818F8198852F
:100C200090958095709561957F4F8F4F9F4F0E9453
:100C300032E84B015C016D857E858F8598890E9425
:100C400030E86D837E838F83988720E030E0A901B0
:100C5000C501B4010E942CE8882349F12D813E8111
:100C60004F815885CA01B9010E9491E86D8B7E8B36
:100C70008F8B988FA7019601C701B6010E9491E85A
:100C80009B01AC016D897E898F89988D0E944EEC05
:100C90006B017C01A5019401C501B4010E944FECD8
:100CA0009B01AC01C701B6010E942BED03C060E0BF
:100CB00070E0CB010E94C4EDF10182889388A48882
:100CC000B58875016401C418D508E608F7080E94C4
:100CD00093EDC61AD70AE80AF90AF7FE6BC020E0BE
:100CE00030E0A90169817A818B819C810E942CE886
:100CF000882309F447C029813A814B815C81CA016C
:100D0000B9010E944FEC6B017C01C501B4010E9446
:100D100030E89B01AC01C701B6010E9491E86B016C
:100D20007C0129893A894B895C89CA01B9010E94F1
:100D300091E89B01AC01C701B6010E944EEC6B012A
:100D40007C012D813E814F815885CA01B9010E94E5
:100D500091E89B01AC01C701B6010E944FEC6B0109
:100D60007C0120E030E040E850E469817A818B81A9
:100D70009C810E9491E89B01AC01C701B6010E94D1
:100D80002BED03C060E070E0CB010E9415ED0E94E6
:100D900093ED2B013C0197FF03C0412C512C3201F4
:100DA000481459046A047B0410F024013501C12C55
:100DB000D12C76018FB7F894D1019C9193FD22C07C
:100DC000F101468A578A608E718EC40CD51CE61CD0
:100DD000F71C5A96CD92DD92ED92FC925D97298593
:100DE0003A854B855C85DB962D933D934D935C93C3
:100DF000DE97FF962D853E854F8558892083318368
:100E0000428353838FBF68960FB6F894DEBF0FBE40
:100E1000CDBFDF91CF911F910F91FF90EF90DF90A9
:100E2000CF90BF90AF909F908F907F906F905F908A
:100E30004F903F902F9008959091C00095FFFCCF68
:100E40008093C60008958F929F92AF92BF92EF92C7
:100E5000FF921F93CF93DF93CDB7DEB7A0970FB666
:100E6000F894DEBF0FBECDBF6115710581059105F8
:100E700079F110E0842E912CA12CB12CEE24E39476
:100E8000F12CEC0EFD1EE10EF11C17FDFA94A501EC
:100E900094010E94F1EBF7016083B901CA011F5F61
:100EA000611571058105910549F7115010F1E1E0D7
:100EB000F0E0EC0FFD1FE10FF11D17FDFA958081A9
:100EC0008A3010F097E301C090E3890FB5DFEDCFD2
:100ED00080E3A0960FB6F894DEBF0FBECDBFDF91C2
:100EE000CF911F91FF90EF90BF90AF909F908F9008
:100EF000A3CFA0960FB6F894DEBF0FBECDBFDF9193
:100F0000CF911F91FF90EF90BF90AF909F908F90E7
:100F10000895CF92DF92EF92FF926B017C0197FFD1
:100F20000AC08DE289DFF094E094D094C094C11C93
:100F3000D11CE11CF11C4AE0C701B601FF90EF9003
:100F4000DF90CF9080CF8F929F92AF92BF92CF923F
:100F5000DF92EF92FF92CF936B017C01B42E20E0E1
:100F600030E0A9010E942CE887FF06C08DE264DF13
:100F7000F7FAF094F7F8F094C0E060E070E080E0F9
:100F80009FE3CB1541F02DEC3CEC4CEC5DE30E9473
:100F900091E8CF5FF6CF9B01AC01C701B6010E947B
:100FA0004FEC6B017C010E9498ED4B015C014AE023
:100FB0004ADFCC2379F1C501B4010E9430E89B01DE
:100FC000AC01C701B6010E944EEC6B017C018EE2C0
:100FD00033DF20E030E040E251E4C701B6010E9477
:100FE00091E84B015C010E9493ED6B01770FEE08D5
:100FF000FF08C701B6018DDFC701B6010E9432E8C4
:101000009B01AC01C501B4010E944EEC6B017C0157
:10101000C150F9F6CF91FF90EF90DF90CF90BF9045
:10102000AF909F908F9008958FB7F8949091DE0DB8
:101030002091DD0D291759F0E92FF0E0E35AF24F26
:10104000208130E09F5F9F779093DE0D02C02FEFED
:101050003FEF8FBFC90108951F920F920FB60F92F5
:1010600011240BB60F922F933F938F939F93EF937F
:10107000FF932091C6009FB7F894E091DD0D81E0C9
:101080008E0F8F773091DE0D831731F0F0E0E35A49
:10109000F24F20838093DD0D9FBFFF91EF919F91D1
:1010A0008F913F912F910F900BBE0F900FBE0F901D
:1010B0001F901895CF92DF92EF92FF92CF93DF931C
:1010C000EC01C090E807D090E907E090EA07F090C3
:1010D000EB07A7019601688179818A819B810E9433
:1010E0002CE887FF04C0C882D982EA82FB82C090C4
:1010F000EC07D090ED07E090EE07F090EF07A70126
:1011000096016C817D818E819F810E942CE887FFF2
:1011100004C0CC82DD82EE82FF82C090F007D090C6
:10112000F107E090F207F090F307A70196016885B8
:1011300079858A859B850E942CE887FF04C0C88634
:10114000D986EA86FB86C0902502D0902602E090E0
:101150002702F0902802A7019601688179818A818F
:101160009B810E9475EE181624F4C882D982EA8207
:10117000FB82C0902902D0902A02E0902B02F090CE
:101180002C02A70196016C817D818E819F810E9436
:1011900075EE181624F4CC82DD82EE82FF82C090B8
:1011A0002D02D0902E02E0902F02F0903002A70185
:1011B0009601688579858A859B850E9475EE18164B
:1011C00024F4C886D986EA86FB86DF91CF91FF900A
:1011D000EF90DF90CF9008954F925F926F927F9241
:1011E0008F929F92AF92BF92CF92DF92EF92FF9237
:1011F0000F931F93CF93DF9300D000D0CDB7DEB70E
:101200007C01FC01E25DF24C149182E0E816F104ED
:1012100029F481E00E940DBC811123C16701CC0C2F
:10122000DD1CCC0CDD1CC6018E5D924C0E94074972
:101230004B015C01612F110F770B880B990B0E94FA
:1012400032E82B013C0120E030E040EC5FE3C501D7
:10125000B4010E9491E8A30192010E9491E8AB01C0
:10126000BC0100E010E09801C7010E9421BA92E0A1
:10127000E916F10479F48EE19DE30E94074920E02C
:1012800030E040EA50E40E942CE887FD09C08EE17E
:101290009DE303C0C6018A5E924C0E94074904C0C8
:1012A00060E070E080EA90E49B01AC01C301B20110
:1012B0000E9491E84B015C0120E030E0A9010E940E
:1012C0002CE8882309F458C000E010E09801B5012B
:1012D000A4017058C7010E9421BA86E0E0E6F3E05D
:1012E000DE01119601900D928A95E1F7F701EE0F5C
:1012F000FF1F81E090E08C0F9D1FE80FF91F808198
:10130000918118161906C4F0E8E3F4E484918F0182
:101310000F5F1F4F882319F08FDDF801F7CFE4EF3F
:10132000FCE384918F010F5F1F4F882319F084DD48
:10133000F801F7CF8AE090E0BC01990F880B990B78
:101340000E9432E89B01AC01F601EA59FC4F608132
:101350007181828193810E942BED2B013C01A501BB
:101360009401C501B4010E944FECAB01BC01930193
:101370008201C7010E9421BA81E0F701E056FB4FCC
:101380008083F701E351FB4F8083F601EF5BF24F5F
:101390001082118212821382C7010E94FFBDC60112
:1013A0008851934C0E940749860103501B4FF60158
:1013B000EB5CF24F20813181428153810E944FECDE
:1013C000F8016083718382839383F2E0EF16F10466
:1013D000D1F42091750E3091760E4091770E509198
:1013E000780E609105057091060580910705909132
:1013F00008050E944EEC60930505709306058093E6
:101400000705909308050E94FD48F601E35BF24F43
:10141000D601A350BB4F8D919D910D90BC91A02DF5
:1014200080839183A283B38382E0E816F104C9F438
:1014300080E026960FB6F894DEBF0FBECDBFDF91D9
:10144000CF911F910F91FF90EF90DF90CF90BF90C1
:10145000AF909F908F907F906F905F904F900C9483
:101460000DBC26960FB6F894DEBF0FBECDBFDF9140
:10147000CF911F910F91FF90EF90DF90CF90BF9091
:10148000AF909F908F907F906F905F904F90089556
:101490000F931F93CF93DF938C01E8E3F4E48491DF
:1014A000EF012196882319F0C7DCFE01F8CFB801BF
:1014B0008BED9CE30E94158282E2BEDC8AE0BCDCFC
:1014C00081E0DF91CF911F910F9108955F9AEDEE2A
:1014D000F4E010828A9A11829FB7F894A8E0B1E0F4
:1014E0008C9181608C939FBF1282129A08958C0117
:1014F000E3EDF3E38491EF012196882319F09CDC5E
:10150000FE01F8CFEBEBFCE38491EF0121968823F9
:1015100019F092DCFE01F8CF0E9406D1D7DF0E94BD
:101520008D6B61E0C8010E94F7D80E9407580E94A5
:101530003B7484E00E94FD5D8091FD108695869548
:10154000109233118093341187E692E00E94E85E96
:101550008091FD1086958695880F109233118093A7
:1015600034118CEA9CE30E94DB5E8091FD1086952D
:101570008695982F990F890F10923311809334110B
:101580008FE99CE30E94DB5E0E9425C38111D1CFCD
:101590002FEF8BE49DE1215080409040E1F700C0A7
:1015A0000000F8942FEF84E39CE0215080409040AD
:1015B000E1F700C000000E9406D1A895FECF4F922F
:1015C0005F926F927F928F929F92AF92BF92CF92D3
:1015D000DF92EF92FF920F931F93CF93DF930E94BE
:1015E000CD680E94975B6B017C0110913A02112338
:1015F00009F45FC08091290D90912A0D009709F49C
:1016000058C04091DF0D5091E00D6091E10D709157
:10161000E20D46015701841A950AA60AB70AB7FCDB
:101620005AC083309105F9F034F401970CF441C0AD
:10163000E8E3F4E406C0049709F03BC0E8E3F4E40F
:1016400026C08491EF012196882319F0F5DBFE0175
:10165000F8CFE1E2FCE38491EF012196882349F180
:10166000EBDBFE01F8CFE8E3F4E48491EF0121968F
:10167000882319F0E1DBFE01F8CFEAE0FCE3849176
:10168000EF0121968823A9F0D7DBFE01F8CF8491E2
:10169000EF012196882319F0CFDBFE01F8CFE2EFAE
:1016A000FBE38491EF012196882319F0C5DBFE014D
:1016B000F8CF212F30E0A8EEB3E00E943FECC60E39
:1016C000D71EE81EF91EC092DF0DD092E00DE09209
:1016D000E10DF092E20D8091AF06843010F40E948B
:1016E00047BF0E94975BC090310DD090320DE090C3
:1016F000330DF090340DC114D104E104F10459F11B
:1017000000912D0D10912E0D20912F0D3091300D47
:101710000C0D1D1D2E1D3F1D5B016C01A01AB10A91
:10172000C20AD30AD7FC17C0E3EDF3E38491EF01BB
:101730002196882319F080DBFE01F8CF60912B0DF4
:1017400070912C0D85E69CE30E9415828AE074DB83
:101750008CE59CE355C0C0903B02D0903C02E090E9
:101760003D02F0903E02C114D104E104F104D9F02D
:1017700000912D0D10912E0D20912F0D3091300DD7
:101780000C0D1D1D2E1D3F1DDC01CB01801B910B7F
:10179000A20BB30BB7FD07C090915A1180915B115A
:1017A000981709F460C18091E70D9091E80D909928
:1017B00002C0019604C0181619062CF401979093E4
:1017C000E80D8093E70D8091E70D9091E80D8E3E36
:1017D0009240BCF0E3EDF3E38491EF01219688237E
:1017E00019F02ADBFE01F8CFECE3FCE38491EF0172
:1017F0002196882319F020DBFE01F8CF83E39CE3D8
:1018000076DE6091130890915A1180915B119817C0
:1018100091F0E0915B118DE4E89FF0011124E5590E
:10182000F74F608180915B1190915A11891719F0DF
:101830008F5F8F70F9CF70E089E00E94985A809195
:10184000080E882309F4F9C000915B0210915C0234
:10185000D0915D02C0915E026091110870911208F2
:101860006E5F7F4F072E000C880B990B0E9432E8A9
:1018700098014D2F5C2F0E942CE887FDDEC0F09070
:101880005B11912CA12CB12CE12C8DE4882E809140
:101890005A11F81609F45BC08F2D90E0889EF00174
:1018A000899EF00D1124EC5DF74F428153816481D4
:1018B0007581452B462B472B81F4468157816085E6
:1018C0007185452B462B472B41F442855385648512
:1018D0007585452B462B472BA9F1889E9001899E43
:1018E000300D1124F901EC5DF74F6F0166857785A6
:1018F000808991890E9432E82B013C01F6016289BE
:101900007389848995890E9430E89B01AC01C301E9
:10191000B2010E942BEDF60123A134A145A156A1ED
:101920000E9491E83B016C019B01AC01692D7A2D6D
:101930008B2D9E2D0E942CE887FF04C0962CA72C8F
:10194000BC2CED2C81E08F0D8F70F82EA0CF209154
:101950005302309154024091550250915602692D24
:101960007A2D8B2D9E2D0E9491E89B01AC01B80130
:101970008D2F9C2F0E944FEC6B017C0198014D2F05
:101980005C2F0E942CE887FD14C000915702109133
:101990005802D0915902C0915A0298014D2F5C2FE4
:1019A000B601C7010E9475EE18161CF08601DE2DE7
:1019B000CF2DC090E30DD090E40DE090E50DF090B8
:1019C000E60DA7019601B8018D2F9C2F0E942CE8EF
:1019D00087FF1CC020E037ED43EA5CE3B8018D2FA0
:1019E0009C2F0E9491E84B015C0128E431EE4AE70C
:1019F0005FE3C701B6010E9491E89B01AC01C501FC
:101A0000B4010E944FEC8B01D82FC92FC801AD2F14
:101A1000BC2F8093E30D9093E40DA093E50DB0935C
:101A2000E60DB8018D2F9C2F0E9493ED7093120844
:101A30006093110880E00E94D3D00E9448D38CE5C7
:101A400091E1DF91CF911F910F91FF90EF90DF9087
:101A5000CF90BF90AF909F908F907F906F905F904E
:101A60004F900C94CE445F9A1092ED048A9A109293
:101A7000EE049FB7F894809108018160809308017B
:101A80009FBF1092EF04129A8ECECF93DF9380E027
:101A900090E00E9485D4CDE1DDE0688379838A837C
:101AA0009B8381E090E00E9485D46C837D838E834C
:101AB0009F8382E090E00E9485D4688779878A8737
:101AC0009B87DF91CF910895CF93DF930E940D49BB
:101AD000E091AE06F0E0E35FFA4F8081882371F079
:101AE000EFEEFBE38491EF012196882319F0A4D94E
:101AF000FE01F8CF8AE0DF91CF919EC9DF91CF91AF
:101B00000895CF93DF938FB7F8949091DE0D909363
:101B1000DD0D8FBFE6EEFBE38491EF012196882374
:101B200019F08AD9FE01F8CF8091190D90911A0D04
:101B3000A0911B0DB0911C0DBC01CD016F5F7F4FBB
:101B40008F4F9F4FE6D98AE077D9DF91CF91BCCFF5
:101B50003F924F925F926F927F928F929F92AF923D
:101B6000BF92CF92DF92EF92FF920F931F93CF938A
:101B7000DF93CDB7DEB72C970FB6F894DEBF0FBE5C
:101B8000CDBF5C01DC0159968D909C905A97F40171
:101B900081859285A385B4859C01AD012F5F3F4F60
:101BA0004F4F5F4F29873A874B875C87D501149643
:101BB000CD90DD90ED90FC901797C114D104E10415
:101BC000F10439F0BFEFCB1ADB0AEB0AFB0A312C28
:101BD00007C0F401C080D180E280F38033243394C5
:101BE000260137011D821E821F821886F40181851D
:101BF0009285A385B4852D813E814F815885281714
:101C000039074A075B0708F064C089859A85AB8568
:101C1000BC858C159D05AE05BF0550F482E0C82E2D
:101C2000D12CE12CF12C92E0492E512C612C712CFD
:101C30009E012F5F3F4FB701A601C4010E9444835C
:101C4000882309F446C089819A81AB81BC81892BA4
:101C50008A2B8B2B41F0260137019FEF491A590A35
:101C6000690A790A05C0C414D504E604F70491F0A2
:101C70002D813E814F8158852F5F3F4F4F4F5F4FE2
:101C80002D833E834F8358873FEFC31AD30AE30A5D
:101C9000F30AACCF0FEF1FEF2FEF3FE0B301A2012C
:101CA000C4010E94B382F82E882399F0D5011496BE
:101CB0004D915D916D917C9117974115510561058D
:101CC000710549F093018201C4010E94B382811120
:101CD00002C0F12C29C0D50114964D925D926D92EF
:101CE0007C921797332051F0D301C2010196A11DB8
:101CF000B11DF40180839183A283B383F5018589AB
:101D00009689A789B08D892B8A2B8B2B69F4D501F5
:101D100055964D925D926D927C92589711968C914A
:101D20001197806811968C938F2D2C960FB6F8948E
:101D3000DEBF0FBECDBFDF91CF911F910F91FF90FE
:101D4000EF90DF90CF90BF90AF909F908F907F905B
:101D50006F905F904F903F900895CF93DF93EC0189
:101D60008B818823B9F1898187FF30C06C857D859F
:101D70008E859F8541E00E947B82882359F1E88906
:101D800080E2E89FF0011124DF01A551B14F1097C7
:101D900009F18C91853EF1F08B81823050F44989B4
:101DA0005A896B897C895C964D935D936D937C9386
:101DB0005F978D899E89AF89B88DE551F14F938FDB
:101DC000828FB58BA48B89818F778983DF91CF91A7
:101DD0000C943B8281E0888380E0DF91CF9108956D
:101DE0008F929F92AF92BF92CF92DF92EF92FF922B
:101DF0000F931F93CF93DF93EC018B81811102C06E
:101E000080E077C009891A892B893C890417150756
:101E100026073707A8F36A017B01823029F4C886B8
:101E2000D986EA86FB860DC0C114D104E104F10411
:101E300051F41C821D821E821F82188619861A8602
:101E40001B8681E056C088849984AA84BB84E98D6E
:101E5000FA8D258530E0275F3F4FB501A401415041
:101E6000510961097109022E04C07695679557954D
:101E700047950A94D2F7D701C6010197A109B10984
:101E800004C0B695A795979587952A95D2F784179C
:101E90009507A607B70720F089288A288B2849F4D8
:101EA0004D895E896F89788D4C835D836E837F83D6
:101EB00004C0841B950BA60BB70B4C015D018E0172
:101EC0000C5F1F4F81149104A104B10409F4A7CF42
:101ED0004C815D816E817F819801898D9A8D0E94F0
:101EE000448391E0891A9108A108B1088111EACFD1
:101EF00087CFDF91CF911F910F91FF90EF90DF90EF
:101F0000CF90BF90AF909F908F9008952F923F9267
:101F10004F925F926F927F928F929F92AF92BF92F9
:101F2000CF92DF92EF92FF920F931F93CF93DF93A5
:101F300000D01F92CDB7DEB79C838B834B015A0133
:101F4000DC0113968C91811103C08FEF9FEFEAC0E3
:101F5000EB81FC81818180FFF8CFAB81BC81519600
:101F60000D911D912D913C91549718964D915D9135
:101F70006D917C911B97C501A0E0B0E068017901EB
:101F8000C41AD50AE60AF70AC816D906EA06FB06F5
:101F900018F45801A41AB50A75018B819C81049626
:101FA0009A838983612C92E0792EE114F10409F47B
:101FB0008BC0AB81BC8118964D915D916D917C91E8
:101FC0001B976A01B1E0DB22EB81FC8123811A01BE
:101FD0002B0189E056944794379427948A95D1F73A
:101FE000818D928D223061F4FC01828D938DA48DC0
:101FF000B58DBC01CD01620D731D841D951D4AC0B8
:10200000DC0114961C9111501221C114D10401F568
:1020100011111EC0452B462B472B59F4EB81FC8137
:1020200085899689A789B08D84839583A683B78394
:102030000FC0AB81BC8114964D915D916D917C91E7
:10204000179729813A810E944483882309F47DCF20
:10205000EB81FC81218D328D84819581A681B781B0
:102060000297A109B109F901058404C0880F991FDD
:10207000AA1FBB1F0A94D2F74685578560897189CC
:10208000840F951FA61FB71FBC01CD01610F711DE5
:10209000811D911D93012C193D0987012E153F05C6
:1020A00008F489010115F2E01F0771F52091EB108A
:1020B0003091EC104091ED105091EE1062177307C3
:1020C0008407950719F420C0C5012CC09401AB0109
:1020D000BC018091F4109091F51057D6882309F433
:1020E00034CF800E911EEB81FC8180859185A28585
:1020F000B385800F911FA11DB11D80879187A28795
:10210000B387E01AF10A51CF40E00E947B82882316
:1021100009F41BCFB6016551714FA801C4010E949B
:1021200061EFDFCF0F900F900F900F90DF91CF9165
:102130001F910F91FF90EF90DF90CF90BF90AF90E5
:102140009F908F907F906F905F904F903F902F90D7
:1021500008950F931F93CF93DF93FC0123812223D4
:1021600011F080E044C08B01EC01FB0187898031D4
:1021700039F18032B1F783E08B83F801428D538DC2
:10218000648D758D4D8B5E8B6F8B788F9E012F5E6E
:102190003F4FC8010E94C583882319F31A8F098F06
:1021A00081E089831C821D821E821F821886198607
:1021B0001A861B861C861D861E861F86188A17C0D7
:1021C00082E08B831D8A1E8A1F8A188EFB01808DF8
:1021D000918DA0E0B0E025E0880F991FAA1FBB1FDA
:1021E0002A95D1F7898B9A8BAB8BBC8BD7CFDF919C
:1021F000CF911F910F9108950F931F93CF93DF936A
:10220000EB01FC012381211102C080E040C022507B
:10221000223028F48FE28883198281E038C08C0153
:10222000FC01648575858685978540E00E947B82E8
:10223000882359F3F8014089F0E24F9FA00111244F
:102240009A012551314F232B01F320E030E090E03B
:102250006EE2F901E40FF51FE551F14F7081703224
:1022600071F02830310529F4DE01A90FB11D6C93FE
:102270009F5FDE01A90FB11D70817C939F5F2F5F6F
:102280003F4F2B30310529F7C90FD11D1882DF913F
:10229000CF911F910F910895CF93DF93EC015DDDF6
:1022A0001B82DF91CF9108950F931F93CF93DF93FC
:1022B0008B010E94975BEB01F2D48F3F49F00E94A3
:1022C000975B6C1B7D0B60177107B0F380E001C05A
:1022D00081E0DF91CF911F910F9108950F931F938C
:1022E000CF93DF93EC0189018C81833039F089E051
:1022F000440F551F661F771F8A95D1F79A01AB01CE
:1023000068E1CE01D3D4882311F086E02FC08EEF90
:102310008EBD80E090E00DB407FEFDCFF801E80F20
:10232000F91F20812EBD0DB407FEFDCF21812EBDEA
:102330000296811522E0920771F70DB407FEFDCFDA
:102340008FEFA8D48FEFA6D4AAD48B838F7185305A
:1023500029F083E18983CE0198D409C068E572E051
:10236000CE01A2DF182F811106C087E18983CE013B
:102370008CD410E00FC020E030E0A9016DE0CE0168
:1023800095D4811103C08BD4882311F086E1EECF60
:10239000CE017BD4812FDF91CF911F910F910895B2
:1023A0004F925F926F927F929F92AF92BF92CF9225
:1023B000DF92EF92FF920F931F93CF93DF931F92C1
:1023C000CDB7DEB78C017B016A01A22EDB015996E5
:1023D0008D919C915A97F801928F818F40E050E047
:1023E000BA01C701FDDC912CF70180859185A2859A
:1023F000B385418952896389748984179507A60733
:10240000B70708F063C025E0B695A795979587951F
:102410002A95D1F7F82FFF70BF2ED70113968C9114
:10242000823008F469C041E050E0BE016F5F7F4F29
:10243000C7016CDD019719F4898190E002C08FEF2C
:102440009FEF019609F458C0F70180859185A28518
:10245000B3854F96A11DB11D80879187A287B38751
:10246000F0E2BF9EC0011124BC016551714F61159E
:10247000710509F441C0DB012C91222319F0253E9E
:10248000D1F47CC191100EC04091EB105091EC1032
:102490006091ED107091EE10F801448755876687C2
:1024A0007787B08AFC01E551F14F8081882361F084
:1024B0009924939499CF4BE050E0C6010E9454EFC9
:1024C000892B09F091CF1AC0992493948A2D827494
:1024D000823491F4992009F49CC0D8015096BC90A4
:1024E00050971C966D917D918D919C911F9741E025
:1024F0000E947B82811180C080E043C1A7FCFCCF99
:10250000F0E2BF9EA00111249A012551314FD9015B
:102510001B968C91817121F08A2D827109F068C01F
:102520008091EB109091EC10A091ED10B091EE1015
:10253000F80184879587A687B787B08AFA01E551A5
:10254000F14F4489558960E070E0BA01552744276E
:10255000D80155964D935D936D937C935897828DDA
:10256000938DA0E0B0E0482B592B6A2B7B2BD80130
:1025700055964D935D936D937C935897D9011B9617
:102580008C91887159F4848D958DA68DB78DF80145
:10259000818B928BA38BB48B81E010C0803141F58D
:1025A00098012F5E3F4FD80159968D919C915A9773
:1025B0000E94C5838823E1F084E0F80183838A2D9B
:1025C0008F70D80111968C931197F801148215829F
:1025D0001682178218961D921D921D921C921B97AF
:1025E000A4FEC0C0C8010E947EC58111BBC084CFBB
:1025F000D80113961C9280CFF8016089F0E26F9F9A
:10260000B00111246551714F6115710509F08AC03F
:1026100073CFD70113968C911397823009F46CCF46
:1026200051968D919D910D90BC91A02D803E9F4F14
:10263000AF41B10508F060CFC7018ADA882309F4F9
:102640005BCF0E943B82882309F456CFD70159966D
:102650002D913C915A9714968D919D910D90BC911E
:10266000A02D0297A109B109F901058404C0880FC2
:10267000991FAA1FBB1F0A94D2F74684578460880B
:102680007188480E591E6A1E7B1E81E08093F310EC
:102690004092EB105092EC106092ED107092EE10A0
:1026A00080E092E0EBEEFEE0DF019C011D92215004
:1026B0003040E1F7BB24B394D7015996ED91FC91DA
:1026C0005A978481B81690F42BEE3EE0B301A20134
:1026D0004B0D511D611D711D8091F4109091F510ED
:1026E000FDDD882309F408CFB394E6CF80E092E0C3
:1026F000A0E0B0E0058404C0880F991FAA1FBB1F8B
:102700000A94D2F7F7014189528963897489840F49
:10271000951FA61FB71F818B928BA38BB48B6BEE7B
:102720007EE0B12C80E2DB011D928A95E9F78BE017
:10273000F601DB0101900D928A95E1F781E298E2C2
:10274000FB01918B808B20E038E037872687938BC5
:10275000828B918F808F378B268B0E943B828111D9
:10276000CFCECACEA5FE08C0F8014189528963893F
:102770007489C80135DB05C081E003C0911098CE93
:1027800083CE0F90DF91CF911F910F91FF90EF902B
:10279000DF90CF90BF90AF909F907F906F905F90B1
:1027A0004F9008952F923F924F925F926F927F9237
:1027B0008F929F92AF92BF92CF92DF92EF92FF9251
:1027C0000F931F93CF93DF93CDB7DEB7C554D109D5
:1027D0000FB6F894DEBF0FBECDBF3C015B018A018E
:1027E000322E1C8E1F8E19821C82672B11F410E072
:1027F000A7C0FC0183818111FACFFA0180818F3259
:1028000061F4CA018C010196F80120812F32D1F3C5
:10281000F50183818250823010F475010AC0618D08
:10282000728DCE01019695DC882309F3CE010196C5
:102830007C016E019CE1C90ED11C26014E01E7E32B
:102840008E0E911CFBE0F80D2596FFAF2597CE016B
:10285000019624969FAF8EAF24972696CFAE2697EB
:102860002D2C35C080E2819325969FAD25979E1330
:10287000F9CFD80190E027E04A2F3B2F8D918111AD
:1028800028C08FA9803209F4B2CF842F932F8C01F6
:10289000FC01208101962F32D1F3222309F44AC092
:1028A00021E0A401B701C6017BDD882309F49FCF95
:1028B000EA14FB0411F0C701EFDCC414D50499F14C
:1028C00026969FAD2697822D7601C92ED82EF4012B
:1028D000C9CF8F32B1F28E3219F0E1E3FDE30AC0C5
:1028E0002A3009F484CF98E02AE0C6CF3196381711
:1028F00009F47DCF34913111F9CF291708F477CF3E
:10290000813208F474CF8F3709F471CF31E0390F79
:10291000F401E90FF11D9FE9980F9A3108F48052F4
:102920008083932FA9CF23969FAD239724968FADB5
:102930002497CACF232DA401B701C30131DD182F7D
:10294000CE0101960E94694FCE014C960E94694FBC
:10295000812FCB5BDF4F0FB6F894DEBF0FBECDBF2C
:10296000DF91CF911F910F91FF90EF90DF90CF906B
:10297000BF90AF909F908F907F906F905F904F909F
:102980003F902F9008952F923F924F925F926F92B7
:102990007F928F929F92AF92BF92CF92DF92EF92EF
:1029A000FF920F931F93CF93DF9300D01F92CDB769
:1029B000DEB78C014B011A01DC0113968C91139741
:1029C0008130C1F411968C9181FF14C082FF18C030
:1029D000F801418952896389748980859185A2852E
:1029E000B38584179507A607B70751F0C801F8D932
:1029F000811106C081E0F80180838FEF9FEF2EC127
:102A0000610184C0D80159968D919C915A97FC011F
:102A1000248121502A013B0139E076946794579430
:102A200047943A95D1F7722E74207A01F1E0FF2293
:102A3000772009F477C080E092E08E199F09560153
:102A40008C159D0508F45C01D80159962D913C9197
:102A50005A9714968D919D910D90BC91A02D02973F
:102A6000A109B109F901058404C0880F991FAA1FA3
:102A7000BB1F0A94D2F74685578560897189840FF8
:102A8000951FA61FB71F9C01AD01270D311D411DCC
:102A9000511D29013A01A11432E0B30609F089C0A1
:102AA0008091EB109091EC10A091ED10B091EE1090
:102AB00084159505A605B70569F41092F3108FEFFC
:102AC0009FEFDC018093EB109093EC10A093ED103E
:102AD000B093EE109401B301A2018091F410909193
:102AE000F510FCDB882309F485CFF80180859185FA
:102AF000A285B3858A0D9B1DA11DB11D808791877D
:102B0000A287B3878A0C9B1CCA18DB08D8011896C9
:102B10004D915D916D917C911B97C114D10409F089
:102B200071CF7DC0E114F10409F085CF14964D9169
:102B30005D916D917C911797411551056105710566
:102B400059F455968D919D910D90BC91A02D0097B3
:102B5000A105B10541F521C09E012F5F3F4F0E94A5
:102B60004483882309F446CF89819A81AB81BC8153
:102B7000F801218D328DF9012789203139F4883F00
:102B8000FFEF9F07A105B10540F40DC0883F2FEF6F
:102B90009207A2072FE0B20730F0C8010E94A88D6B
:102BA000811149CF27CFF80184839583A683B7830A
:102BB00042CFE114F10419F5D80118964D915D91B9
:102BC0006D917C911B9751968D919D910D90BC912B
:102BD000A02D481759076A077B0788F00E943B829F
:102BE000882309F407CF81E08093F3104092EB1023
:102BF0005092EC106092ED107092EE1008C041E01F
:102C0000C301B2010E947B82882309F4F3CEA5019F
:102C1000B401C7018551914F0E9461EF66CF519673
:102C20008D919D910D90BC91A02D84179507A607BD
:102C3000B70740F4F801418B528B638B748B818111
:102C400080688183D80111968C9183FD02C0C101F7
:102C500005C0C80182D88111FACFCCCE0F900F9059
:102C60000F900F90DF91CF911F910F91FF90EF90F8
:102C7000DF90CF90BF90AF909F908F907F906F909C
:102C80005F904F903F902F90089561E0FC0180810C
:102C90000C942D5A8EBD0DB407FEFDCF08958FEF15
:102CA0008EBD0DB407FEFDCF8EB50895CF92DF9295
:102CB000EF92FF921F93CF93DF9300D01F92CDB777
:102CC000DEB76C01162FFC019281892F806A8695F0
:102CD0008CBD90FD03C081E0963009F480E08DBD8D
:102CE00060E0F601808129833A834B835C830E94F4
:102CF0002D5A6CE271E0C601D7DA812F8064CADFF9
:102D000088E1E82EF12C5C814B813A812981DA013E
:102D1000C9010E2C04C0B695A795979587950A947E
:102D2000D2F729833A834B835C83B4DFF8E0EF1A50
:102D3000F10829813A814B815C8188EFE8168FEF99
:102D4000F80629F7112321F0183021F08FEF03C086
:102D500085E901C087E89EDF1C3009F4A0DF10E0A0
:102D60009EDFF601838387FF04C01F3F11F01F5FC2
:102D7000F7CF0F900F900F900F90DF91CF911F9191
:102D8000FF90EF90DF90CF900895EF92FF920F9316
:102D90001F93CF93DF93EC0179018C81833039F05D
:102DA00089E0440F551F661F771F8A95D1F79A0156
:102DB000AB0161E1CE017ADF882329F084E08983C9
:102DC000CE0163DF35C00E94975B8B0168DF8B8388
:102DD0008F3F49F40E94975B601B710B6D3271400D
:102DE000A8F381E103C08E3F39F08FE08983CE01E3
:102DF0004CDF8FEF4FDF1CC08FEF8EBDF701D70187
:102E0000A150BE4F0DB407FEFDCF9EB591938EBD70
:102E1000EA17FB07B9F70DB407FEFDCF8EB58C930B
:102E20003EDF3DDFCE0131DF8FEF34DF81E001C0D7
:102E300080E0DF91CF911F910F91FF90EF90089567
:102E40008F929F92AF92BF92CF92DF92EF92FF92BA
:102E50000F931F93CF93DF9300D01F92CDB7DEB7B0
:102E600089E3882E8EE0982E91E2A92E9EE0B92E5D
:102E70000FEE1DE0C12CD12C7601C394F4016191B9
:102E80007191819191914F01F50121913191419180
:102E900051915F0129833A834B835C830E9430E820
:102EA00029813A814B815C810E9491E80E9498EDD2
:102EB000F80161937193819391938F01C616D706A0
:102EC000E806F90610F46B017C01F9E48F16FEE0C8
:102ED0009F06A1F66FEF7FEFCB01A70196010E943D
:102EE000F1EB2093040E3093050E4093060E5093A1
:102EF000070E0F900F900F900F90DF91CF911F91C1
:102F00000F91FF90EF90DF90CF90BF90AF909F9088
:102F10008F9008952F923F924F925F926F927F927F
:102F20008F929F92AF92BF92CF92DF92EF92FF92D9
:102F30000F931F93CF93DF9300D01F92CDB7DEB7CF
:102F40007B016A011901A1E2BEE02D913D914D91F5
:102F50005C91FC0160817181828193810E9491E882
:102F60000E9480EE2B013C010AE411E1D8016D932F
:102F70007D938D939C9313972091250E3091260E6F
:102F80004091270E5091280EF70160817181828156
:102F900093810E9491E80E9480EE4B015C01D80170
:102FA00014966D937D938D939C9317972091290E82
:102FB00030912A0E40912B0E50912C0EF60160811B
:102FC0007181828193810E9491E80E9480EE6B0161
:102FD0007C01D80118966D937D938D939C931B97DC
:102FE00020912D0E30912E0E40912F0E5091300ECB
:102FF000F10160817181828193810E9491E80E9438
:1030000080EED8011C966D937D938D939C931F97B2
:1030100069837A838B839C830E94A3D42FB7F8940F
:10302000EBE1F4E140825182628273828482958274
:10303000A682B782C086D186E286F38669817A81CC
:103040008B819C8164877587868797872FBF1092B5
:10305000361110923711109238111092391180E107
:10306000EAE3F1E1DF011D928A95E9F70F900F90F5
:103070000F900F90DF91CF911F910F91FF90EF90E4
:10308000DF90CF90BF90AF909F908F907F906F9088
:103090005F904F903F902F9008950F931F93CF9381
:1030A000DF93C1E2DEE001E115E029913991499118
:1030B000599160E070E080E89FE30E942BEDF801F9
:1030C00061937193819391938F01FEE0C133DF0788
:1030D00061F729E035E045E055E061E075E08DEF0E
:1030E00094E018DFDF91CF911F910F91A9CE2F921D
:1030F0003F924F925F926F927F928F929F92AF9288
:10310000BF92CF92DF92EF92FF920F931F93CF93D4
:10311000DF93CDB7DEB7C557D1090FB6F894DEBF40
:103120000FBECDBF3B014A015901EFA6FBAA0BAF71
:1031300021961FAF21973C2C2091210E3091220E19
:103140004091230E5091240EDC016D917D918D9163
:103150009C910E9491E80E9480EEAE966CAF7DAF8C
:103160008EAF9FAFAE972091250E3091260E4091E5
:10317000270E5091280EF301608171818281938125
:103180000E9491E80E9480EEE2966CAF7DAF8EAF18
:103190009FAFE2972091290E30912A0E40912B0E7D
:1031A00050912C0ED4016D917D918D919C910E9436
:1031B00091E80E9480EEE6966CAF7DAF8EAF9FAF38
:1031C000E69720912D0E30912E0E40912F0E5091AA
:1031D000300EF50160817181828193810E9491E8B6
:1031E0000E9480EE6A966CAF7DAF8EAF9FAF6A97FC
:1031F00080914A1190914B11A0914C11B0914D11B9
:10320000AE96CCACDDACEEACFFACAE97C81AD90A2A
:10321000EA0AFB0A80914E1190914F11A091501132
:10322000B0915111E2968CAC9DACAEACBFACE297C4
:10323000881A990AAA0ABB0A8091521190915311D7
:10324000A0915411B0915511E6960CAD1DAD2EAD67
:103250003FADE697081B190B2A0B3B0B0FAB18AFC2
:1032600029AF3AAF8091EE0D83FF0EC06A962CAD68
:103270003DAD4EAD5FAD6A97209356113093571117
:1032800040935811509359118091561190915711B4
:10329000A0915811B09159116A964CAC5DAC6EACCE
:1032A0007FAC6A97481A590A6A0A7B0A09F499C0DE
:1032B0008091E90D811145C0609198047091990445
:1032C00080919A0490919B040E9493ED072E000C2C
:1032D000880B990B0E9432E820913F023091400206
:1032E00040914102509142020E942CE887FF29C080
:1032F0006A968CAD9DADAEADBFAD6A978093561109
:1033000090935711A0935811B0935911E8E3F4E446
:1033100084918F010F5F1F4F882321F00E941C872B
:10332000F801F6CFE0E6FDE384918F010F5F1F4FB8
:10333000882321F00E941C87F801F6CF412C512CE4
:1033400032014BA65CA66DA67EA677FE0BC00027B9
:103350001127980104191509260937090BA71CA77D
:103360002DA73EA760912D0E70912E0E80912F0EED
:103370009091300E0E9493ED9B01AC01A8ECB0E05F
:103380000E942FEC2BA53CA54DA55EA562177307E7
:10339000840795074CF56A968CAD9DADAEADBFAD7B
:1033A0006A978093561190935711A0935811B09338
:1033B0005911E8E3F4E484918F010F5F1F4F8823D4
:1033C00021F00E941C87F801F6CFE1E4FDE384912F
:1033D0008F010F5F1F4F882321F00E941C87F80187
:1033E000F6CF412C512C3201D701C6018827B7FDF9
:1033F00083959927AA27BB27282EB7FE03C0E82F5D
:10340000E2602E2E0FA918AD29AD3AAD37FF03C0EB
:10341000122D1460212E77FE03C0222D2860222E4B
:10342000032D10E0C301B2010E9432E8F801EE0F53
:10343000FF1FEE0FFF1FED5BFD4F208131814281A9
:1034400053810E9491E82B013C01000F111FF801EC
:10345000EF5DFD4F60817181072E000C880B990B89
:103460000E9432E89B01AC01C301B2010E9491E8C5
:103470002AE037ED43E25CE30E9491E82B013C0136
:1034800020E030E0A9010E9475EE18164CF420E00F
:1034900030E040E05FE3C301B2010E944FEC08C09E
:1034A000A301920160E070E080E09FE30E944EEC97
:1034B0000E9493ED6CAF7DAF8EAF9FAF80915A119C
:1034C0008F5F8F706F968FAF6F9780915B116F9644
:1034D0000FAD6F97801303C00E94DF8AF6CFE09193
:1034E0005A110E2F10E01CA70BA71DE4E19FF0015D
:1034F0001124EC5DF74F108222A2D701C601F7FE1E
:1035000007C088279927DC018C199D09AE09BF09DE
:1035100082839383A483B5838DE40BA51CA5809F30
:10352000F001819FF00D1124EC5DF74FD501C4012E
:10353000B7FE07C088279927DC0188199909AA09CD
:10354000BB0986839783A087B1878DE40BA51CA553
:10355000809FF001819FF00D1124EC5DF74F8FA942
:1035600098ADA9ADBAADB7FF07C0B095A09590953D
:1035700081959F4FAF4FBF4F82879387A487B587B1
:103580008DE40BA51CA5809FF001819FF00D1124F7
:10359000EC5DF74F2CAD3DAD4EAD5FAD2687378767
:1035A000408B518B428153816481758106811781E3
:1035B00020853185041715072607370714F48A017B
:1035C0009B018DE4ABA5BCA58A9FF0018B9FF00DFC
:1035D0001124EC5DF74F82859385A485B58580170E
:1035E0009107A207B30764F48CAD9DADAEADBFAD3E
:1035F00080179107A207B30764F4D901C8010DC071
:103600000CAD1DAD2EAD3FAD081719072A073B07BE
:1036100024F08CAD9DADAEADBFAD2DE40BA51CA5CA
:10362000209FF001219FF00D1124EC5DF74F828B5C
:10363000938BA48BB58B0697A105B10510F40C9460
:1036400018A5DF01A95BBF4F809113089091140862
:103650008D939C933182452B462B472B09F05F9825
:103660008DE40BA51CA5809FF001819FF00D112416
:10367000EC5DF74F86819781A085B185892B8A2BD8
:103680008B2B09F08A988DE40BA51CA5809FF00177
:10369000819FF00D1124EC5DF74F82859385A48501
:1036A000B585892B8A2B8B2B41F09FB7F89480919D
:1036B00008018E7F809308019FBF2CAD3DAD4EADBC
:1036C0005FAD232B242B252B71F08091030E8823D3
:1036D00019F081508093030E31100EC0129880E2D1
:1036E0008093030E09C02090490E30904A0E00913D
:1036F0004B0E10914C0E08C020904D0E30904E0E87
:1037000000914F0E1091500E9101A8016FA57BA959
:103710008BAD21969FAD21970E942CE887FD02C0BA
:103720000C9410A5C701B6010E9432E82091110542
:103730003091120540911305509114050E9491E8B3
:103740006FA778AB89AB9AAB698B7A8B8B8B9C8B91
:10375000C501B4010E9432E820911505309116058B
:1037600040911705509118050E9491E84B015C01AA
:103770006D8B7E8B8F8B988F6FA978AD89AD9AAD4D
:103780000E9432E82091190530911A0540911B05DD
:1037900050911C050E9491E86B017C01698F7A8F22
:1037A0008B8F9C8F20911D0530911E0540911F0528
:1037B00050912005C301B2010E9491E86D8F7E8F68
:1037C0008F8F98A32DE44BA55CA5249FF001259F26
:1037D000F00D1124EC5DF74F4280538064807580BA
:1037E00056E04516510461047104E4F446805780A4
:1037F00060847184A6E04A1651046104710494F453
:103800004284538464847584B6E04B165104610489
:10381000710444F4DC01CB01BF7787A790ABA1AB67
:10382000B2AB34C02FA538A949A95AA9CA01B90118
:103830000E9491E82B013C01A5019401C501B4014E
:103840000E9491E89B01AC01C301B2010E944FECC0
:103850004B015C01A7019601C701B6010E9491E8E6
:103860009B01AC01C501B4010E944FEC0E94BAEE6D
:103870002DE44BA55CA5249FF001259FF00D11249C
:10388000EC5DF74F67A770AB81AB92AB8DE4ABA556
:10389000BCA58A9FF0018B9FF00D1124EC5DF74FC2
:1038A00027A530A941A952A960E070E080E89FE314
:1038B0000E942BED26966CAF7DAF8EAF9FAF269703
:1038C0009B01AC01B101C8010E9491E86B017C0130
:1038D00080915A1190915B11891B8F702B968FAF3D
:1038E0002B97A701960160E074E284E799E40E94B7
